:1000000012EF3BF0000000000000000000000000C4
:100010000000000000000000361D0000000000008D
:1000200000000000000000000000000000000000D0
:100030000000000000000000000000000000F31CB1
:1000400000000000000000009826000000000000F2
:1000500000000000000000000000000000000000A0
:100060000000000000000000000000000000000090
:100070000000000000000000461D0000000000001D
:100080000000000000000000000000000000000070
:100090000000000000000000000000000000000060
:0C00A00000000000000000000000000054
:0C00AC00000E3D01E1BF010E006E1200CD
:0C00B800000E3D01F9BF010E006E1200A9
:0400C400F9DF12004E
:0400C800F1DF120052
:1000CC00FBDF005202E10000FBD762000BFBEAFDF4
:0200DC00120010
:1000DE00F4DF005202E10000FBD762000BFBD2FD01
:0200EE001200FE
:0800F000C1CAC2FAF4DF1200DC
:0800F800C1CAC2FAF0DF1200D8
:08010000C1CAC2FAE3DF1200DC
:100108000B820BAE8EEF00F003680268016800688E
:080118000A360232FF0E12004C
:100120000B840BAE9BEF00F0010E036E026A016AB6
:0A013000006A0A360232FF0E1200C8
:08013A00C1CAC2FAC6DF1200BF
:0E014200026A016A006A086A036A000E12006F
:080150000AAE029E000E12002F
:100158000CB0EEEF00F00CA294EF01F00E6A000E66
:10016800026405EF01F0F00E0214D8A4D0EF00F0FD
:10017800023A01380F0B02260138F00B016E0038E5
:100188000F0B01260038F00B006E08380F0B002605
:100198000838F00B086E0E84D89002BEE9EF00F024
:1001A80008360036013602360E2A02BEE9EF00F0A4
:1001B80008360036013602360E2A02BEE9EF00F094
:1001C80008360036013602360E2A0E5003648AEFCE
:1001D80001F0035E0BBC08AE8FEF01F0D880800EF3
:1001E80008640030000E002201220222D8A08FEFFE
:1001F80001F0023201320032034A94EF01F08FEF2E
:1002080001F001C002F000C001F008C000F0086A67
:10021800000E0E8602643CEF01F0F00E0214D8A422
:1002280024EF01F0023A01380F0B02260138F00BD7
:10023800016E00380F0B01260038F00B006E0E849B
:10024800D89002BEE9EF00F00036013602360E2AD9
:1002580002BEE9EF00F00036013602360E2A02BE71
:10026800E9EF00F00036013602360E2AE9EF00F019
:1002780001C002F000C001F0006A000E0E960E8860
:10028800026469EF01F0F00E0214D8A454EF01F0F3
:10029800023A01380F0B02260138F00B016E0E846A
:1002A800D89002BEE9EF00F0013602360E2A02BEEF
:1002B800E9EF00F0013602360E2A02BEE9EF00F03F
:1002C800013602360E2AE9EF00F001C002F0016A99
:1002D800000E0E86026499EF01F0F00E0214D8A405
:1002E80078EF01F0023A0E84D89002BEE9EF00F0F0
:1002F80002360E2A02BEE9EF00F002360E2A02BECE
:10030800E9EF00F002360E2AE9EF00F0010E0C6E5C
:1003180003DF9CEF01F0020E0C6E16DF9CEF01F07C
:10032800040E0C6EEDDE9CEF01F0080E0C6E05DF7E
:020338001200B1
:10033A00D250026ED29E0500FF6A0150FE6E005036
:08034A00FD6E02BED28E12000E
:100352006200C7F7E1FF6200CBF7E2FF620003FB36
:0E036200E6FFEFC900F0F0C901F0E6DF12007F
:100370000C6A0E6A0250D8A4D1EF01F001C002F05D
:1003800000C001F0006A0E860250D8A4D1EF01F03F
:1003900001C002F0016A0E960E880250D8B4E3EF55
:1003A00001F00E50035ED8A4D8A0E8EF01F0D89079
:1003B00002BEEDEF01F0003601360236032ED8EF13
:1003C00001F0E8EF01F0010E0C6EBBDEF0EF01F082
:1003D000020E0C6EA5DEF0EF01F0040E0C6EB8DE1E
:0203E000120009
:0803E2000B6A0B86FF0E1200EE
:1003EA000B800BAE01EF02F0026A0AAEFF0E026E3C
:0C03FA00016E006E0A360232FF0E120087
:10040600025006180E6E086A096A0B6A03500764E2
:10041600F6EF02F006500A6E068E028E03500B6E41
:100426000750036E000E0B6446EF02F00B50075E9A
:10043600D8B4E7EF02F0070E0764B5EF02F0075EE7
:1004460000C008F001C000F002C001F0026A074EC9
:10045600E7EF02F007648AEF02F0075E00C008F0DB
:1004660001C000F0016A074EE7EF02F0076468EF8B
:1004760002F0075E00C008F0006A074EE7EF02F0E0
:1004860007644FEF02F00AC002F005C001F004C095
:1004960000F0086A10EF04F0030E07645AEF02F04A
:1004A600075E08380F0B086E074EE7EF02F0D8908C
:1004B6000832074EE7EF02F0D8900832074EE7EF12
:1004C60002F0D8900832E7EF02F0030E076479EFE6
:1004D60002F0075E08380F0B086E0038F00B08268E
:1004E60000380F0B006E074EE7EF02F0D89000328F
:1004F6000832074EE7EF02F0D89000320832074E76
:10050600E7EF02F0D89000320832E7EF02F0030E70
:100516000764A1EF02F0075E08380F0B086E00387B
:10052600F00B082600380F0B006E0138F00B002682
:1005360001380F0B016E074EE7EF02F0D89001323B
:1005460000320832074EE7EF02F0D890013200324F
:100556000832074EE7EF02F0D89001320032083237
:10056600E7EF02F0030E0764D2EF02F0075E0838E9
:100576000F0B086E0038F00B082600380F0B006EC4
:100586000138F00B002601380F0B016E0238F00B14
:10059600012602380F0B026E074EE7EF02F0D890E5
:1005A6000232013200320832074EE7EF02F0D890ED
:1005B6000232013200320832074EE7EF02F0D890DD
:1005C6000232013200320832096A000E0EAEDBEF4B
:1005D60003F0081E001E011E021E082A0022012228
:1005E6000222DBEF03F00750D8A4FCEF02F010EF75
:1005F60004F0096A02C00AF0028E068E0750035CF8
:10060600076ED8B4CEEF03F0070E07649CEF03F035
:10061600075E0450096E0550046E0650056E066AA4
:10062600074ECEEF03F0070E076471EF03F0075E87
:100636000450096E0550046E056A074ECEEF03F0AE
:10064600070E07644FEF03F0075E0450096E046A55
:10065600074ECEEF03F0070E076436EF03F00AC02D
:1006660002F010EF04F0030E076441EF03F0075E9B
:1006760009380F0B096E074ECEEF03F0D8900932FA
:10068600074ECEEF03F0D8900932074ECEEF03F0B7
:10069600D8900932CEEF03F0030E076460EF03F043
:1006A600075E09380F0B096E0438F00B092604386B
:1006B6000F0B046E074ECEEF03F0D89004320932CA
:1006C600074ECEEF03F0D89004320932074ECEEF34
:1006D60003F0D89004320932CEEF03F0030E07641C
:1006E60088EF03F0075E09380F0B096E0438F00B2C
:1006F600092604380F0B046E0538F00B042605385E
:100706000F0B056E074ECEEF03F0D890053204327C
:100716000932074ECEEF03F0D89005320432093283
:10072600074ECEEF03F0D890053204320932CEEFF1
:1007360003F0030E0764B9EF03F0075E09380F0BE9
:10074600096E0438F00B092604380F0B046E0538C1
:10075600F00B042605380F0B056E0638F00B052640
:1007660006380F0B066E074ECEEF03F0D890063212
:10077600053204320932074ECEEF03F0D890063226
:10078600053204320932074ECEEF03F0D890063216
:10079600053204320932086A000E0EAEDBEF03F0B2
:1007A600091E041E051E061E092A0422052206220B
:1007B6000950082604500022055001220650022244
:1007C6000EBEF2EF03F0D8A001EF04F002320132C0
:1007D60000320832033E01EF04F00BEF04F0D8B00C
:1007E60006EF04F0000E081E001E011E021E082A57
:1007F6000022012202220A7E06EF04F0010E0C6E90
:10080600A8DC12EF04F0020E0C6EA3DC12EF04F06B
:10081600040E0C6E76DC12EF04F0000E0C6E120065
:10082600BFCA00F00A01BF07005232E06200EFFAC9
:10083600E9FF6200F3FAEAFFEE50000A10E06200F8
:10084600EFFAE9FF6200F3FAEAFF6200F7FAD9FF6E
:100856006200FBFADAFFEE50DE1801E113D0620007
:10086600EFFAE9FF6200F3FAEAFF6200F7FAD9FF4E
:100876006200FBFADAFFDE50EE5C006E016A000EE3
:10088600015A08D00A01BB4BBC2BBD4BBE2BC8D7A7
:06089600006A016A120075
:10089C000B6A0350D8B494EF04F002500A6E028E27
:1008AC008E0E035E03AE98EF04F0036C080E035C2F
:1008BC00D8A073EF04F0036E013602C001F0026A97
:1008CC00080E035CD8A073EF04F0036E0136016AC6
:1008DC000350D8A4D8907DEF04F00350D8B47DEF2A
:1008EC0004F0D89002320132032E77EF04F00BBCE7
:1008FC0001A08AEF04F0D8A08AEF04F0012AD8B442
:10090C00022A02BEA7EF04F00AAEACEF04F0021EFE
:10091C00011E012AD8B4022AACEF04F0026A016A63
:10092C00ACEF04F00B800BAEB0EF04F0026A0AAE31
:10093C00B0EF04F0FF0E026E016E0A360232B0EF19
:10094C0004F0010E0C6E4BDDB2EF04F0000E0C6ED9
:10095C00B2EF04F0FF0E0C6E0150006E0250016EEF
:02096C00120077
:10096E000B6A0C6A0A6A086A0350D8B43FEF05F0A6
:10097E00028E9E0E035E03BECAEF04F0D8B4CAEF19
:10098E0004F02FEF05F0036C080E035CD8A0FCEF0B
:10099E0004F0036E083600C008F001C000F002C07B
:1009AE0001F0026A080E035CD8A0FCEF04F0036E9F
:1009BE00083600C008F001C000F0016A080E035CA2
:1009CE00D8A0FCEF04F0036E083600C008F0006AF1
:1009DE00080E035CD8A0FCEF04F0036E0836086A1C
:1009EE000350D8A4D89008EF05F00350D8B408EF00
:1009FE0005F0D8900232013200320832032E00EF99
:100A0E0005F00BBC08A019EF05F0D8A019EF05F002
:100A1E00082AD8B4002AD8B4012AD8B4022A02BEB1
:100A2E0043EF05F00AAE3FEF05F0021E011E001E59
:100A3E00081E082AD8B4002AD8B4012AD8B4022A2B
:100A4E003FEF05F0026A016A006A086A3FEF05F09F
:100A5E000B800BAE48EF05F0026A0AAE48EF05F0C8
:100A6E00026E016E006E086E0A36023248EF05F015
:100A7E00000E0C6A49EF05F0010E0C6EAFDC49EF6B
:100A8E0005F0FF0E0250036E0150026E0050016E13
:060A9E000850006E12007A
:100AA400D29E3901E585550EE66FAA0EE66FE58301
:020AB40012002E
:100AB60000C008F00150006E016A026A036A0B6A00
:100AC6000C6A016A026A036A960E036E0A6A00AE2F
:100AD60073EF05F0081E001E082AD8B4002A0A8EF5
:100AE60000C001F008C000F0086A026A3EDC12008D
:060AF600067E86DC120002
:100AFC00BBCA02F0BCCA03F002C000F003C001F094
:100B0C00024A032A600003F0E9FF600007F0EAFFE5
:100B1C00EE5201E0F1D70A01BB51025C006EBC51F0
:0E0B2C000358016E010E005E000E015A120009
:100B3A00086A096A000E0762036425EF06F002508C
:100B4A0006180A6E075003267E0ED8A0B3EF05F0EA
:100B5A00035ED8B02AEF06F0B7EF05F0035ED8A01F
:100B6A002FEF06F0028E068E02C00EF001C00BF0C7
:100B7A0000C00DF0005004026F00D0FF0CF00150CD
:100B8A0005026F00D0FF00F06F00CCFF08F00402EE
:100B9A00F3500C26F4500822000E00220D500502D4
:100BAA00F3500C26F4500822000E002202500402D0
:100BBA00F3500826F450002202500502016A000E82
:100BCA000122F3500026F45001220D500602F35080
:100BDA000826F4500022026A000E012202220B505B
:100BEA000602F3500026F4500122000E02220E5093
:100BFA000602F3500126F450022202BE0DEF06F05F
:100C0A0008360036013602360306D8B42FEF06F04E
:100C1A0020EF06F0D880800E08640030000E002213
:100C2A0001220222D8A020EF06F00232013200325D
:100C3A00034A2AEF06F00AAE029E000E32EF06F0D1
:100C4A00010EA1EC00F032EF06F0020E84EC00F087
:0C0C5A0032EF06F0040E90EC00F01200E7
:0E0C6600550E3A01BF6FAA0EBF6FBF8112007C
:100C74000450000A12E10550000A0FE10650000A70
:100C84000CE10750000A09E1FF0E006EFF0E016E31
:100C94007F0E026EFF0E036EA8D0086A096A075021
:100CA400D8B4E5EF06F00350D8B4EAEF06F00250EA
:100CB40006180A6E028E068E0E6A02C008F001C083
:100CC4000CF000C00DF004500D5E0550D8A0053C9A
:100CD4000C5E0650D8A0063C085E086A0C6A0D6AD1
:100CE400D8A07CEF06F0D8900232013200320832EC
:100CF400010E0E6E0750035ED8A089EF06F07E0E3B
:100D04000E240326D8B0EFEF06F08FEF06F07E0E28
:100D14000E240326D8A0F4EF06F0180E0B6E0D3641
:100D24000C3608360036013602360E360450005EA4
:100D34000550D8A0053C015E0650D8A0063C025ED2
:100D440006340E120EA0AAEF06F00D80B5EF06F0E1
:100D5400045000260550D8B0053C01260650D8B0F2
:100D6400062802260D900B2E91EF06F0DBEF06F01D
:100D7400D8900036013602360E360450005E055017
:100D8400D8A0053C015E0650D8A0063C025E06349D
:100D94000E10010B0D26D8B00C2AD8B4082AD8A4FA
:100DA400DBEF06F008320C320D32032AD8B4EFEF31
:100DB40006F00AAE089E0850026E0C50016E0D50EB
:100DC400006EF7EF06F0010EF1EC01F0F7EF06F01C
:100DD400020EA1EC00F0F7EF06F0040E84EC00F034
:0C0DE400F7EF06F0080E90EC00F0120093
:0E0DF000550E3A01BF6FAA0EBF6FBF911200E1
:100DFE006200EFFAE9FF6200F3FAEAFFEE500A0131
:100E0E00BD1905E1BBCA00F0BCCA01F013D0BBCAC4
:100E1E0000F0BCCA01F0BB4BBC2B600003F0E9FF35
:100E2E00600007F0EAFF6F00B8FF00F00052E0E14B
:060E3E00006A016A1200C7
:100E44000A6A0350D8A40A800750D8A40A820A5018
:100E5400D8B485EF07F0030AD8B43EEF07F00AB020
:100E640039EF07F006AE83EF07F081EF07F002AE2B
:100E740081EF07F083EF07F00250800B0A6E029EA9
:100E84000650800B069E0A18D8B44FEF07F00A509C
:100E9400D8B481EF07F083EF07F00750035CD8B4B0
:100EA40059EF07F0D8A075EF07F07BEF07F0065075
:100EB400025CD8B463EF07F0D8A075EF07F07BEFBE
:100EC40007F00550015CD8B46DEF07F0D8A075EFBA
:100ED40007F07BEF07F00450005CD8B485EF07F00F
:100EE400D8B07BEF07F00A52D8B483EF07F081EF54
:100EF40007F00A52D8B481EF07F083EF07F0D880E7
:0E0F04001200D8901200D880D884120012007B
:100F12000A01BE6B6200EFFAE9FF6200F3FAEAFF30
:100F22006F00B8FFBDFABD51000A10E0BDCAC0FA99
:100F3200A9EC01F00A01BE2BBE51BB25E96E000EE1
:0E0F4200BC21EA6E6F00B8FFBDFAEDD71200B9
:100F5000086A096A100E0C6E01340836093604500E
:100F6000085E0550D8A0053C095ED8B007D00450F3
:100F700008260550D8B0053C0926D8900036013621
:060F80000C2EEAD712005E
:100F86000050086E0150006E016A026A036A0B6A1D
:100F96000C6A960E036E0A6A00C001F008C000F0E3
:0A0FA600086A026AB8EC01F01200BC
:100FB0000A01A86B050EA85D0AE2A851A625E16EFC
:100FC000000EA721E26E200EE66EA82BF3D7A851E3
:100FD000A625E16E000EA721E26EE66AA807A851D9
:100FE000A625A96F000EA721AA6F0A0E046E000E97
:100FF000056EA4CA00F0A5CA01F0AADF08C000F07F
:1010000009C001F0300E00266200A7FAE1FF62007D
:10101000ABFAE2FF600003F0E6FF0A0E046E000E7A
:10102000056EA4CA00F0A5CA01F092DF00C0A4FAC0
:1010300001C0A5FA000E011802E1000E001801E13E
:0810400002D0A807CCD7120072
:101048003F013E9FA4CA04F0A5CA05F0A6CA06F04F
:10105800A7CA07F0000E006E000E016E700E026E39
:10106800830E036EEBDE010ED8B0000E006E005248
:1010780046E0A4CA00F0A5CA01F0A6CA02F0A7CAB1
:1010880003F03F0E046E350E056E060E066E810ED9
:10109800076E4FDD68DC00C0E4F101C0E5F102C075
:1010A800E6F103C0E7F1E40E0701C36F010EC46F58
:1010B800020EC325E96E000EC421EA6E6F00A7FF79
:1010C800E9FF6F00ABFFEAFF6F00BBFF3DFF010EBA
:1010D800C325E96E000EC421EA6E6F00A7FFE9FF81
:1010E8006F00ABFFEAFF6F00BBFF3CFF61000FFF23
:1010F800E9FF610013FFEAFF6F00BBFF3BFF12002F
:101108000D0E0A01C16F80EC00F00A0E0A01C16FD2
:0611180080EC00F0120063
:10111E000050086E0150006E0250016E0350026EB8
:10112E00036A0B6A0C6A9E0E036E0A6A020E0C6E3E
:06113E00ACEC00F0120011
:101144000A01AA51000805E3070EAB6F000EAC6F4D
:1011540012D0AA51160805E2170EAD6F000EAE6F3D
:1011640006D0AA51010FAD6FAE6B000EAE23ADCA0F
:10117400ABFAAECAACFAABCAB5FAACCAB6FAAF6B44
:10118400B06B046A056A066A076AA4CA00F0A5CAB5
:1011940001F0A6CA02F0A7CA03F052DE010ED8B0CD
:1011A400000E006E00520BE06200A3FAE1FF620041
:1011B400A7FAE2FF2D0EE66EA84BA92BA67FA4CAC0
:1011C40004F0A5CA05F0A6CA06F0A7CA07F0006A8B
:1011D400016A026A036A34DE010ED8B0000E006EA2
:1011E400005235E0000E046E000E056E000E066E11
:1011F4007F0E076EA4CA00F0A5CA01F0A6CA02F0C9
:10120400A7CA03F01DDE010ED8B0000E006E005216
:101214001EE0A4CA00F0A5CA01F0A6CA02F0A7CA3B
:1012240003F0000E046E000E056E200E066E820E94
:10123400076E81DC00C0A4FA01C0A5FA02C0A6FAB8
:1012440003C0A7FA010EAF5F000EB05BCBD7000E50
:10125400046E000E056E200E066E820E076EA4CA82
:1012640000F0A5CA01F0A6CA02F0A7CA03F0E8DD9F
:10127400000ED8B0010E006E00521DE0000E046E88
:10128400000E056E200E066E820E076EA4CA00F0D4
:10129400A5CA01F0A6CA02F0A7CA03F0E9DC00C09F
:1012A400A4FA01C0A5FA02C0A6FA03C0A7FA0A016B
:1012B400AF4BB02BCCD7AF51B527B051B623010EED
:1012C400B16F000EB26F000EB76F000EB86F000E54
:1012D400B96F7F0EBA6F800EB219006E800EB61908
:1012E400005C02E1B551B15D1DE2000E046E000E1A
:1012F400056E200E066E820E076EB7CA00F0B8CADD
:1013040001F0B9CA02F0BACA03F0B2DC00C0B7FAFD
:1013140001C0B8FA02C0B9FA03C0BAFA0A01B14B63
:10132400B22BD9D7000E046E000E056E000E066EA9
:10133400800E076EB7CA00F0B8CA01F0B9CA02F04D
:10134400BACA03F095DCA4CA04F0A5CA05F0A6CA7B
:1013540006F0A7CA07F003EC02F000C0A4FA01C02B
:10136400A5FA02C0A6FA03C0A7FA000E046E000E86
:10137400056E200E066E820E076E62DD000ED8B07A
:10138400010E006E00520BE0000E0A01A46F000E65
:10139400A56F000EA66F7F0EA76FAF4BB02B0A018F
:1013A400800EB019006E800E005C02E1000EAF5D8D
:1013B4003EE26200A3FAE1FF6200A7FAE2FF300E08
:1013C400E66EA84BA92B6200A3FAE1FF6200A7FA1C
:1013D400E2FF2E0EE66EA84BA92B800EB619006E06
:1013E400800E005C02E1000EB55D04E2B551AF5F12
:1013F400B651B05BFF0EB16FFF0EB26F800EB01925
:10140400006E800EB219005C02E1B151AF5D0FE2D3
:101414006200A3FAE1FF6200A7FAE2FF300EE66E73
:10142400A84BA92B010EB15F000EB25BE7D7B16BDD
:10143400B26B800EB219006E800EB619005C02E128
:10144400B551B15D68E2A4CA00F0A5CA01F0A6CA0C
:1014540002F0A7CA03F04EEC04F000C0B3FA01C0D6
:10146400B4FA300E00266200A3FAE1FF6200A7FA84
:10147400E2FF600003F0E6FFA84BA92BB251B019BC
:1014840002E1AF51B1190AE16200A3FAE1FF62007F
:10149400A7FAE2FF2E0EE66EA84BA92BB3CA00F002
:1014A400B4CA01F05BEC05F000C0B7FA01C0B8FAA9
:1014B40002C0B9FA03C0BAFA00C004F001C005F0D2
:1014C40002C006F003C007F0A4CA00F0A5CA01F0E8
:1014D400A6CA02F0A7CA03F07BEC05F000C0A4FA88
:1014E40001C0A5FA02C0A6FA03C0A7FA000E046E52
:1014F400000E056E200E066E820E076E9DEC05F042
:1015040000C0A4FA01C0A5FA02C0A6FA03C0A7FA53
:10151400B14BB22B8ED76200A3FAE1FF6200A7FAA7
:06152400E2FFE66A12007E
:10152A000A01A451170802E2006A11D3A551000A60
:10153A00D8A4B2D0A75301E056DC60D062009BFA6F
:10154A0000FAA5D062009BFA01FAA1D062009BFAC8
:10155A0002FA9DD062009BFA03FA99D062009BFAC4
:10156A0004FA95D062009BFA05FA91D062009BFAC0
:10157A0006FA8DD062009BFA07FA89D062009BFABC
:10158A0008FA85D062009BFA09FA81D062009BFAB8
:10159A000AFA7DD062009BFA0BFA79D062009BFAB4
:1015AA000CFA75D062009BFA0DFA71D062009BFAB0
:1015BA000EFA6DD062009BFA0FFA69D062009BFAAC
:1015CA0010FA65D062009BFA11FA61D062009BFAA8
:1015DA0012FA5DD062009BFA13FA59D062009BFAA4
:1015EA0014FA55D062009BFA15FA51D062009BFAA0
:1015FA0016FA4DD062009BFA17FA49D00A01A45193
:10160A00000A9CE0A451010A9DE0A451020A9EE04E
:10161A00A451030A9FE0A451040AA0E0A451050AB8
:10162A00A1E0A451060AA2E0A451070AA3E0A4512A
:10163A00080AA4E0A451090AA5E0A4510A0AA6E0EE
:10164A00A4510B0AA7E0A4510C0AA8E0A4510D0A60
:10165A00A9E0A4510E0AAAE0A4510F0AABE0A451D2
:10166A00100AACE0A451110AADE0A451120AAEE08E
:10167A00A451130AAFE0A451140AB0E0A451150A08
:10168A00B1E0A451160AB2E0A451170AB3E00A0164
:10169A00A75302E033EC06F00A01A551010AD8A4C7
:1016AA0053D1A75302E0F8EC06F0A4D0620093FAF3
:1016BA00C0FA45D1620093FAC1FA41D1620093FAA5
:1016CA00C2FA3DD1620093FAC3FA39D1620093FAA1
:1016DA00C4FA35D1620093FAC5FA31D1620093FA9D
:1016EA00C6FA2DD1620093FAC7FA29D1620093FA99
:1016FA00C8FA25D1620093FAC9FA21D1620093FA95
:10170A00CAFA1DD1620093FACBFA19D1620093FA90
:10171A00CCFA15D1620093FACDFA11D1620093FA8C
:10172A00CEFA0DD1620093FACFFA09D1620093FA88
:10173A00D0FA05D1620093FAD1FA01D1620093FA84
:10174A00D2FAFDD0620093FAD3FAF9D0620093FA82
:10175A00D4FAF5D0620093FAD5FAF1D0620093FA7E
:10176A00D6FAEDD0620093FAD7FAE9D0620093FA7A
:10177A00D8FAE5D0620093FAD9FAE1D0620093FA76
:10178A00DAFADDD0620093FADBFAD9D0620093FA72
:10179A00DCFAD5D0620093FADDFAD1D0620093FA6E
:1017AA00DEFACDD0620093FADFFAC9D0620093FA6A
:1017BA00E0FAC5D0620093FAE1FAC1D0620093FA66
:1017CA00E2FABDD0620093FAE3FAB9D0620093FA62
:1017DA00E4FAB5D0620093FAE5FAB1D0620093FA5E
:1017EA00E6FAADD0620093FAE8FAA9D0620093FA59
:1017FA00E9FAA5D00A01A651000AD8B457D7A651CA
:10180A00010AD8B457D7A651020AD8B457D7A65155
:10181A00030AD8B457D7A651040AD8B457D7A65141
:10182A00050AD8B457D7A651060AD8B457D7A6512D
:10183A00070AD8B457D7A651080AD8B457D7A65119
:10184A00090AD8B457D7A6510A0AD8B457D7A65105
:10185A000B0AD8B457D7A6510C0AD8B457D7A651F1
:10186A000D0AD8B457D7A6510E0AD8B457D7A651DD
:10187A000F0AD8B457D7A651100AD8B457D7A651C9
:10188A00110AD8B457D7A651120AD8B457D7A651B5
:10189A00130AD8B457D7A651140AD8B457D7A651A1
:1018AA00150AD8B457D7A651160AD8B457D7A6518D
:1018BA00170AD8B457D7A651180AD8B457D7A65179
:1018CA00190AD8B457D7A6511A0AD8B457D7A65165
:1018DA001B0AD8B457D7A6511C0AD8B457D7A65151
:1018EA001D0AD8B457D7A6511E0AD8B457D7A6513D
:1018FA001F0AD8B457D7A651200AD8B457D7A65129
:10190A00210AD8B457D7A651220AD8B457D7A65114
:10191A00230AD8B457D7A651240AD8B457D7A65100
:10192A00250AD8B457D7A651260AD8B457D7A651EC
:10193A00270AD8B457D7A651280AD8B457D70A01C4
:10194A00A75302E033EC06F0A8D00A01A5B102D0F1
:10195A00C29001D0C280F9D00A01A5B102D0C292C8
:10196A0001D0C282F2D00A01A5B102D0C29401D03C
:10197A00C284EBD00A01A5B102D0C29601D0C286B8
:10198A00E4D00A01A5B102D0C29801D0C288DDD044
:10199A000A01A5B102D0C29A01D0C28AD6D00A01E0
:1019AA00A5B102D0C29C01D0C28CCFD00A01A5B188
:1019BA0002D0C29E01D0C28EC8D00A01A5B102D0FF
:1019CA00C39001D0C380C1D00A01A5B102D0C3928D
:1019DA0001D0C382BAD00A01A5B102D0C39401D002
:1019EA00C384B3D00A01A5B102D0C39601D0C3867D
:1019FA00ACD00A01A5B102D0C39801D0C388A5D042
:101A0A000A01A5B102D0C39A01D0C38A9ED00A01A5
:101A1A00A5B102D0C39C01D0C38C97D00A01A5B14D
:101A2A0002D0C39E01D0C38E90D00A01A5B102D0C4
:101A3A00C49001D0C48089D00A01A5B102D0C49251
:101A4A0001D0C48282D00A01A5B102D0C49401D0C7
:101A5A00C4847BD00A01A5B102D0C49601D0C48641
:101A6A0074D00A01A5B102D0C49801D0C4886DD03F
:101A7A000A01A5B102D0C49A01D0C48A66D00A016B
:101A8A00A5B102D0C49C01D0C48C5FD00A01A5B113
:101A9A0002D0C49E01D0C48E58D00A01A451000AB3
:101AAA00D8B453D7A451010AD8B456D7A451020ABC
:101ABA00D8B459D7A451030AD8B45CD7A451040A9C
:101ACA00D8B45FD7A451050AD8B462D7A451060A7C
:101ADA00D8B465D7A451070AD8B468D7A451080A5C
:101AEA00D8B46BD7A451090AD8B46ED7A4510A0A3C
:101AFA00D8B471D7A4510B0AD8B474D7A4510C0A1C
:101B0A00D8B477D7A4510D0AD8B47AD7A4510E0AFB
:101B1A00D8B47DD7A4510F0A81E0A451100A85E0F8
:101B2A00A451110A89E0A451120A8DE0A451130AA2
:101B3A0091E0A451140A95E0A451150A99E0A45120
:101B4A00160A9DE0A451170AA1E0FF0E006E1200CA
:101B5A000901566B576B010E0001DD5D016E000E27
:101B6A00DE59026E02500901575D02E10150565DCD
:101B7A0018E2FC0E5625E16E090E5721E26E6F003F
:101B8A0087FFE1FF6F008BFFE2FFE66A010E562531
:101B9A00006E000E5721016E00C056F901C057F9B8
:101BAA00DAD7FC6B566B576B546B556B0A017C6B1F
:101BBA007D6B0801B66B3D01F289F96BFA6B09017D
:0C1BCA00526B536B236A390193871200A1
:101BD60062009BFAF6FF62009FFAF7FF6200A3FA23
:101BE600F8FF09006F00D4FF00F000521FE062000A
:101BF6009BFAF6FF62009FFAF7FF6200A3FAF8FF6E
:101C060009006F00D4FF00F0620093FAE1FF620062
:101C160097FAE2FF600003F0E6FF0A01A44BA52B4A
:101C2600010EA627000EA723A823D2D7620093FA97
:0C1C3600E1FF620097FAE2FFE66A12008C
:0E1C4200A4CABBFAA5CABCFA89EC07F01200CE
:101C5000000E0A01A51902E1000EA4193CE0620081
:101C600093FAE9FF620097FAEAFFEE5234E0A6CA5F
:101C7000BBFAA7CABCFA7EEC05F000C0BFFAA4CA42
:101C8000BBFAA5CABCFAA6CABDFAA7CABEFA13EC2B
:101C900004F0000E011802E1000E001805E1A4CACC
:101CA00000F0A5CA01F019D0010E0A01A425BB6FEE
:101CB000000EA521BC6F62009BFAE9FF62009FFA4B
:101CC000EAFF6F00B8FFBDFAFFEC06F000C0A4FA0F
:0C1CD00001C0A5FABDD7006A016A12002D
:101CDC00620093FAF6FF620097FAF7FF62009BFA34
:101CEC00F8FF09006F00D4FF00F0005216E062000C
:101CFC0093FAF6FF620097FAF7FF62009BFAF8FF7F
:101D0C0009006F00D4FFC1FA80EC00F0010E0A014B
:0C1D1C00A427000EA523A623DBD712008D
:101D28000A01A86B620093FAE9FF620097FAEAFFDA
:101D3800EE5219E0A6CABBFAA7CABCFA620093FA27
:101D4800E9FF620097FAEAFF6F00B8FFBDFAFFECFF
:101D580006F0000E011802E1000E001804E1A44B81
:0C1D6800A52BA82BDFD7A8CA00F01200A2
:101D7400220E0C6E086A096A0A6A0B6A0C06D8B449
:101D84001FD0D8900B320A320932083203320232A1
:101D940001320032D8A0F2D70C06D8B409D00450CE
:101DA40008260550092206500A2207500B22EAD7BA
:101DB400045008260550092206500A2207500B2217
:021DC40012000B
:101DC600A5CA00F00032009E0032009E0032009E3E
:101DD6000032009E130E0024F66EBD0EF76E000E46
:101DE600F722000EF86E000EF82209006F00D4FFED
:101DF60000F062009BFAE1FF62009FFAE2FF6000DA
:101E060003F0E6FF010E0A01A625E16E000EA721EA
:101E1600E26E0F0EA515006E130E0024F66EBD0EB3
:101E2600F76E000EF722000EF86E000EF82209007B
:101E36006F00D4FF00F0600003F0E6FF020EA62557
:101E4600E16E000EA721E26EA4CA00F00032009EE9
:101E56000032009E0032009E0032009E130E0024C7
:101E6600F66EBD0EF76E000EF722000EF86E000E2F
:101E7600F82209006F00D4FF00F0600003F0E6FFCF
:101E8600030EA625E16E000EA721E26E0F0EA41525
:101E9600006E130E0024F66EBD0EF76E000EF722CE
:101EA600000EF86E000EF82209006F00D4FF00F055
:101EB600600003F0E6FF040EA625E16E000EA721E2
:061EC600E26EE66A120064
:101ECC00086A080E0C6E003408360450085ED8B050
:0E1EDC0002D00826D89000360C2EF5D7120042
:101EEA000A01A86BA96B620093FAE9FF620097FAEC
:101EFA00EAFFEE521AE0A6CABBFAA7CABCFA620007
:101F0A0093FAE9FF620097FAEAFF6F00B8FFBDFA99
:101F1A00FFEC06F0000E011802E1000E001805E0C1
:101F2A00A44BA52BA84BA92BDED7A8CA00F0A9CA97
:041F3A0001F01200A0
:101F3E006E0094F7A8FA6F0048FFA7FA62009BFAAA
:101F4E00E3F93F0E3901E517E585000E0A01A415E8
:101F5E00036EA551030B046E04C000F0016A60000D
:101F6E0003F0E1F9FF0EA4153901E06F52EC05F014
:101F7E00E5A301D0FDD70A01A7BF02D0D29E01D0A2
:0A1F8E00D28E6200A3FAE5F91200FA
:101F98000B6A0A6A096A005004026F00D0FF09F050
:101FA8006F00CCFF08F0015005026F00D0FF0BF066
:101FB8006F00CCFF0AF000500502F3500926F450D8
:101FC8000A22E86A0B2201500402F3500926F45051
:101FD8000A22E86A0B2208C000F009C001F00AC012
:081FE80002F00BC003F012002F
:101FF0002F6A306A316A326A336A0801BB51000ABB
:06200000D8B4346A12009E
:10200600BB92BB94BB96BB980801BB51000AD8B4DF
:04201600BA9E12005C
:10201A000A019551390806E3300E955D03E3010E76
:08202A00006E01D0006A1200F3
:1020320095CA04F096CA05F00A0199519A112CE04A
:10204200010E995F000E9A5B04C002F005C003F016
:10205200044A052A97CA00F098CA01F0974B982BB8
:10206200600003F0E9FF600007F0EAFF60000BF098
:10207200E1FF60000FF0E2FF6F00BBFFE6FF6000D0
:102082000BF0E9FF60000FF0EAFF6F00B8FF00F00D
:10209200005201E101D0D0D799CA00F09ACA01F0EA
:1020A200010E995F000E9A5B005001100AE0600079
:1020B20013F0E1FF600017F0E2FFE66A044A052A26
:0C20C200EBD795CA00F096CA01F012009E
:1020CE0095CA04F096CA05F004C002F005C003F0EC
:1020DE00044A052A97CA00F098CA01F00A01974BE4
:1020EE00982B600003F0E9FF600007F0EAFF600044
:1020FE000BF0E1FF60000FF0E2FF6F00BBFFE6FFA9
:10210E0060000BF0E9FF60000FF0EAFFEE5201E015
:0C211E00DBD795CA00F096CA01F0120051
:10212A00000E0A01961902E1000E951904E165C92B
:10213A0095FA66C996FA9551961103E1006A016A01
:10214A005FD0620057FAE9FF62005BFAEAFF6F00AC
:10215A00B8FF00F0005203E1006A016A51D095CA43
:10216A00A4FA96CAA5FA97CAA6FA98CAA7FAB8DE2E
:10217A00955100269651012200C095FA01C096FA9F
:10218A00600003F0E9FF600007F0EAFF6F00B8FFA4
:10219A0000F0005208E10901656B666B000E006EE3
:1021AA00000E016E2DD095CAA4FA96CAA5FA97CA4E
:1021BA00A6FA98CAA7FAB3DD000E016E9551002659
:1021CA009651012200C065F901C066F9600003F06A
:1021DA00E9FF600007F0EAFFEE520BE0620097F5B4
:1021EA00E1FF62009BF5E2FFE66A0901654B662B97
:1021FA0003D00901656B666B95CA00F096CA01F0B7
:02220A001200C0
:10220C000A01956B966B976B986B3F013E9F820E04
:10221C000A01A46FB90EA56F000EA66F59DD0A0155
:10222C00956B966B800E9619006E800E005C02E129
:10223C000B0E955DD8B0ABD095CA00F096CA01F0E4
:10224C00003600900136003600900136590E0024FD
:10225C00E96E000E0120EA6E6F00A7FFE9FF6F0028
:10226C00ABFFEAFF6F00B8FF00F06F00B8FF01F0A2
:10227C00C3EC07F03F0E046E350E056E060E066EAF
:10228C00810E076E9DEC05F0B7EC04F000C0E4F194
:10229C0001C0E5F102C0E6F103C0E7F1E40E07016D
:1022AC00C36F010EC46F020EC325E96E000EC4216C
:1022BC00EA6E6F00A7FFE9FF6F00ABFFEAFF6F004C
:1022CC00BBFF3DFF010EC325E96E000EC421EA6E73
:1022DC006F00A7FFE9FF6F00ABFFEAFF6F00BBFFCA
:1022EC003CFF61000FFFE9FF610013FFEAFF6F0085
:1022FC00BBFF3BFF3F013E8F0A01976B986B95CA62
:10230C0000F096CA01F000360090013600360090BD
:10231C000136590E0026000E0122020E0024D96E41
:10232C00000E0120DA6E6F0067FFE9FF6F006BFF94
:10233C00EAFF6F00B8FF01F06F00B8FF02F0025027
:10234C00985D02E10150975D0FE2110E0B6E3C0E91
:10235C000C6ECB0E0D6E0D2EFED70C2EFCD70B2E4D
:10236C00FAD7974B982BCBD73F013E9F090E0B6E9C
:10237C001E0E0C6EE40E0D6E0D2EFED70C2EFCD721
:10238C000B2EFAD700000A01954B962B4BD7120057
:10239C000A01966B976B986B996B9A6B9B6BD29EA1
:1023AC007A0EA46FBC0EA56F000EA66F91DCED0E1D
:1023BC000A01A46FB60EA56F000EA66F89DC0A0188
:1023CC00A46BA56BB4C0A6FAB4DD030E0B6E080E9D
:1023DC000C6E770E0D6E0D2EFED70C2EFCD70B2E21
:1023EC00FAD70A0E046EB4C000F06ADD300E002479
:1023FC000A01C16F80EC00F00A0E046EB4C000F04C
:10240C005FDD08C000F0300E00240A01C16F80ECC3
:10241C0000F084EC08F0C60E0A01A46FB90EA56F8B
:10242C00000EA66F55DC100E0A019A6F000E9B6F02
:10243C0007011C51030802E2030E1C6F300E1C2511
:10244C00006E00C095FA00C0C1FA80EC00F084EC7C
:10245C0008F09ACAA4FA9BCAA5FA95CAA6FA69DD2D
:10246C00030E0B6E080E0C6E770E0D6E0D2EFED736
:10247C000C2EFCD70B2EFAD70A01966B976B800E9D
:10248C009719006E800E005C02E1060E965DD8B0C6
:10249C0090D0670EA46FC10EA56F000EA66F18DC4E
:1024AC00300E0A019625C16F80EC00F0510E0A0126
:1024BC00A46FC20EA56F000EA66F0ADC040E026E8E
:1024CC0096CA00F097CA01F0025005E00036009061
:1024DC000136FF0FFAD7200E0026000E012200C095
:1024EC009AFA01C09BFA00C0A4FA01C0A5FA670EC3
:1024FC000A01A66F090EA76F60DC670EA46F090EA8
:10250C00A56F21EC0EF0440EA46FC20EA56F000E49
:10251C00A66F6EEC0EF00A01986B996B800E9919F0
:10252C00006E800E005C02E1040E985D3CE2050E2C
:10253C00006E000E016E96CA04F097CA05F026DDF7
:10254C00960E0026000E012298510024E96E995136
:10255C000120EA6E6F00A7FFE9FF6F00ABFFEAFFF7
:10256C006F00B8FF00F000C095FA00C0C1FA80EC13
:10257C0000F00A0198519A25A46F99519B21A56FDF
:10258C0095CAA6FAD6DC030E0B6E080E0C6E770EEF
:10259C000D6E0D2EFED70C2EFCD70B2EFAD70A0182
:1025AC00984B992BBBD784EC08F00A01964B972BD0
:1025BC0066D7ED0EA46FAF0EA56F000EA66F6EEC76
:1025CC000EF00A01966B976B800E9719006E800EB9
:1025DC00005C02E1060E965D37E2290E9625E96E47
:1025EC00000E9721EA6E6F00A7FFE9FF6F00ABFFAB
:1025FC00EAFF300EEE24006E00C095FA00C0C1FA5E
:10260C0080EC00F0800E0A019625006E000E9721DA
:10261C00016E00C09AFA01C09BFA00C0A4FA01C076
:10262C00A5FA95CAA6FA85DC030E0B6E080E0C6E85
:10263C00770E0D6E0D2EFED70C2EFCD70B2EFAD767
:10264C000A01964B972BC0D70E0EA46FB00EA56F38
:10265C00000EA66F6EEC0EF00A01966B976B800E57
:10266C009719006E800E005C02E1060E965D32E258
:10267C00900E96259A6F000E97219B6F520E962501
:10268C00E96E000E9721EA6E6F00A7FFE9FF6F005D
:10269C00ABFFEAFF300EEE24006E00C095FA00C0CE
:1026AC00C1FA80EC00F09ACAA4FA9BCAA5FA95CAA2
:1026BC00A6FA3FDC030E0B6E080E0C6E770E0D6E39
:1026CC000D2EFED70C2EFCD70B2EFAD70A01964BEB
:1026DC00972BC5D79C0EA46FA90EA56F000EA66FE5
:1026EC006EEC0EF00A01966B976B800E9719006ECC
:1026FC00800E005C02E1060E965D33E2A00E96257C
:10270C009A6F000E97219B6F2F0E9625E96E000E87
:10271C009721EA6E6F00A7FFE9FF6F00ABFFEAFF9E
:10272C00300EEE24006E00C095FA00C0C1FA80ECA9
:10273C0000F09ACAA4FA9BCAA5FA95CAA6FA9FEC0D
:10274C000FF0030E0B6E080E0C6E770E0D6E0D2E29
:10275C00FED70C2EFCD70B2EFAD70A01964B972BD3
:10276C00C4D7270EA46FB30EA56F000EA66F6EEC28
:10277C000EF0286A0A01966B976B800E9719006E03
:10278C00800E005C02E1040E965D33E2B00E9625DD
:10279C009A6F000E97219B6F240E9625E96E000E02
:1027AC009721EA6E6F00A7FFE9FF6F00ABFFEAFF0E
:1027BC006F00B8FF00F000C095FA00C0C1FA80ECC1
:1027CC0000F09ACAA4FA9BCAA5FA95CAA6FA9FEC7D
:1027DC000FF0030E0B6E080E0C6E770E0D6E0D2E99
:1027EC00FED70C2EFCD70B2EFAD70A01964B972B43
:1027FC00C4D7060EA46FB20EA56F000EA66F6EECBA
:10280C000EF0300E2224006E00C095FA00C0C1FA02
:10281C0080EC00F0C00E0A01A46F000EA56F95CAE3
:10282C00A6FA9FEC0FF0030E0B6E080E0C6E770ED3
:10283C000D6E0D2EFED70C2EFCD70B2EFAD784EC7A
:06284C0008F0D28E12001C
:10285200B40E0A01956F000E966F670EA46F090EF3
:10286200A56FAD0EA66FBD0EA76F000EA86FEBECA5
:102872000DF095CAA4FA96CAA5FA6E0E0A01A66FC1
:10288200090EA76FD8EC07F02A0E0901736F300EFC
:1028920007011C250901776F670E0A01A46F090E53
:1028A200A56F21EC0EF0B30EA46FC10EA56F000E42
:1028B200A66F6EEC0EF00D0E3E01F16FF881000076
:1028C200F8A101D0FDD76F00C0FBE7F9000E0901A6
:1028D200E86FE7C901F0006A3E01EF510026000EE1
:1028E200012200C018F701C019F700C0A4FA01C004
:1028F200A5FA670E0A01A66F090EA76FD8EC07F0BA
:10290200570EA46FC20EA56F000EA66F6EEC0EF0EE
:10291200670E0A01A46F090EA56F21EC0EF0540E8A
:10292200A46FC20EA56F000EA66F6EEC0EF007012B
:1029320019511E5D02E118511D5D0AE22051195D17
:1029420002E11F51185D04E2010E0101EA6F02D09B
:102952000101EA6B070119510101E95D04E1070177
:1029620018510101E85D0EE2080184510701195D69
:1029720004E1080183510701185D04E2010E080118
:10298200826F02D00801826B070119510801815D33
:1029920004E1070118510801805D0DE27F51070132
:1029A200195D04E108017E510701185D04E2010E80
:1029B20008017D6F02D008017D6B0101EA51010A15
:1029C20009E1850E0A01A46FB80EA56F000EA66F6D
:1029D2006EEC0EF008018251010A09E16A0E0A0149
:1029E200A46FB40EA56F000EA66F6EEC0EF0080178
:1029F2007D51010A09E1AD0E0A01A46FB70EA56F60
:102A0200000EA66F6EEC0EF0080182510101EA255C
:102A1200006E016A000E012208017D510024026E3F
:102A2200000E0120036E000E031802E1000E0218D0
:102A320009E1400E0A01A46FBB0EA56F000EA66F3E
:102A42006EEC0EF084EC08F0ADEC0DF0520E0B6E55
:102A52002B0E0C6E000E0D6E0D2EFED70C2EFCD71B
:102A62000B2EFAD70000FC0E0A01A46F090EA56F07
:102A7200750EA66F080EA76F28EC0EF000C07CFA48
:102A820001C07DFA010E0A01955F000E965B000EF1
:102A9200011802E1000E001809E1000E006E9651C5
:102AA200005C02E19551000801E2D7D6ADEC0DF0D1
:062AB2000701C26B1200D7
:102AB80095CAA4FA96CAA5FA97CAA6FA010E0A01F7
:082AC800A76F95EC0AF0120063
:102AD0000B6A0A6A096A086A0E6A033408360450E7
:102AE000085E0550D8A0053C095E0650D8A0063CFB
:102AF0000A5E0750D8A0073C0B5EE86AD8A0010E1A
:102B00000E5E0336070E0C6E0334083609360A369D
:102B10000B360E36045003A012D0085E0550D8A024
:102B2000053C095E0650D8A0063C0A5E0750D8A0B6
:102B3000073C0B5EE86AD8A0010E0E5E11D0082695
:102B40000550D8B0053C09260650D8B0063C0A26E8
:102B50000750D8B0073C0B26E86AD8B0010E0E2605
:102B600003360C2ED1D70234083609360A360B3616
:102B70000E36045003A012D0085E0550D8A0053CC4
:102B8000095E0650D8A0063C0A5E0750D8A0073C54
:102B90000B5EE86AD8A0010E0E5E11D00826055023
:102BA000D8B0053C09260650D8B0063C0A26075086
:102BB000D8B0073C0B26E86AD8B0010E0E260236C4
:102BC000070E0C6E0234083609360A360B360E36FE
:102BD000045002A012D0085E0550D8A0053C095E42
:102BE0000650D8A0063C0A5E0750D8A0073C0B5EF2
:102BF000E86AD8A0010E0E5E11D008260550D8B0A4
:102C0000053C09260650D8B0063C0A260750D8B025
:102C1000073C0B26E86AD8B0010E0E2602360C2EB1
:102C2000D1D70134083609360A360B360E36045031
:102C300002A012D0085E0550D8A0053C095E0650DF
:102C4000D8A0063C0A5E0750D8A0073C0B5EE86A95
:102C5000D8A0010E0E5E11D008260550D8B0053C54
:102C600009260650D8B0063C0A260750D8B0073CC3
:102C70000B26E86AD8B0010E0E260136070E0C6E40
:102C80000134083609360A360B360E36045001A0D8
:102C900012D0085E0550D8A0053C095E0650D8A0A9
:102CA000063C0A5E0750D8A0073C0B5EE86AD8A035
:102CB000010E0E5E11D008260550D8B0053C09263D
:102CC0000650D8B0063C0A260750D8B0073C0B2661
:102CD000E86AD8B0010E0E2601360C2ED1D700348A
:102CE000083609360A360B360E36045001A012D0CB
:102CF000085E0550D8A0053C095E0650D8A0063CE9
:102D00000A5E0750D8A0073C0B5EE86AD8A0010E07
:102D10000E5E11D008260550D8B0053C0926065095
:102D2000D8B0063C0A260750D8B0073C0B26E86A04
:102D3000D8B0010E0E260036070E0C6E0034083691
:102D400009360A360B360E36045000A012D0085E43
:102D50000550D8A0053C095E0650D8A0063C0A5E86
:102D60000750D8A0073C0B5EE86AD8A0010E0E5EA3
:102D700011D008260550D8B0053C09260650D8B019
:102D8000063C0A260750D8B0073C0B26E86AD8B0A4
:102D9000010E0E2600360C2ED1D700B00ED00450F6
:102DA00008260550D8B0053C09260650D8B0063C88
:0C2DB0000A260750D8B0073C0B26120082
:0C2DBC006F00A0F701F001C000F0120051
:102DC8006E0094F705F03F0E3901E517000E0A0171
:102DD8009515036E9651030B046E04C000F0016A4A
:102DE800600003F0E1F9FF0E95153901E06FE58108
:0E2DF800600017F0E5F96E008CF700F0120095
:102E06000A01976B986B956B966B800E9619006E00
:102E1600800E005C02E1030E955DD8B0B7D00801C4
:102E2600BB51000A03E17F0EC21602D0FF0EC26E2E
:102E360031D0BA88C298150E0C6EC60E0D6E0D2EC8
:102E4600FED70C2EFCD7000039D0BA8AC29A150ECE
:102E56000C6EC60E0D6E0D2EFED70C2EFCD7000086
:102E66002DD0BA8CC29C150E0C6EC60E0D6E0D2E94
:102E7600FED70C2EFCD7000021D00801BA98BA9ACA
:102E8600BA9CBB51000A03E17F0EC21602D0FF0EA8
:102E9600C26E14D0000E0A01961902E1000E9519B1
:102EA600C8E0000E961902E1010E9519CEE0000E5B
:102EB600961902E1020E9519D4E0DFD70901FBAF9E
:102EC6005ED02A0E0C6E8D0E0D6E0D2EFED70C2EBC
:102ED600FCD7000000000F0ECA14006E00C097FA5F
:102EE60000C098FA020E0B6E380E0C6EAD0E0D6E0B
:102EF6000D2EFED70C2EFCD70B2EFAD70F0ECA14AA
:102F0600016E01C097FA0150000839E20A01975193
:102F1600981935E1BC88090E006E000E016E026E2E
:102F2600036E95CA04F096CA05F0000E96BFFF0E12
:102F3600066E076EBAEC0EF0950E0026B30E012251
:102F4600000E022297510024F66E000E0120F76E45
:102F5600000E0220F86E6F00DBFFF6FF6F00DFFF4A
:102F6600F7FF6F00E3FFF8FF09006F00D4FFBFF81B
:102F76000F0ECA14016E0150000801E2F9D70A01CA
:0E2F8600BA98BA9ABA9C954B962B3FD7120078
:102F94000A01A06BA16BA26BA36B95CA00F0000E93
:102FA400016E003600900136A20E0024E96E010E77
:102FB4000120EA6E6F00A7FFE9FF6F00ABFFEAFF95
:102FC4006F00B8FF62F96F00B8FF63F93F013E9FDD
:102FD400040E3F6F0A019651000813E2F00EA46F2D
:102FE400BE0EA56F000EA66F6EEC0EF0300E0A0139
:102FF4009525C16F80EC00F0200E0A01C16F80ECB2
:1030040000F00A01976B986B975109016225E96EEC
:103014000A01985109016321EA6E6F00A7FFE9FFD5
:103024006F00ABFFEAFF6F00B8FF01F001C09FFA29
:103034000150FF0A01E111D00A019651000804E28F
:103044009FCAC1FA80EC00F00A01974B982B000E3E
:10305400985D02E1400E975DD7E30A01965100089E
:1030640017E2200EC16F80EC00F097CAA4FA98CA48
:10307400A5FA670E0A01A66F090EA76FD8EC07F030
:10308400670EA46F090EA56F21EC0EF084EC08F016
:103094000A01A06BA16BA26BA36B5A0E7C6F090E85
:1030A4007D6F974B982B9D6B9E6B9651010814E294
:1030B4009DCAA4FA9ECAA5FA670EA66F090EA76F49
:1030C400D8EC07F0670EA46F090EA56F21EC0EF083
:1030D4002D0EC16F80EC00F00A01975109016225A1
:1030E400E96E0A01985109016321EA6E6F00A7FF96
:1030F400E9FF6F00ABFFEAFF6F00B8FF01F001C00A
:103104009FFA0150FF0A01E116D162007FFA3DFFE8
:103114009FCAA2FA0A01975109016225006E0A01A9
:10312400985109016321016E010E0024E96E000E1D
:103134000120EA6E6F00A7FFE9FF6F00ABFFEAFF13
:103144006F00B8FF01F001C09FFA0150FF0A01E1CE
:10315400F2D062007FFA3CFF9FCAA1FA0A0197519C
:1031640009016225006E0A01985109016321016E6B
:10317400020E0024E96E000E0120EA6E6F00A7FF24
:10318400E9FF6F00ABFFEAFF6F00B8FF01F001C079
:103194009FFA0150FF0A01E1CED062007FFA3BFFA3
:1031A4009FCAA0FA0A019651010832E2A0CA00F0AF
:1031B400A1CA01F0A2CA02F0A3CA03F08FEC08F07E
:1031C400F80E046EE70E056E7D0E066E780E076E21
:1031D4009DEC05F000C0A4FA01C0A5FA02C0A6FA4D
:1031E40003C0A7FA670EA86F090EA96F010EAA6F94
:1031F400A2EC08F0670EA46F090EA56F21EC0EF087
:103204006A0EA46FBE0EA56F000EA66F6EEC0EF0D4
:103214000A01975109016225006E0A0198510901BA
:103224006321016E030E0024E96E000E0120EA6E94
:103234006F00A7FFE9FF6F00ABFFEAFF6F00B8FF65
:1032440001F001C09FFA0150FF0A01E174D09FCA46
:103254009BFA000E0A019C6F9BCA9CFA9B6B9751C8
:1032640009016225006E0A01985109016321016E6A
:10327400040E0024E96E000E0120EA6E6F00A7FF21
:10328400E9FF6F00ABFFEAFF6F00B8FF01F001C078
:103294009FFA0150FF0A01E14ED00A019F519B257C
:1032A400016E000E9C21026E01C09BFA02C09CFAC2
:1032B4000250070802E10150D00804E2D00E9B6FCF
:1032C400070E9C6F9651010812E29BCAA4FA9CCA8D
:1032D400A5FA670EA66F090EA76FD8EC07F0670E64
:1032E400A46F090EA56F21EC0EF084EC08F03F01E9
:1032F4003E8F0A01996B9A6B9C519A5D02E19B5136
:10330400995D0CE2150E0C6EC60E0D6E0D2EFED7D9
:103314000C2EFCD70000994B9A2BEED73F013E9F11
:10332400050E0A019727000E98239D4B9E2B9F5153
:10333400FF0AD8A4BAD63F013E9F030E3F6F0A018D
:10334400965101081BE2430EA46FBD0EA56F000E3B
:10335400A66F6EEC0EF097CAA4FA98CAA5FA670E87
:103364000A01A66F090EA76FD8EC07F0670EA46FC9
:10337400090EA56F21EC0EF084EC08F0090E0B6E1B
:103384001E0E0C6EE40E0D6E0D2EFED70C2EFCD709
:083394000B2EFAD70000120015
:10339C000901FB9395CAB9F896CABAF8CF0EB16E6B
:0E33AC002C0EB06E3901A4919481B2801200F3
:1033BA000A019B6B9C6B030E07011B6F1A6B030EB2
:1033CA003F013F6F95CA04F096CA05F097CA06F006
:1033DA0098CA07F0000E006E000E016E700E026EA3
:1033EA00830E036E22EC07F0010ED8B0000E006EB9
:1033FA00005228E095CAA4FA96CAA5FA97CAA6FA6C
:10340A0098CAA7FA24EC08F03F013E8F0A019B6B89
:10341A009C6B800E9C19006E800E9A19005C02E16A
:10342A0099519B5D0CE2150E0C6EC60E0D6E0D2E9B
:10343A00FED70C2EFCD700009B4B9C2BEAD73F01F2
:10344A003E9F19D00A019B6B9C6B800E9C19006EE3
:10345A00800E9A19005C02E199519B5D0CE2150EEF
:10346A000C6EC60E0D6E0D2EFED70C2EFCD700006C
:08347A009B4B9C2BEAD71200CA
:1034820008017C6B040E7A6F7B6B4C0E0A01A46FF1
:10349200000EA56FF90EA66FC10EA76F000EA86FE2
:1034A200EBEC0DF04C6ABC9ABC98600E0A01A46F5A
:1034B200B20EA56F000EA66F6EEC0EF000018A4BE5
:1034C2008B2B670E0A01A46F090EA56F530EA66F10
:1034D200BD0EA76F000EA86FEBEC0DF08AC0A4FA28
:1034E2008BC0A5FA6E0E0A01A66F090EA76FD8EC63
:1034F20007F02A0E0901736F670E0A01A46F090E05
:10350200A56F21EC0EF084EC08F03901A1919181B4
:1035120008017B6BBF6B0901FB9F1E0E0A01956FB1
:10352200000E966F3ADF6EDC00018951040A02E157
:10353200B00E8819D8B4BC888951040802E18851B8
:10354200B5080DE2FB0E0A01A46FBE0EA56F000EB8
:10355200A66F6EEC0EF0BC980001886B896B0901B6
:10356200FBBF03D0FBB301D0DED7FBA334D00801ED
:103572007C51000830E20901FB93010E08017B6FC8
:10358200430E0A01A46FB30EA56F000EA66F6EEC78
:103592000EF04C0E0A01A46F000EA56FE50EA66F89
:1035A200C10EA76F000EA86FEBEC0DF04C6A08017C
:1035B2007C6BBC8ABC98000E0A01956F000E966F58
:1035C200160E976F880E986FF40E996F010E9A6F10
:1035D200F3DEBC9AD0D00901FBAFCDD008017B51FC
:1035E200000AD8A4C8D000018551010A09E14F0E92
:1035F2000A01A46FC00EA56F000EA66F6EEC0EF04E
:10360200BC9ABC88BC96000E0A01956F000E966F9C
:10361200160E976F890E986FF40E996F010E9A6FBE
:10362200CBDE030E08017C5D3FE25150000A11E13E
:10363200BC86BC9ABC9800018551010A09E19F0E23
:103642000A01A46FC10EA56F000EA66F6EEC0EF0FC
:1036520010D0BC8ABC98BC9600018551010A09E1D0
:10366200EA0E0A01A46FBF0EA56F000EA66F6EECE4
:103672000EF0290E0B6E960E0C6E7F0E0D6E0D2E39
:10368200FED70C2EFCD70B2EFAD700018551010A6A
:1036920009E17C0E0A01A46FC10EA56F000EA66F90
:1036A2006EEC0EF0BC9ABC980801BF51230A2BE1C4
:1036B2000B0E0A01A46FAD0EA56F000EA66F6EEC85
:1036C2000EF008017C6B4C0E0A01A46F000EA56F70
:1036D200EA0EA66FC10EA76F000EA86FEBEC0DF0FD
:1036E2004C6ABC98BC8A000E0A01956F000E966F58
:1036F200160E976F880E986FE80E996F030E9A6FE9
:103702005BDEBC9A38D008017C51030802E2030E4A
:103712007C6F4C0EE16E000EE26E7C51E126D8B059
:10372200E22A6F0087FFE1FF6F008BFFE2FF62007A
:10373200FFF2E6FF7C2B840E0A01A46FBE0EA56F7A
:10374200000EA66F6EEC0EF0300E08017C250A0109
:10375200C16F80EC00F0270E0A01A46FBF0EA56FA7
:10376200000EA66F6EEC0EF04C0E0A01A46F000E56
:10377200A56F21EC0EF00901FB9F08017A517C5DD7
:06378200D8A09CD6120045
:10378800160E0A01956F966B130E976F5CEC15F089
:10379800170E0A01956F010E966F250E976F5CEC58
:0437A80015F0120006
:1037AC000A018B6B8C6B000E8C5D02E10A0E8B5D3B
:1037BC000BE28B518925E16E8C518A21E26E200E31
:1037CC00E66E8B4B8C2BEFD78B518925E16E8C5190
:1037DC008A21E26EE66A010E8B5F000E8C5B8B51C8
:1037EC0089258D6F8C518A218E6F0A0E046E000E06
:1037FC00056E066E076E85CA00F086CA01F087CA90
:10380C0002F088CA03F068EC15F008C000F009C09B
:10381C0001F00AC002F00BC003F0300E002662006B
:10382C0037FAE1FF62003BFAE2FF600003F0E6FFCB
:10383C000A0E046E000E056E066E076E85CA00F049
:10384C0086CA01F087CA02F088CA03F068EC15F04A
:10385C0000C085FA01C086FA02C087FA03C088FA54
:10386C00000E046E031808E10450021805E1045020
:10387C00011802E10050000A01E105D0010E8B5F36
:08388C00000E8C5BACD71200AA
:0E389400526A536A546A556A566A576A12009D
:1038A2000A01876B886B896B8A6B8B6B8C6B956B50
:1038B200966BE4EC16F000C086FA030E0B6E080E4F
:1038C2000C6E770E0D6E0D2EFED70C2EFCD70B2E26
:1038D200FAD70A018551010A36E17D0EA46FB20EB4
:1038E200A56F000EA66F6EEC0EF0BE0E0A01A46F5D
:1038F200BC0EA56F000EA66F6EEC0EF00A0E046EE3
:1039020086CA00F066EC0FF0300E00240A01C16F87
:1039120080EC00F00A0E046E86CA00F066EC0FF02E
:1039220008C000F0300E00240A01C16F80EC00F0E4
:1039320084EC08F0F20E0A01A46FB90EA56F000E16
:10394200A66F6EEC0EF0100E0A01956F000E966FC8
:10395200E4EC16F000C086FA030E0B6E080E0C6E35
:10396200770E0D6E0D2EFED70C2EFCD70B2EFAD72E
:103972000A018551010A0FE186CAC1FA80EC00F002
:1039820084EC08F0920E0A01A46FB00EA56F000E2F
:10399200A66F6EEC0EF00A01876B886B800E881999
:1039A200006E800E005C02E1060E875DD8B0CAD0C0
:1039B2008551010A17E13A0EA46FC00EA56F000EE1
:1039C200A66F6EEC0EF0300E0A018725C16F80ECF7
:1039D20000F05A0E0A01A46FC20EA56F000EA66F68
:1039E2006EEC0EF0040E006E87CA8BFA88CA8CFA4F
:1039F200005006E00A018B378B918C37FF0FF9D705
:103A02000A01200E8B27000E8C238551010A18E132
:103A12008BCAA4FA8CCAA5FA670EA66F090EA76F05
:103A2200E3EC0EF0670EA46F090EA56F21EC0EF009
:103A3200440EA46FC20EA56F000EA66F6EEC0EF0C0
:103A42000A01896B8A6B800E8A19006E800E005CF7
:103A520002E1040E895D37E289518B25956F8A5107
:103A62008C21966FE4EC16F000C086FA030E0B6E02
:103A7200080E0C6E770E0D6E0D2EFED70C2EFCD797
:103A82000B2EFAD7110E006E000E016E87CA04F0DB
:103A920088CA05F0CCEC0FF0EE0E0026000E0122D3
:103AA2000A0189510024E16E8A510120E26E6F0001
:103AB20087FFE1FF6F008BFFE2FF62001BFAE6FF68
:103AC200894B8A2BC0D7110E006E000E016E87CA79
:103AD20004F088CA05F0CCEC0FF0EE0E0026000EC2
:103AE200012289510024E16E8A510120E26E6F00A9
:103AF20087FFE1FF6F008BFFE2FFE66A8551010A53
:103B02001DE1440EA46FC20EA56F000EA66F6EECEF
:103B12000EF0110E006E000E016E87CA04F088CA04
:103B220005F0CCEC0FF0EE0E00240A01A46F000E9B
:103B32000120A56F21EC0EF084EC08F00A01874BFE
:103B4200882B2CD78551010A08E1AE0EA46FAE0E68
:103B5200A56F000EA66F6EEC0EF00A01876B886BE4
:103B6200800E8819006E800E005C02E1060E875DF1
:103B72002AE2800E8725006E000E8821016E00C0A9
:103B82008BFA01C08CFA00C095FA01C096FAE4ECF7
:103B920016F000C086FA030E0B6E080E0C6E770E3E
:103BA2000D6E0D2EFED70C2EFCD70B2EFAD70A0166
:103BB2008551010A04E186CAC1FA80EC00F00A01CB
:103BC200874B882BCDD78551010A08E1F50EA46FEA
:103BD200AD0EA56F000EA66F6EEC0EF00A01876B9C
:103BE200886B800E8819006E800E005C02E1060E62
:103BF200875D2AE2900E8725006E000E8821016EF5
:103C020000C08BFA01C08CFA00C095FA01C096FA86
:103C1200E4EC16F000C086FA030E0B6E080E0C6E72
:103C2200770E0D6E0D2EFED70C2EFCD70B2EFAD76B
:103C32000A018551010A04E186CAC1FA80EC00F04A
:103C42000A01874B882BCDD78551010A08E1E50E81
:103C5200A46FAA0EA56F000EA66F6EEC0EF00A01FD
:103C6200876B886B800E8819006E800E005C02E103
:103C7200060E875D2AE2A00E8725006E000E8821BF
:103C8200016E00C08BFA01C08CFA00C095FA01C027
:103C920096FAE4EC16F000C086FA030E0B6E080EDC
:103CA2000C6E770E0D6E0D2EFED70C2EFCD70B2E42
:103CB200FAD70A018551010A04E186CAC1FA80ECE9
:103CC20000F00A01874B882BCDD78551010A08E104
:103CD200E60EA46FB30EA56F000EA66F6EEC0EF08B
:103CE2000A01876B886B800E8819006E800E005C5B
:103CF20002E1040E875D2AE2B00E8725006E000EF7
:103D02008821016E00C08BFA01C08CFA00C095FABE
:103D120001C096FAE4EC16F000C086FA030E0B6EB0
:103D2200080E0C6E770E0D6E0D2EFED70C2EFCD7E4
:103D32000B2EFAD70A018551010A04E186CAC1FA9B
:103D420080EC00F00A01874B882BCDD78551010A00
:103D520008E1710EA46FB00EA56F000EA66F6EEC97
:103D62000EF0C00E0A01956F000E966FE4EC16F08D
:103D720000C086FA030E0B6E080E0C6E770E0D6EE7
:103D82000D2EFED70C2EFCD70B2EFAD70A01855129
:103D9200010A04E186CAC1FA80EC00F00A018551E9
:0A3DA200010A02E184EC08F01200AF
:103DAC0008017C6B010E7A6F84EC08F0420E0A015C
:103DBC00A46FB20EA56F000EA66F6EEC0EF06B0E1C
:103DCC000A01A46FB90EA56F000EA66F6EEC0EF073
:103DDC000901FB9F08017B6B1E0E0A01956F000EFB
:103DEC00966FCEEC19F0A191918103EC17F00901BB
:103DFC00FBBF03D0FBB301D0F8D7FBA328D0FB93B8
:103E0C00010E08017B6FBC8ABC98800E0A01A46F5E
:103E1C00BD0EA56F000EA66F6EEC0EF00801BF6B09
:103E2C007C51585C02E37C51585E7C6B000E0A019D
:103E3C00956F000E966F160E976F880E986FE80EA2
:103E4C00996F030E9A6FDDEC19F0BC9A67D00901DB
:103E5C00FBAF64D0BC9ABC88BC9600018551010AAA
:103E6C0009E15D0E0A01A46FC00EA56F000EA66FCE
:103E7C006EEC0EF0000E0A01956F000E966F160E8A
:103E8C00976F890E986FE80E996F030E9A6FDDECA1
:103E9C0019F0BC9ABC9800018551010A09E1410E48
:103EAC000A01A46FC00EA56F000EA66F6EEC0EF08B
:103EBC00010E08017C6F582AE50E0A01A46FBE0E94
:103ECC00A56F000EA66F6EEC0EF00A0E046E58C0B5
:103EDC0000F066EC0FF0300E00240A01C16F80EC8C
:103EEC0000F00A0E046E58C000F066EC0FF008C02B
:103EFC0000F0300E00240A01C16F80EC00F0670E58
:103F0C000A01A46FBF0EA56F000EA66F6EEC0EF02B
:103F1C00BFC8C1FA80EC00F084EC08F008017C51B9
:0C3F2C00000AD8B44CD7BFC800F0120047
:103F3800670E0A01A46F090EA56F530EA66FBF0E78
:103F4800A76F000EA86FEBEC0DF018C7A4FA19C7FD
:103F5800A5FA690E0A01A66F090EA76FD8EC07F03B
:103F68002A0E09016E6F670E0A01A46F090EA56F6C
:103F780021EC0EF00801BB51010A15E1CAAE0AD0C6
:103F8800CA0E0A01A46FB50EA56F000EA66F6EECDF
:103F98000EF009D0B10E0A01A46FB50EA56F000E80
:103FA800A66F6EEC0EF0070119511E5D02E1185163
:103FB8001D5D0AE22051195D02E11F51185D04E2FE
:103FC800010E0101EA6F02D00101EA6B07011951E4
:103FD8000101E95D04E1070118510101E85D0EE204
:103FE800080184510701195D04E1080183510701A3
:103FF800185D04E2010E0801826F02D00801826B8D
:10400800070119510801815D04E1070118510801F0
:10401800805D0DE27F510701195D04E108017E51C1
:104028000701185D04E2010E08017D6F02D0080146
:104038007D6B0101EA51010A09E1260E0A01A46F0C
:10404800B90EA56F000EA66F6EEC0EF00801825136
:10405800010A09E1840E0A01A46FB40EA56F000ECF
:10406800A66F6EEC0EF008017D51010A09E15D0EA4
:104078000A01A46FB60EA56F000EA66F6EEC0EF0C7
:10408800080182510101EA25006E016A000E012231
:1040980008017D510024026E000E0120036E02C04B
:1040A800E7F903C0E8F9000E031802E1000E021850
:1040B80009E12C0E0A01A46FBB0EA56F000EA66FB6
:1040C8006EEC0EF05350010A23E1BBA20AD0050E94
:1040D8000A01A46FB70EA56F000EA66F6EEC0EF066
:1040E80016D02A50090A0AE10F0E0A01A46FB90E68
:1040F800A56F000EA66F6EEC0EF009D06D0E0A01CA
:10410800A46FB80EA56F000EA66F6EEC0EF009D066
:10411800360E0A01A46FBC0EA56F000EA66F6EECDA
:104128000EF05450010A23E1BBA40AD04D0E0A0137
:10413800A46FB70EA56F000EA66F6EEC0EF016D02A
:104148002B50090A0AE1540E0A01A46FB90EA56F93
:10415800000EA66F6EEC0EF009D0350E0A01A46FA2
:10416800B70EA56F000EA66F6EEC0EF009D0E00E2C
:104178000A01A46FBC0EA56F000EA66F6EEC0EF0C0
:104188005550010A23E1BBA60AD07D0E0A01A46F8F
:10419800B70EA56F000EA66F6EEC0EF016D02C5061
:1041A800090A0AE13D0E0A01A46FB90EA56F000EB7
:1041B800A66F6EEC0EF009D0950E0A01A46FB70E2B
:1041C800A56F000EA66F6EEC0EF009D0AD0E0A01B9
:1041D800A46FBC0EA56F000EA66F6EEC0EF05650C5
:1041E800010A23E1BBA80AD0650E0A01A46FB70E25
:1041F800A56F000EA66F6EEC0EF016D02D50090AB2
:104208000AE1F80E0A01A46FB80EA56F000EA66F9A
:104218006EEC0EF009D01D0E0A01A46FB70EA56F43
:10422800000EA66F6EEC0EF009D09C0E0A01A46F6A
:10423800BC0EA56F000EA66F6EEC0EF00801BB5108
:10424800000A26E15750010A23E1BAAE0AD0B30E9C
:104258000A01A46FB80EA56F000EA66F6EEC0EF0E3
:1042680016D02E50090A0AE19C0E0A01A46FB80E56
:10427800A56F000EA66F6EEC0EF009D0C50E0A01F0
:10428800A46FB70EA56F000EA66F6EEC0EF009D0E6
:10429800CF0E0A01A46FBC0EA56F000EA66F6EECC0
:1042A8000EF04E0E0A01A46FC20EA56F000EA66F87
:0642B8006EEC0EF0120096
:1042BE000A01886B030E885D0AE288518625E16E3D
:1042CE00000E8721E26E200EE66E882BF3D7885102
:1042DE008625E16E000E8721E26EE66A8807885118
:1042EE008625896F000E87218A6F0A0E046E85CA95
:1042FE0000F066EC0FF008C000F0300E00266200F1
:10430E0027FAE1FF62002BFAE2FF600003F0E6FFFE
:10431E000A0E046E85CA00F066EC0FF000C085FA36
:0E432E000050000A01E102D08807D9D7120022
:06433C00DEEC16F0120099
:1043420085CAE9F986CAEAF987CAEBF988CAECF99B
:1043520089CAEFF98ACAF0F98BCAF1F98CCAF2F963
:104362008DCAF3F98ECAF4F98FCAF5F990CAF6F933
:1043720091CAF7F992CAF8F993CAF9F994CAFAF903
:02438200120027
:104384000A0185510308D8A0856B86510308D8A07B
:10439400866BF00E3D01F2170A0185513D01F213BF
:1043A400300EF21386CA00F00036009000360090FA
:1043B40000360090003600900050F413F38F120082
:1043C4000A018C6B8D6B010E0001856F0A01856BF0
:1043D400866B39019397D29EFC0E0A01A46F090ED5
:1043E400A56F21EC0EF084EC08F00A018C6B00013F
:1043F400856BFC0E0A01A46F090EA56F350EA66F1E
:10440400000EA76F28EC0EF000C07CFA01C07DFA04
:10441400000E026E0150025C02E100500008D8B0A8
:10442400E9D30A018C2BFC0EBB6F090EBC6F7EEC2A
:1044340005F000C089FA01C08AFA00018551010A19
:104444001CE1A30E0A01A46FC00EA56F000EA66F97
:104454006EEC0EF089CAA4FA8ACAA5FA670E0A019C
:10446400A66F090EA76FD8EC07F0670EA46F090EAC
:10447400A56F21EC0EF084EC08F0000E0A018A19F5
:1044840002E14D0E8919D8B48C2BFC0EA46F090ED1
:10449400A56F400EA66F000EA76F28EC0EF000C0AB
:1044A4007CFA01C07DFA000E026E0150025C02E14A
:1044B4000050000802E20A018C2B0A01FC0EA46FD2
:1044C400090EA56F390EA66F000EA76F28EC0EF02B
:1044D40000C07CFA01C07DFA000E026E0150025C3D
:1044E40002E10050000802E20A018C2B0A01FC0ED2
:1044F400A46F090EA56F990EA66F010EA76F28EC85
:104504000EF000C07CFA01C07DFA000E026E01506C
:10451400025C02E10050000802E20A018C2B0A014D
:10452400B10EA46FC00EA56F000EA66F6EEC0EF058
:10453400300E0A018C25C16F80EC00F084EC08F089
:104544000A012851300A04E129513B0AD8B48C2BC2
:104554008C51060AD8A44CD37CCA95FA7DCA96FA23
:10456400970E976F010E986F95EC10F000C07CFACF
:1045740001C07DFA670E0A01956F090E966F00C09F
:1045840097FA01C098FA67EC10F08C6B000E7D1955
:1045940002E1000E7C19D8B4E0D2956B966BA00EA4
:1045A400976F010E986F95EC10F000C07CFA01C073
:1045B4007DFA670E0A01956F090E966F00C097FA8F
:1045C40001C098FA67EC10F02FD2876B886B090151
:1045D400586B596B000E595D02E1040E585D19E2E7
:1045E400670E5825E96E090E5921EA6E6F00A7FF80
:1045F400E9FF6F00ABFFEAFF6F00B8FF95FA0DEC1F
:1046040010F0005202E0874B882B0901584B592BBC
:10461400E1D7000E0A01881902E1040E871960E14E
:10462400050E006E000E016E85CA04F086CA05F000
:10463400CCEC0FF0960E0024956F000E0120966FBF
:10464400670E976F090E986F040E996F000E9A6F9C
:1046540019EC10F0520E8525E16E000E8621E26EF3
:104664006F0087FFE1FF6F008BFFE2FF010EE66E34
:10467400040E8C2700018551010A31E1C60E0A019E
:10468400A46FC00EA56F000EA66F6EEC0EF00A0E9E
:10469400046E8CCA00F066EC0FF0300E00240A01A0
:1046A400C16F80EC00F00A0E046E8CCA00F066EC58
:1046B4000FF008C000F0300E00240A01C16F80EC36
:1046C40000F0090E0A01C16F80EC00F0670E0A01C8
:1046D400A46F090EA56F21EC0EF084EC08F00AD04B
:1046E400630E0701C26F0E0E0A01856F000E866FFE
:1046F4007C6B7D6B2DD200018551010A31E1FE0EE8
:104704000A01A46FC00EA56F000EA66F6EEC0EF02A
:104714000A0E046E8CCA00F066EC0FF0300E002412
:104724000A01C16F80EC00F00A0E046E8CCA00F01E
:1047340066EC0FF008C000F0300E00240A01C16FCF
:1047440080EC00F0090E0A01C16F80EC00F0670EE6
:104754000A01A46F090EA56F21EC0EF084EC08F099
:10476400F7D167C98BFA00018551010A2EE13D0E8C
:104774000A01A46FC10EA56F000EA66F6EEC0EF0B9
:104784000A0E046E8CCA00F066EC0FF0300E0024A2
:104794000A01C16F80EC00F00A0E046E8CCA00F0AE
:1047A40066EC0FF008C000F0300E00240A01C16F5F
:1047B40080EC00F0090E0A01C16F80EC00F08BCA96
:1047C400C1FA80EC00F084EC08F00A018B51300A45
:1047D40007E08B51310A04E08B51390A01E019D00A
:1047E400070E855D006E000E8659016E290E0024A9
:1047F400E16E000E0120E26E300E8B5D006E6F00E4
:1048040087FFE1FF6F008BFFE2FF600003F0E6FF2C
:104814000BD00E0E856F000E866F7C6B7D6B630E66
:104824000701C26F0A018C6B93D100018551010A03
:1048340031E14B0E0A01A46FC10EA56F000EA66FE5
:104844006EEC0EF00A0E046E8CCA00F066EC0FF0EB
:10485400300E00240A01C16F80EC00F00A0E046ED1
:104864008CCA00F066EC0FF008C000F0300E002493
:104874000A01C16F80EC00F0090E0A01C16F80ECDF
:1048840000F0670E0A01A46F090EA56F21EC0EF06B
:1048940084EC08F05DD167C98BFA00018551010AE7
:1048A4002EE1590E0A01A46FC10EA56F000EA66F6A
:1048B4006EEC0EF00A0E046E8CCA00F066EC0FF07B
:1048C400300E00240A01C16F80EC00F00A0E046E61
:1048D4008CCA00F066EC0FF008C000F0300E002423
:1048E4000A01C16F80EC00F0090E0A01C16F80EC6F
:1048F40000F08BCAC1FA80EC00F084EC08F00A01E5
:104904008B51300A04E08B51310A01E039D0000E9A
:10491400861902E1130E851919E10801BB51000A39
:1049240015E00E0E0A01855D006E000E8659016EBB
:10493400520E0024E16E000E0120E26E6F0087FF2C
:10494400E1FF6F008BFFE2FFE66A19D00A010E0E49
:10495400855D006E000E8659016E520E0024E16ED4
:10496400000E0120E26E300E8B5D006E6F0087FF3B
:10497400E1FF6F008BFFE2FF600003F0E6FF09D068
:10498400150E856F000E866F7C6B7D6B630E0701C1
:10499400C26FDED084EC08F000018551010A31E1D8
:1049A400520E0A01A46FC10EA56F000EA66F6EEC25
:1049B4000EF00A0E046E8CCA00F066EC0FF0300E96
:1049C40000240A01C16F80EC00F00A0E046E8CCA48
:1049D40000F066EC0FF008C000F0300E00240A016D
:1049E400C16F80EC00F0090E0A01C16F80EC00F089
:1049F400670E0A01A46F090EA56F21EC0EF084EC7A
:104A040008F00A017C6B7D6BA3D05D0EA46FBF0E12
:104A1400A56F000EA66F6EEC0EF0630E0701C26F59
:104A24000A017C6B7D6B94D0000E861902E1000EA6
:104A34008519D8B4CAD5000E861902E1010E85196C
:104A4400D8B4C3D5000E861902E1020E8519D8B474
:104A5400BCD5000E861902E1030E8519D8B4B5D56C
:104A6400000E861902E1040E8519D8B4AED5000EE5
:104A7400861902E1050E8519D8B4A7D5000E86194A
:104A840002E1060E8519D8B436D6000E861902E165
:104A9400070E8519D8B465D6000E861902E1080EF2
:104AA4008519D8B45ED6000E861902E1090E85195F
:104AB400D8B457D6000E861902E10A0E8519D8B467
:104AC40050D6000E861902E10B0E8519D8B449D6CA
:104AD400000E861902E10C0E8519D8B442D6000ED8
:104AE400861902E10D0E8519D8B49FD6000E8619D9
:104AF40002E10E0E8519D8B4CED6000E861902E155
:104B04000F0E8519D8B4C7D6000E861902E1100E0F
:104B14008519D8B4C0D6000E861902E1110E851984
:104B2400D8B4B9D6000E861902E1120E8519D8B48C
:104B3400B2D6000E861902E1130E8519D8B4ABD68D
:104B4400000E861902E1140E8519D8B423D75DD757
:104B54000A01854B862B8C2B19D584EC08F0260E84
:104B64000A018C5D17E2010E07011C6F100E0A0189
:104B7400A46F000EA56F310EA66F9FEC0FF0080E08
:104B84000A01956F010E966FCAEC17F0630E0701C8
:104B9400C26F2ED007011C6B2250000803E2010EE5
:104BA4000001856F100E0A01A46F000EA56F300E70
:104BB400A66F9FEC0FF003EC10F0F8EC0FF00A0175
:104BC400A46BA56B630EA66F9FEC0FF00001866BC0
:104BD400876B496A0701C26BBC84CEEC11F00A01F1
:104BE4007C6B7D6B0901FC6B06EC11F00701C26B59
:104BF4000001856BFC0E0A01A46F090EA56F8A0ED5
:104C0400A66F010EA76F28EC0EF000C07CFA01C05D
:104C14007DFA000E026E0150025C02E100500008B1
:104C24000EE22D0E0A01A46FB60EA56F000EA66F3C
:104C34006EEC0EF029EC14F00A017C6B7D6B0A011A
:104C4400FC0EA46F090EA56F6F0EA66F010EA76F61
:104C540028EC0EF000C07CFA01C07DFA000E026E52
:104C64000150025C02E1005000086AE2535000085F
:104C74005AE22A50090A57E03050000A36E1BB8252
:104C84002A50000A17E1010E306EA10E0A01A46F2A
:104C9400000EA56F310EA66F9FEC0FF0030E0B6E86
:104CA400080E0C6E770E0D6E0D2EFED70C2EFCD753
:104CB4000B2EFAD72A50010A17E1750E0A01A46FC8
:104CC400B60EA56F000EA66F6EEC0EF0520E0B6EB4
:104CD4002B0E0C6E000E0D6E0D2EFED70C2EFCD777
:104CE4000B2EFAD70000BB921AD02A50000A17E103
:104CF400BB92306AA10E0A01A46F000EA56F300E9C
:104D0400A66F9FEC0FF0030E0B6E080E0C6E770E61
:104D14000D6E0D2EFED70C2EFCD70B2EFAD7010EDE
:104D24000A018D6F0BD00A01D50EA46FB60EA56FC4
:104D3400000EA66F6EEC0EF00A018D6B7C6B7D6B22
:104D44000A01FC0EA46F090EA56F660EA66F010E74
:104D5400A76F28EC0EF000C07CFA01C07DFA000EAB
:104D6400026E0150025C02E1005000086AE25450F5
:104D740000085AE22B50090A57E03150000A36E184
:104D8400BB842B50000A17E1010E316EA20E0A01FA
:104D9400A46F000EA56F310EA66F9FEC0FF0030EEB
:104DA4000B6E080E0C6E770E0D6E0D2EFED70C2EAC
:104DB400FCD70B2EFAD72B50010A17E1BD0E0A01BE
:104DC400A46FB60EA56F000EA66F6EEC0EF0520E19
:104DD4000B6E2B0E0C6E000E0D6E0D2EFED70C2ED0
:104DE400FCD70B2EFAD70000BB941AD02B50000A24
:104DF40017E1BB94316AA20E0A01A46F000EA56FDD
:104E0400300EA66F9FEC0FF0030E0B6E080E0C6EA7
:104E1400770E0D6E0D2EFED70C2EFCD70B2EFAD767
:104E2400020E0A018D6F0BD00A01A50EA46FB60EF7
:104E3400A56F000EA66F6EEC0EF00A018D6B7C6BF5
:104E44007D6B0A01FC0EA46F090EA56F810EA66F7F
:104E5400010EA76F28EC0EF000C07CFA01C07DFAA9
:104E6400000E026E0150025C02E1005000086AE28A
:104E7400555000085AE22C50090A57E03250000AF3
:104E840036E1BB862C50000A17E1010E326EA30EE8
:104E94000A01A46F000EA56F310EA66F9FEC0FF0F0
:104EA400030E0B6E080E0C6E770E0D6E0D2EFED7D4
:104EB4000C2EFCD70B2EFAD72C50010A17E18D0EBD
:104EC4000A01A46FB60EA56F000EA66F6EEC0EF06D
:104ED400520E0B6E2B0E0C6E000E0D6E0D2EFED7A9
:104EE4000C2EFCD70B2EFAD70000BB961AD02C50F0
:104EF400000A17E1BB96326AA30E0A01A46F000EE2
:104F0400A56F300EA66F9FEC0FF0030E0B6E080E0C
:104F14000C6E770E0D6E0D2EFED70C2EFCD70B2EBD
:104F2400FAD7030E0A018D6F0BD00A01150EA46F78
:104F3400B60EA56F000EA66F6EEC0EF00A018D6B17
:104F44007C6B7D6B0A01FC0EA46F090EA56F780EB5
:104F5400A66F010EA76F28EC0EF000C07CFA01C00A
:104F64007DFA000E026E0150025C02E1005000085E
:104F7400D8B079D05650000869E22D50090A66E08D
:104F84003350000A45E12D50090AD8A4BB882D509E
:104F9400090A09E1450E0A01A46FB60EA56F000EB9
:104FA400A66F6EEC0EF02D50000A17E1010E336E61
:104FB400A40E0A01A46F000EA56F310EA66F9FEC1C
:104FC4000FF0030E0B6E080E0C6E770E0D6E0D2E89
:104FD400FED70C2EFCD70B2EFAD72D50010A17E161
:104FE400250E0A01A46FB80EA56F000EA66F6EEC15
:104FF4000EF0520E0B6E2B0E0C6E000E0D6E0D2E5F
:10500400FED70C2EFCD70B2EFAD70000BB981AD073
:105014002D50000A17E1BB98336AA40E0A01A46F4D
:10502400000EA56F300EA66F9FEC0FF0030E0B6EF3
:10503400080E0C6E770E0D6E0D2EFED70C2EFCD7BF
:105044000B2EFAD7040E0A018D6F0BD00A01F50E50
:10505400A46FB70EA56F000EA66F6EEC0EF00A01DA
:105064008D6B7C6B7D6B0A01FC0EA46F090EA56F22
:10507400CB0EA66F010EA76F28EC0EF000C07CFAD1
:1050840001C07DFA000E026E0150025C02E1005084
:1050940000086EE2575000085EE20801BB51000AA6
:1050A4005AE12E50090A57E03450000A36E1BA8E0C
:1050B4002E50000A17E1010E346EA50E0A01A46FEA
:1050C400000EA56F310EA66F9FEC0FF0030E0B6E52
:1050D400080E0C6E770E0D6E0D2EFED70C2EFCD71F
:1050E4000B2EFAD72E50010A17E1550E0A01A46FB0
:1050F400B80EA56F000EA66F6EEC0EF0520E0B6E7E
:105104002B0E0C6E000E0D6E0D2EFED70C2EFCD742
:105114000B2EFAD70000BB981AD02E50000A17E1C4
:10512400BA9E346AA50E0A01A46F000EA56F300E54
:10513400A66F9FEC0FF0030E0B6E080E0C6E770E2D
:105144000D6E0D2EFED70C2EFCD70B2EFAD7050EA6
:105154000A018D6F0BD00A013D0EA46FB80EA56F26
:10516400000EA66F6EEC0EF00A018D6B7C6B7D6BEE
:105174000A01FC0EA46F090EA56FC00EA66F010EE6
:10518400A76F28EC0EF000C07CFA01C07DFA000E77
:10519400026E0150025C02E10050000810E28B0E26
:1051A4000A01A46FBC0EA56F000EA66F6EEC0EF084
:1051B400010E486E010E466E0A017C6B7D6B0A017E
:1051C400FC0EA46F090EA56FDC0EA66F010EA76F6F
:1051D40028EC0EF000C07CFA01C07DFA000E026ECD
:1051E4000150025C02E10050000817E29D0E0A0122
:1051F400A46FBE0EA56F000EA66F6EEC0EF0090E26
:105204000B6E1E0E0C6EE40E0D6E0D2EFED70C2EC4
:10521400FCD70B2EFAD70000FF00FC0E0A01A46F86
:10522400090EA56FD40EA66F010EA76F28EC0EF021
:1052340000C07CFA01C07DFA000E026E0150025CCF
:1052440002E10050000837E2B60E0A01A46F010E15
:10525400A56F21EC0EF0070E7C25E96E000E7D2172
:10526400EA6E6F00A7FFE9FF6F00ABFFEAFF6F0074
:10527400B8FFBCF8300E0801BC5D14E3340EBC5D0D
:1052840011E2070E0A017C25E96E000E7D21EA6E0B
:105294006F00A7FFE9FF6F00ABFFEAFF300EEE5C83
:1052A40007011C6F0A017C6B7D6B060E956F010E66
:1052B400966FCAEC17F00A018D5100083AE2070113
:1052C4001C6B100E0A01A46F000EA56F300EA66FA2
:1052D4009FEC0FF0030E0B6E080E0C6E770E0D6E26
:1052E4000D2EFED70C2EFCD70B2EFAD79E0E0A01DC
:1052F400A46FB40EA56F000EA66F6EEC0EF0300E08
:105304000A018D25C16F80EC00F0C90E0A01A46F5B
:10531400BB0EA56F000EA66F6EEC0EF00A018D6B2E
:10532400080E956F010E966FCAEC17F00A018D6B8B
:1053340062D0BC8ABC98BC96000E956F000E966F26
:10534400160E976F880E986FF40E996F010E9A6F70
:10535400DDEC19F0BC9ABC98BC96290E0B6E960E27
:105364000C6E7F0E0D6E0D2EFED70C2EFCD70B2E61
:10537400FAD7BC8ABC98BC96000E0A01956F000E41
:10538400966F160E976F880E986FF40E996F010E34
:105394009A6FDDEC19F0BC9ABC98BC96290E0B6E82
:1053A400960E0C6E7F0E0D6E0D2EFED70C2EFCD7B6
:1053B4000B2EFAD7BC8ABC98BC96000E0A01956FD6
:1053C400000E966F160E976F880E986FF40E996FF5
:1053D400010E9A6FDDEC19F0BC9ABC98BC96290EAC
:1053E4000B6E960E0C6E7F0E0D6E0D2EFED70C2ED0
:0E53F400FCD70B2EFAD7ADEC0DF0D28E1200C6
:10540200296A090E2A6E090E2B6E090E2C6E090EE0
:085412002D6E090E2E6E120032
:10541A000901646B0A017F6B806B856B51EC1CF090
:10542A004C0E0A01BB6F000EBC6F8C0EBD6F000ED6
:10543A00BE6F040EBF6F13EC04F0000E011802E1F8
:10544A00000E00180FE1010E0A01A46FB40EA56F39
:10545A00000EA66F6EEC0EF0140E0901646F140EA6
:10546A00006E89D00A017F6B806B000E801902E101
:10547A007E517F1960E04C0EBB6F000EBC6F050EAB
:10548A00006E000E016E7FCA04F080CA05F0CCECF3
:10549A000FF0960E0024BD6F000E0120BE6F040EA1
:1054AA00BF6F13EC04F0000E011802E1000E0018A1
:1054BA0011E10A017F510A0F0901646FA30E0A0163
:1054CA00A46FBB0EA56F000EA66F6EEC0EF064C93A
:1054DA0000F051D04C0E0A01BB6F000EBC6F110ECA
:1054EA00006E000E016E7FCA04F080CA05F0CCEC93
:1054FA000FF0EE0E0024BD6F000E0120BE6F040EE9
:10550A00BF6F13EC04F0000E011802E1000E001840
:10551A0011E10A017F511E0F0901646F9C0E0A01F5
:10552A00A46FBA0EA56F000EA66F6EEC0EF064C9DA
:10553A0000F021D011D08F0E0A01A46FBD0EA56F05
:10554A00000EA66F6EEC0EF0300E0A017E25C16FBA
:10555A0080EC00F084EC08F00A017F4B802B800E6F
:10556A008019006E800E005C02E1060E7F5DD8A0F5
:08557A007CD764C900F01200A7
:1055820008017C6B040E7A6F7B6B4C0E0A01A46FD0
:10559200000EA56F170EA66FC20EA76F000EA86FA2
:1055A200EBEC0DF04C6ABC9ABC989A0E0A01A46FFF
:1055B200B20EA56F000EA66F6EEC0EF000018A4BC4
:1055C2008B2B670E0A01A46F090EA56F7C0EA66FC6
:1055D200BB0EA76F000EA86FEBEC0DF08AC0A4FA09
:1055E2008BC0A5FA6E0E0A01A66F090EA76FD8EC42
:1055F20007F02A0E0901736F300E07011C250901FD
:10560200776F670E0A01A46F090EA56F21EC0EF0E9
:105612003E01F88100000000F8A101D0FDD76F0023
:10562200C0FBE7F9000E0901E86FE7C919F70701A6
:10563200186B3E01EF5107011827000E1923225063
:10564200000803E29CEC1FF002D084EC08F0030E89
:1056520007011C5D03E2ADEC0DF007D03901939711
:105662009EEC21F000C0B6F8236AA1919181080155
:105672007B6BBF6B0901FB9F1E0E0A01956F000E2B
:10568200966FCEEC19F003EC17F02350010A16E1E5
:105692004A50010A13E12250020A02E1E2EC21F02F
:1056A2000001866B0801B76BB86BBD6BBE6B476AB6
:1056B2000001876B496ABC84BC98BC9A000189517D
:1056C200040A02E1B00E8819D8B4BC8889510408D2
:1056D20002E18851B5080EE2060E0A01A46FBF0E60
:1056E200A56F000EA66F6EEC0EF0BC9ABC9800017E
:1056F200886B896BCCA204D04850010A01E033D0F8
:10570200020E0B6EA00E0C6E920E0D6E0D2EFED7BB
:105712000C2EFCD70B2EFAD70000CCB21FD0020EF3
:105722000B6EA00E0C6E920E0D6E0D2EFED70C2E71
:10573200FCD70B2EFAD70000CCA2F1D7010E466E91
:10574200BC9ABC988551010A09E1A60E0A01A46F10
:10575200C10EA56F000EA66F6EEC0EF04850010A46
:1057620002E1010E466E4650010A01E106D009012E
:10577200FBBF03D0FBB301D086D70901FBA33AD00C
:1057820008017C51000836E20901FB93010E080171
:105792007B6FB70E0A01A46FB20EA56F000EA66F43
:1057A2006EEC0EF04C0E0A01A46F000EA56F120EE5
:1057B200A66FC20EA76F000EA86FEBEC0DF04C6A3D
:1057C20008017C51585C02E37C51585E7C6BBC8AB8
:1057D200BC98000E0A01956F000E966F160E976F19
:1057E200880E986FF40E996F010E9A6FDDEC19F026
:1057F200BC9AECD00901FBAFE9D008017B51000A49
:10580200D8A4E4D0476ABC9ABC88BC9600018551F2
:10581200010A09E1DB0E0A01A46FC00EA56F000E9A
:10582200A66F6EEC0EF0000E0A01956F000E966FD9
:10583200160E976F890E986FF40E996F010E9A6F7C
:10584200DDEC19F0030E08017C5D24E25150000AE0
:1058520011E100018551010A09E1CD0E0A01A46F8F
:10586200C00EA56F000EA66F6EEC0EF0BC86BC9A41
:10587200BC9810D000018551010A09E1320E0A01DB
:10588200A46FC00EA56F000EA66F6EEC0EF0BC8A60
:10589200BC98BC96290E0B6E960E0C6E7F0E0D6E8A
:1058A2000D2EFED70C2EFCD70B2EFAD700018551F8
:1058B200010A09E1F70E0A01A46FC00EA56F000EDE
:1058C200A66F6EEC0EF0BC9ABC980801BF51230A79
:1058D20031E1930E0A01A46FAC0EA56F000EA66F04
:1058E2006EEC0EF008017C51585C02E37C51585E6C
:1058F2007C6B4C0E0A01A46F000EA56F030EA66FFF
:10590200C20EA76F000EA86FEBEC0DF04C6ABC98AC
:10591200BC8A000E0A01956F000E966F160E976FE5
:10592200880E986FE80E996F030E9A6FDDEC19F0EE
:10593200BC9A4CD008017C51030802E2030E7C6F32
:105942004C0EE16E000EE26E7C51E126D8B0E22AE6
:105952006F0087FFE1FF6F008BFFE2FF6200FFF243
:10596200E6FF7C2B582AB50E0A01A46FBE0EA56F66
:10597200000EA66F6EEC0EF00A0E046E58C000F018
:1059820066EC0FF0300E00240A01C16F80EC00F0CB
:105992000A0E046E58C000F066EC0FF008C000F06A
:1059A200300E00240A01C16F80EC00F03D0E0A01A6
:1059B200A46FBF0EA56F000EA66F6EEC0EF04C0E1C
:1059C2000A01A46F000EA56F21EC0EF00901FB9FE6
:1059D2004650010A01E105D008017A517C5DD8A048
:1059E200EDD50A017E6B7F6B4650010A01E134D08E
:1059F2004C0E7E25E96E000E7F21EA6E6F00A7FF36
:105A0200E9FF6F00ABFFEAFF6F00B8FFBCF8BCC84C
:105A120095FA0DEC10F00050000A12E17F0EA46F0F
:105A2200A70EA56F000EA66F6EEC0EF008017C6B40
:105A32005850030802E2040E585E2A0EBF6F0CD0C3
:105A42000A017E4B7F2B800E7F19006E800E005C58
:0A5A520002E1040E7E5DC8E31200BD
:105A5C00960E0A01A46F000EA56F350EA66FC20E2E
:105A6C00A76F000EA86FEBEC0DF09B0E0A01A46F54
:105A7C00000EA56F210EA66FC20EA76F000EA86FA9
:105A8C00EBEC0DF0A00E0A01A46F000EA56F080E32
:105A9C00A66FC20EA76F000EA86FEBEC0DF0A50E53
:105AAC000A01A46F000EA56FFE0EA66FC10EA76FA4
:105ABC00000EA86FEBEC0DF0AA0E0A01A46F000EFD
:105ACC00A56F0D0EA66FC20EA76F000EA86FEBECA4
:105ADC000DF0AF0E0A01A46F000EA56F1C0EA66F81
:0E5AEC00C20EA76F000EA86FEBEC0DF01200BB
:105AFA0039019491050EB56EB28AB298B292B294F7
:105B0A00B39EB46ACF0EB16E2C0EB06E8481000EB5
:105B1A000801BA1902E1000EB91904E1040EB96FBD
:105B2A00000EBA6F0901FB933901A491B2901200D9
:105B3A0039019791050EA26EA16A9E6A770EA06E30
:105B4A00F30E9F6E0901FB8939018781A791A08E07
:045B5A00978112001D
:105B5E0000018551010A1BE15B0E0A01A46FAA0E1A
:105B6E00A56F000EA66F6EEC0EF06C0E0A01A46F00
:105B7E00B10EA56F000EA66F6EEC0EF0F80E0A01B8
:105B8E00A46FA40EA56F000EA66F6EEC0EF03F0173
:105B9E003E9F3E993E91D40E0101E46F090EE56FD2
:105BAE00000EE66F000EE76F000E0901466F400E05
:105BBE00476F1D0E486F8A0E496F00018551010A0D
:105BCE003FE1120E0A01A46FAB0EA56F000EA66F79
:105BDE006EEC0EF0E4C185FAE5C186FAE6C187FAED
:105BEE00E7C188FA670E0A01896F090E8A6FD6EC33
:105BFE001BF0670EA46F090EA56F21EC0EF0440E7C
:105C0E00A46FC20EA56F000EA66F6EEC0EF046C905
:105C1E00A4FA47C9A5FA48C9A6FA49C9A7FA670E50
:105C2E000A01A86F090EA96F010EAA6FA2EC08F067
:105C3E00670EA46F090EA56F21EC0EF084EC08F030
:105C4E00E40E0701C36F010EC46F00018551010AF6
:105C5E0020E1D80E0A01A46FBD0EA56F000EA66F2F
:105C6E006EEC0EF0E4C185FAE5C186FAE6C187FA5C
:105C7E00E7C188FA670E0A01896F090E8A6FD6ECA2
:105C8E001BF0670EA46F090EA56F21EC0EF084ECCD
:105C9E0008F0020E0701C325E96E000EC421EA6E5C
:105CAE006F00A7FFE9FF6F00ABFFEAFF6F00BBFFBE
:105CBE003DFF010EC325E96E000EC421EA6E6F0092
:105CCE00A7FFE9FF6F00ABFFEAFF6F00BBFF3CFFD2
:105CDE0061000FFFE9FF610013FFEAFF6F00BBFFDA
:105CEE003BFF1A6B030E1B6F00018551010AD8A4EE
:105CFE0092D0EE0E0A01A46FBB0EA56F000EA66F1A
:105D0E006EEC0EF0300E07011B250801BC6FBCC8EF
:105D1E00C1FA80EC00F0560E0A01A46FC00EA56FFA
:105D2E00000EA66F6EEC0EF0030E006E000E016EEE
:105D3E001BC704F0000E056ECCEC0FF0DF0E002436
:105D4E00E96E000E0120EA6E6F00A7FFE9FF6F00FB
:105D5E00ABFFEAFF6F00B8FFA4FA6F00B8FFA5FA19
:105D6E006F00B8FFA6FA6EEC0EF01BC700F0000E27
:105D7E00016E026E036E0036009001360236033657
:105D8E0000360090013602360336680E0024F66E99
:105D9E00BB0E0120F76E000E0220F86E6F00DBFFC7
:105DAE00F6FF6F00DFFFF7FF6F00E3FFF8FF09005C
:105DBE006F00D4FF4EF909006F00D4FF4FF90900B0
:105DCE006F00D4FF50F909006F00D4FF51F9090E8E
:105DDE000A01C16F80EC00F04EC9A4FA4FC9A5FAB2
:105DEE0050C9A6FA51C9A7FA670E0A01A86F090E83
:105DFE00A96F010EAA6FA2EC08F0670EA46F090E30
:105E0E00A56F21EC0EF0CB0EA46FC10EA56F000E88
:105E1E00A66F6EEC0EF0050E016E1AC700F0015063
:105E2E0004E000360090FF0FFBD707011B51001056
:105E3E003F013F6F00018551010A09E1C40E0A01BD
:105E4E00A46FA30EA56F000EA66F6EEC0EF0E4C14C
:105E5E0000F0E5C101F0E6C102F0E7C103F08FECFE
:105E6E0008F01BC704F0000E056E066E076E0436B2
:105E7E000490053606360736043604900536063687
:105E8E000736680E0424F66EBB0E0520F76E000E64
:105E9E000620F86E6F00DBFFF6FF6F00DFFFF7FFE7
:105EAE006F00E3FFF8FF09006F00D4FF04F0090054
:105EBE006F00D4FF05F009006F00D4FF06F0090053
:105ECE006F00D4FF07F09DEC05F0000E046E000E7F
:105EDE00056E000E066E940E076E3AEC06F000C0CC
:105EEE004AF901C04BF902C04CF903C04DF900014B
:105EFE008551010A2EE1980E0A01A46FB50EA56F09
:105F0E00000EA66F6EEC0EF04AC9A4FA4BC9A5FAA4
:105F1E004CC9A6FA4DC9A7FA670E0A01A86F090E59
:105F2E00A96F010EAA6FA2EC08F0670EA46F090EFE
:105F3E00A56F21EC0EF084EC08F0290E0B6E960E78
:105F4E000C6E7F0E0D6E0D2EFED70C2EFCD70B2E6B
:085F5E00FAD70901FB8B1200C8
:105F66004B6A0A017E6B7F6B806B816B060EA46F9A
:105F7600A70EA56F000EA66F6EEC0EF003EC10F0E8
:105F860007011C6B4A6A4B6A70D3090E4B6E0801F7
:105F9600BF6B516ACB0E0A01A46FB30EA56F000E3C
:105FA600A66F6EEC0EF0586A08017C6B040E7A6FD1
:105FB6004AEC1CF0F8EC0FF04C0E0A01A46F000E30
:105FC600A56FD60EA66FC10EA76F000EA86FEBECDD
:105FD6000DF04C6A000E0A01A46F000EA56F160E96
:105FE600A66F890EA76F24EC08F00A01806B816BFF
:105FF600806B816B41EC1AF0BF512A0A03E1090E4E
:106006004B6E87D0960E0A01A46F000EA56FD10EB7
:10601600A66FC10EA76F000EA86FEBEC0DF04C0E2D
:106026000A01BB6F000EBC6F960EBD6F000EBE6FF1
:10603600040EBF6F13EC04F0000E011802E1000E0F
:10604600001853E1710E0A01A46FBD0EA56F000E74
:10605600A66F6EEC0EF0050E006E000E016E7ECA87
:1060660004F07FCA05F0CCEC0FF0960E00240A016E
:10607600A46F000E0120A56F21EC0EF0BF0EA46FD9
:10608600C10EA56F000EA66F6EEC0EF0BC8ABC9812
:10609600BC9600018551010A09E1FA0E0A01A46FB6
:1060A600BF0EA56F000EA66F6EEC0EF0520E0B6EB5
:1060B6002B0E0C6E000E0D6E0D2EFED70C2EFCD781
:1060C6000B2EFAD70000BC9ABC9800018551010A34
:1060D60009E18E0E0A01A46FC00EA56F000EA66F11
:1060E6006EEC0EF0010E4B6E14D0500E0A01A46F2A
:1060F600B00EA56F000EA66F6EEC0EF0960E0A019E
:10610600A46F000EA56F21EC0EF084EC08F0090ECA
:106116004B6EC8D24D0E0A01A46FB10EA56F000ECC
:10612600A66F6EEC0EF0090E4B6ED6EC1EF0BF514C
:10613600300A3BE100018551010A09E1F20E0A012C
:10614600A46FBF0EA56F000EA66F6EEC0EF0BC8A94
:10615600BC98BC96D00E0A01A46FB40EA56F000EB3
:10616600A66F6EEC0EF0520E0B6E2B0E0C6E000E22
:106176000D6E0D2EFED70C2EFCD70B2EFAD7000077
:10618600BC9ABC9800018551010A09E16B0E0A010F
:10619600A46FC00EA56F000EA66F6EEC0EF00A017E
:1061A600804B812B020E4B6E0BD00A01CA0EA46FD8
:1061B600B80EA56F000EA66F6EEC0EF0090E4B6EB4
:1061C60071D2A80E0A01A46FAF0EA56F000EA66FBE
:1061D6006EEC0EF0090E4B6ED6EC1EF0290E0B6E11
:1061E600960E0C6E7F0E0D6E0D2EFED70C2EFCD766
:1061F6000B2EFAD7BF512A0A38E1120E0A01A46FF4
:10620600BC0EA56F000EA66F6EEC0EF00001855158
:10621600010A09E1D20E0A01A46FBF0EA56F000E96
:10622600A66F6EEC0EF0BC8ABC98BC96520E0B6E36
:106236002B0E0C6E000E0D6E0D2EFED70C2EFCD7FF
:106246000B2EFAD70000BC9ABC9800018551010AB2
:1062560009E1790E0A01A46FC00EA56F000EA66FA4
:106266006EEC0EF0030E4B6E0BD0B00E0A01A46F4F
:10627600B30EA56F000EA66F6EEC0EF0090E4B6EF8
:1062860011D26C0E0A01A46FA90EA56F000EA66F9F
:106296006EEC0EF0090E4B6E0A01806B816B010EDF
:1062A600516E41EC1AF0BF512A0A03E1090E4B6EFA
:1062B60098D0BC8ABC98BC9600018551010A09E1B8
:1062C6000A0E0A01A46FC00EA56F000EA66F6EEC33
:1062D6000EF0520E0B6E2B0E0C6E000E0D6E0D2E6A
:1062E600FED70C2EFCD70B2EFAD70000BC9ABC9812
:1062F60000018551010A09E1870E0A01A46FC00E4B
:10630600A56F000EA66F6EEC0EF0F40E0A01A46FD8
:10631600BD0EA56F000EA66F6EEC0EF04C0E0A01B8
:10632600A46F000EA56F21EC0EF084EC08F00A01B4
:10633600806B816BD30EA46FB20EA56F000EA66F95
:106346006EEC0EF08C0E0A01A46F000EA56F21EC08
:106356000EF04C0EBB6F000EBC6F8C0EBD6F000EA8
:10636600BE6F040EBF6F13EC04F0000E011802E1BD
:10637600000E00180DE1960E0A01A46FBF0EA56F60
:10638600000EA66F6EEC0EF00A01804B812B09D031
:106396000A011C0EA46FBE0EA56F000EA66F6EEC52
:1063A6000EF0800E006E800E0A018119005C02E17B
:1063B600805100080BE2290EA46FBE0EA56F000ED9
:1063C600A66F6EEC0EF0090E4B6E0BD0A90E0A01ED
:1063D600A46FBE0EA56F000EA66F6EEC0EF0040E37
:1063E6004B6E60D1D10E0A01A46FB00EA56F000EE0
:1063F600A66F6EEC0EF0090E4B6ED6EC1EF0BF517A
:106406002A0AD8A48BD0BC86BC9ABC9800018551B8
:10641600010A09E1640E0A01A46FC00EA56F000E01
:10642600A66F6EEC0EF0520E0B6E2B0E0C6E000E5F
:106436000D6E0D2EFED70C2EFCD70B2EFAD70000B4
:10644600BC9ABC9800018551010A09E1480E0A016F
:10645600A46FC00EA56F000EA66F6EEC0EF0960E22
:106466000A01956F000E966F4C0E976F000E986F8F
:10647600040E996F000E9A6F19EC10F0960EA46F29
:10648600000EA56F21EC0EF0C50EA46FC10EA56F10
:10649600000EA66F6EEC0EF0010E526E020E0A0191
:1064A600A46FBE0EA56F000EA66F6EEC0EF0BC8A32
:1064B600BC98BC9600018551010A09E1CA0E0A0181
:1064C600A46FBF0EA56F000EA66F6EEC0EF0000E49
:1064D6000A01956F000E966F160E976F880E986FCD
:1064E600F40E996F010E9A6FDDEC19F0BC9ABC9808
:1064F60000018551010A09E1720E0A01A46FC00E5E
:10650600A56F000EA66F6EEC0EF00A01806B816B14
:10651600BC8407011C6B050E4B6E0BD0720E0A0174
:10652600A46FBA0EA56F000EA66F6EEC0EF0090EE4
:106536004B6EB8D084EC08F0630E0001B46F160EF3
:106546000A01A46FAC0EA56F000EA66F6EEC0EF0DE
:10655600D2AE03D00801C08102D00801C091CEECB2
:1065660011F0B70E0A01A46FB40EA56F000EA66F48
:106576006EEC0EF0010E4A6E0801C0A101D0D28E5B
:106586000701C26B8FD0360E0A01A46FB40EA56F39
:10659600000EA66F6EEC0EF04B6A690E0A01A46F30
:1065A600BC0EA56F000EA66F6EEC0EF00001876B99
:1065B600866BBC84BC8A000E0A01956F000E966F2E
:1065C600160E976F880E986FF40E996F010E9A6FDC
:1065D600DDEC19F0BC9A290E0B6E960E0C6E7F0E32
:1065E6000D6E0D2EFED70C2EFCD70B2EFAD7BC8ABD
:1065F600000E0A01956F000E966F160E976F880EA5
:10660600986FF40E996F010E9A6FDDEC19F0BC9A33
:10661600290E0B6E960E0C6E7F0E0D6E0D2EFED78E
:106626000C2EFCD70B2EFAD7BC8A000E0A01956FEA
:10663600000E966F160E976F880E986FF40E996F70
:10664600010E9A6FDDEC19F0BC9A290E0B6E960EB0
:106656000C6E7F0E0D6E0D2EFED70C2EFCD70B2E5C
:10666600FAD74B6A1FD04B6A1DD04B50000AD8B4DC
:106676008CD44B50010AD8B44DD54B50020AD8B42D
:10668600A0D54B50030AD8B4FCD54B50040AD8B455
:10669600A9D64B50050AD8B44DD74B50090AD8B4E1
:0E66A60072D7E1D74A50000AD8B46ED4120061
:1066B400C4EC1BF03C0E0A01856F430E866F000E7E
:1066C400876F000E886F000E896F010E8A6FC10EEE
:1066D4008B6F0A0E8C6FFF0E8D6FFF0E8E6F000E88
:1066E4008F6F000E906FC40E916F000E926F000EAC
:1066F400936F000E946FA1EC21F0856B866BC2EC56
:0467040021F012006E
:106708003A01406BCA6AC280C282C284C286C298F9
:10671800BA98C29ABA9AC29CBA9C800E416FC28E2D
:10672800506BCB6AE10EC36EFF0E516F3E01BC6B1E
:10673800B86BC3803A01508BC38EC38CC392BB9293
:10674800C394BB94C396BB96C398BB98C28E606B28
:10675800CC6ACA0EC46EFF0E616FC490BC90C4822E
:10676800C494BC84C496BC96C498C49ABC98BC9A79
:086778003E01C16BC19F12003C
:10678000050E0A017E5D44E2110EA46FBF0EA56FD7
:10679000000EA66F6EEC0EF0300E0A017E25C16F62
:1067A00080EC00F0830E0A01A46FC10EA56F000EED
:1067B000A66F6EEC0EF0120E0A017E25F66EC00E6C
:1067C000F76E000EF722000EF86E000EF8226F0032
:1067D000DBFFF6FF6F00DFFFF7FF6F00E3FFF8FF5F
:1067E00009006F00D4FF00F0001E0050CB14BB6EF8
:1067F0002F0EE16E000EE26E7E51E126D8B0E22A45
:106800006F0087FFE1FF6F008BFFE2FFE66A21D098
:106810007E51050A1EE10801BB51000A1AE1180E5B
:106820000A01A46FBB0EA56F000EA66F6EEC0EF0F2
:10683000BA8E2F0EE16E000EE26E0A017E51E12645
:10684000D8B0E22A6F0087FFE1FF6F008BFFE2FF05
:04685000E66A1200E2
:10685400520EE96E000EEA6E0001DA51E926D8B054
:10686400EA2A6F00A7FFE9FF6F00ABFFEAFFEE50D3
:106874000008D8B00FD2DC0E0A01A46FB90EA56FC0
:10688400000EA66F6EEC0EF084EC08F00001DA51F5
:106894000008D8B0FBD1060EDA5DD8B0F7D19F0E50
:1068A4000A01A46FBF0EA56F000EA66F6EEC0EF06A
:1068B400300E0001DA250A01C16F80EC00F0290EC8
:1068C400E96E000EEA6E0001DA51E926D8B0EA2A30
:1068D4006F00A7FFE9FF6F00ABFFEAFF6F00B8FF8F
:1068E4007EFA000E0A017F6F000E7F6FB8D12F0E63
:1068F400E96E000EEA6E0001DA51E926D8B0EA2A00
:106904006F00A7FFE9FF6F00ABFFEAFFEE50000A3C
:1069140052E1B90E0A01A46FC10EA56F000EA66F55
:106924006EEC0EF00001DA51050A02E1BA8E1BD0BA
:10693400120EDA25F66EC00EF76E000EF722000E68
:10694400F86E000EF8226F00DBFFF6FF6F00DFFF2A
:10695400F7FF6F00E3FFF8FF09006F00D4FF00F0BA
:106964000050CB10BB6E2F0EE16E000EE26EDA51BA
:10697400E126D8B0E22A6F0087FFE1FF6F008BFFAA
:10698400E2FF010EE66EDA51A00F0A01A46FA56BB7
:10699400000EA523310EA66F9FEC0FF0030E0B6EB5
:1069A400080E0C6E770E0D6E0D2EFED70C2EFCD736
:1069B4000B2EFAD751D0950E0A01A46FC00EA56F05
:1069C400000EA66F6EEC0EF00001DA51050A02E12A
:1069D400BA9E1CD0120EDA25F66EC00EF76E000EAB
:1069E400F722000EF86E000EF8226F00DBFFF6FFB0
:1069F4006F00DFFFF7FF6F00E3FFF8FF09006F0090
:106A0400D4FF00F0001E0050CB14BB6E2F0EE16EBD
:106A1400000EE26EDA51E126D8B0E22A6F0087FF59
:106A2400E1FF6F008BFFE2FFE66ADA51A00F0A0173
:106A3400A46FA56B000EA523300EA66F9FEC0FF07C
:106A4400030E0B6E080E0C6E770E0D6E0D2EFED718
:106A54000C2EFCD70B2EFAD70701C26B16D1B00E41
:106A64000A01A46FB90EA56F000EA66F6EEC0EF0AE
:106A74000001DA51050A02E1BA8E1BD0120EDA25A2
:106A8400F66EC00EF76E000EF722000EF86E000EC2
:106A9400F8226F00DBFFF6FF6F00DFFFF7FF6F00E8
:106AA400E3FFF8FF09006F00D4FF00F00050CB10A3
:106AB400BB6E2F0EE16E000EE26EDA51E126D8B005
:106AC400E22A6F0087FFE1FF6F008BFFE2FF010EF8
:106AD400E66E520E0B6E2B0E0C6E000E0D6E0D2E0E
:106AE400FED70C2EFCD70B2EFAD70000C10E0A01DC
:106AF400A46FBE0EA56F000EA66F6EEC0EF0120E04
:106B04000001DA25F66EC00EF76E000EF722000EB5
:106B1400F86E000EF8226F00DBFFF6FF6F00DFFF58
:106B2400F7FF6F00E3FFF8FF09006F00D4FF00F0E8
:106B3400001E0050CB14BB6E2F0EE16E000EE26EF1
:106B4400DA51E126D8B0E22A6F0087FFE1FF6F0037
:106B54008BFFE2FFE66ADA51A00F0A01A46FA56B6E
:106B6400000EA523300EA66F9FEC0FF0030E0B6EE4
:106B7400080E0C6E770E0D6E0D2EFED70C2EFCD764
:106B84000B2EFAD70701C26B80D0BC0E0A01A46F8A
:106B9400BD0EA56F000EA66F6EEC0EF00001DA516B
:106BA400050A02E1BA9E1CD0120EDA25F66EC00E5A
:106BB400F76E000EF722000EF86E000EF8226F003A
:106BC400DBFFF6FF6F00DFFFF7FF6F00E3FFF8FF67
:106BD40009006F00D4FF00F0001E0050CB14BB6E00
:106BE4002F0EE16E000EE26EDA51E126D8B0E22AF1
:106BF4006F0087FFE1FF6F008BFFE2FFE66ADA5167
:106C0400A00F0A01A46FA56B000EA523300EA66F7A
:106C14009FEC0FF0030E0B6E080E0C6E770E0D6ECC
:106C24000D2EFED70C2EFCD70B2EFAD7060E000124
:106C3400DB6F000EDC6F520E0B6E2B0E0C6E000E13
:106C44000D6E0D2EFED70C2EFCD70B2EFAD700009E
:106C54000701C26B1AD00701630EC26F16D0000E73
:106C64000A017F1902E1000E7E19D8B440D6000E45
:106C74007F1902E1010E7E19D8B4F1D6000E7F19F6
:106C840002E1090E7E1981E0E6D703D0630E070105
:106C9400C26F1ED0CA0E0A01A46FBD0EA56F000EEE
:106CA400A66F6EEC0EF0300E0001DA250A01C16FFA
:106CB40080EC00F0E80E0A01A46FB10EA56F000E7F
:106CC400A66F6EEC0EF084EC08F0630E0701C26F41
:026CD4001200AC
:106CD6000A01806B816B7E6B7F6B826B836B540EBC
:106CE600A46FBB0EA56F000EA66F6EEC0EF00A0128
:106CF600956B966BE4EC16F000C0B4F0050E0B6EC7
:106D06000F0E0C6EF10E0D6E0D2EFED70C2EFCD74F
:106D16000B2EFAD7B4C085FA670E0A01866F090EE4
:106D2600876F5FEC21F0670EA46F090EA56F21EC4B
:106D36000EF084EC08F0020E0A01A46FB50EA56FE2
:106D4600000EA66F6EEC0EF0100E0A01826F000E9A
:106D5600836F100E956F000E966FE4EC16F000C070
:106D660084FA030E0B6E080E0C6E770E0D6E0D2E4A
:106D7600FED70C2EFCD70B2EFAD70A018451330806
:106D860002E2330E846F84CAC1FA80EC00F084EC10
:106D960008F0300E0A01845D016E01C01CF7030E77
:106DA600015CD8B023D2630EA46FA80EA56F000EA7
:106DB600A66F6EEC0EF00A017E6B7F6B800E7F195C
:106DC600006E800E005C02E1060E7E5DD8B0BBD080
:106DD600800EA46FC00EA56F000EA66F6EEC0EF0AF
:106DE600300E0A017E25C16F80EC00F05D0E0A01AF
:106DF600A46FC20EA56F000EA66F6EEC0EF0040E09
:106E0600026E7ECA00F07FCA01F0025005E000362D
:106E160000900136FF0FFAD7200E0026000E012241
:106E260000C082FA01C083FA00C0A4FA01C0A5FA24
:106E3600670E0A01A66F090EA76FE3EC0EF0670E48
:106E4600A46F090EA56F21EC0EF0440EA46FC20EBE
:106E5600A56F000EA66F6EEC0EF00A01806B816BBB
:106E6600800E8119006E800E005C02E1040E805DCA
:106E760037E280518225956F81518321966FE4EC2C
:106E860016F000C084FA030E0B6E080E0C6E770E19
:106E96000D6E0D2EFED70C2EFCD70B2EFAD7050E37
:106EA600006E000E016E7ECA04F07FCA05F0CCECBF
:106EB6000FF0960E0026000E01220A0180510024D2
:106EC600E16E81510120E26E6F0087FFE1FF6F00E6
:106ED6008BFFE2FF620013FAE6FF804B812BC0D7DF
:106EE600050E006E000E016E7ECA04F07FCA05F024
:106EF600CCEC0FF0960E0026000E012280510024E5
:106F0600E16E81510120E26E6F0087FFE1FF6F00A5
:106F16008BFFE2FFE66A050E006E000E016E7ECA6A
:106F260004F07FCA05F0CCEC0FF0960E0024A46F97
:106F3600000E0120A56F21EC0EF084EC08F00A018A
:106F46007E4B7F2B3BD7CC0EA46FA90EA56F000EF0
:106F5600A66F6EEC0EF00A017E6B7F6B800E7F19BA
:106F6600006E800E005C02E1060E7E5D38E2800E49
:106F76007E25006E000E7F21016E00C082FA01C0E0
:106F860083FA00C095FA01C096FAE4EC16F000C048
:106F960084FA030E0B6E080E0C6E770E0D6E0D2E18
:106FA600FED70C2EFCD70B2EFAD784CAC1FA80EC7A
:106FB60000F0290E0A017E25E16E000E7F21E26EA9
:106FC600300E845D006E6F0087FFE1FF6F008BFF60
:106FD600E2FF600003F0E6FF7E4B7F2BBFD78A0EF1
:106FE600A46FAA0EA56F000EA66F6EEC0EF00A0136
:106FF6007E6B7F6B800E7F19006E800E005C02E157
:10700600060E7E5D38E2900E7E25006E000E7F2114
:10701600016E00C082FA01C083FA00C095FA01C071
:1070260096FAE4EC16F000C084FA030E0B6E080E16
:107036000C6E770E0D6E0D2EFED70C2EFCD70B2E7A
:10704600FAD784CAC1FA80EC00F0520E0A017E25F6
:10705600E16E000E7F21E26E300E845D006E6F00E1
:1070660087FFE1FF6F008BFFE2FF600003F0E6FFA2
:107076007E4B7F2BBFD7B90EA46FA70EA56F000E50
:10708600A66F6EEC0EF00A017E6B7F6B800E7F1989
:10709600006E800E005C02E1060E7E5D38E2A00EF8
:1070A6007E25006E000E7F21016E00C082FA01C0AF
:1070B60083FA00C095FA01C096FAE4EC16F000C017
:1070C60084FA030E0B6E080E0C6E770E0D6E0D2EE7
:1070D600FED70C2EFCD70B2EFAD784CAC1FA80EC49
:1070E60000F02F0E0A017E25E16E000E7F21E26E72
:1070F600300E845D006E6F0087FFE1FF6F008BFF2F
:10710600E2FF600003F0E6FF7E4B7F2BBFD73E0E0B
:10711600A46FAF0EA56F000EA66F6EEC0EF00A01FF
:107126007E6B7F6B800E7F19006E800E005C02E125
:10713600040E7E5D35E2B00E7E25006E000E7F21C8
:10714600016E00C082FA01C083FA00C095FA01C040
:1071560096FAE4EC16F000C084FA030E0B6E080EE5
:107166000C6E770E0D6E0D2EFED70C2EFCD70B2E49
:10717600FAD784CAC1FA80EC00F0240E0A017E25F3
:10718600E16E000E7F21E26E6F0087FFE1FF6F0068
:107196008BFFE2FF620013FAE6FF7E4B7F2BC2D71E
:1071A600400EA46FAC0EA56F000EA66F6EEC0EF02F
:1071B600C00E0A01956F000E966FE4EC16F000C043
:1071C60084FA030E0B6E080E0C6E770E0D6E0D2EE6
:1071D600FED70C2EFCD70B2EFAD784CAC1FA80EC48
:1071E60000F0300E0A01845D226E78D0430EA46F43
:1071F600A70EA56F000EA66F6EEC0EF0300E0701FF
:107206001C250A01C16F80EC00F084EC08F0200E0A
:107216000A01826F000E836F200EA46F000EA56F09
:10722600670EA66F090EA76FE3EC0EF0670EA46F4C
:10723600090EA56F21EC0EF0440EA46FC20EA56FC9
:10724600000EA66F6EEC0EF00A01806B816B800E4D
:107256008119006E800E005C02E1040E805D29E259
:1072660080518225956F81518321966FE4EC16F04B
:1072760000C084FA030E0B6E080E0C6E770E0D6EB0
:107286000D2EFED70C2EFCD70B2EFAD7960E0A0122
:107296008025E16E000E8121E26E6F0087FFE1FF1F
:1072A6006F008BFFE2FF620013FAE6FF804B812B33
:1072B600CED7960E8025E16E000E8121E26E6F001C
:1072C60087FFE1FF6F008BFFE2FFE66A960EA46F71
:1072D600000EA56F21EC0EF084EC08F084EC08F0AB
:0272E600120094
:1072E8005350000805E230B002D0BB9201D0BB82F7
:1072F8005450000805E231B002D0BB9401D0BB84E1
:107308005550000805E232B002D0BB9601D0BB86CA
:107318005650000805E233B002D0BB9801D0BB88B4
:107328005750000809E20801BB51000A05E134B0D2
:0A73380002D0BA9E01D0BA8E1200F6
:1073420009006F00D7FFE6FF0006FAE10106F8E147
:02735200120027
:1073CC0000C01FF001C01EF002C01DF03901A3A7C0
:1073DC0075D093A773D09EEC21F000C0B6F83D0198
:1073EC00F9AB0FD0F99B010E0901ED25006E000ED3
:1073FC00EE21016E00C0EDF901C0EEF96F00A0F7AF
:10740C00B6F83D01F9A70FD0010E0901ED25006E6C
:10741C00000EEE21016E00C0EDF901C0EEF99EECFC
:10742C0021F000C0B6F80801B6510A0A0FE0020EAE
:10743C000001DD5D016E000EDE59026E0901535133
:10744C00025C02E15251015C01E31AD00901010E08
:10745C00236EFC0E5625E16E090E5721E26E6F006D
:10746C0087FFE1FF6F008BFFE2FFE66A390193971C
:10747C0056C952F957C953F90901566B576B1ED0AF
:10748C00236AFC0E5625E16E090E5721E26E6F0041
:10749C0087FFE1FF6F008BFFE2FF6200DBF2E6FF8C
:1074AC0056C952F957C953F9010E5625006E000EF4
:1074BC005721016E00C056F901C057F91FC000F0EA
:0A74CC001EC001F01DC002F0110007
:1074D8000CC021F00DC020F03901A1A113D091A159
:1074E80011D02A0E0C6E8D0E0D6E0D2EFED70C2EA1
:1074F800FCD700000000CBA002D00901FB8F3901A6
:0E750800A191919121C00CF020C00DF0110056
:1075180000C01CF001C01BF002C01AF03901A7A17D
:1075280076D097A174D0030E07011C5D29E2800E66
:10753800006E800E0001DC19005C02E1DB510008DE
:107548001FE2010EDB15016EDCC002F0000E021610
:10755800000E021802E1000E011804E13F013E8FFF
:10756800BC8A03D03F013E9FBC9A010E0001DB5D3F
:10757800006E000EDC59016E00C0DBF001C0DCF0CB
:107588004750010A40E1010E0801BD25006E000EBA
:10759800BE21016E00C0BDF801C0BEF8010EBD15C8
:1075A800016EBEC802F0000E0216000E021802E1BB
:1075B800010E011802E1BC8A01D0BC9A0801000E34
:1075C800006EB851005C02E1B75100081CE2010EE0
:1075D800B75D006E000EB859016E00C0B7F801C063
:1075E800B8F8010EB715016EB8C802F0000E021601
:1075F800000E021802E1010E011803E13F013E8F5F
:1076080002D03F013E9F3901A791F30E9F6E1CC027
:0C76180000F01BC001F01AC002F01100CD
:1076240030EC61F0600E3901D96F080EDF6FDCBDFC
:1076340001D0FDD7090E0B6E1E0E0C6EE40E0D6EFE
:107644000D2EFED70C2EFCD70B2EFAD7000084EC9F
:1076540033F0236A0901FB93FB95606B616B5E6BEE
:107664005F6B0801B96BBA6B0001DB6BDC6B856B7C
:107674000901FB9B0101E46BE56BE66BE76BE40E30
:107684000701C36F010EC46FF8EC06F0170EE56F27
:10769400156B260E106F146B136B33EC06F0080198
:1076A400C46BC56B000EC55D02E1050EC45D10E23E
:1076B4004C0EC425E16E000EC521E26E6F0087FFFB
:1076C400E1FF6F008BFFE2FFE66AC44BC52BEAD7EC
:1076D4007F0E0001DD6F000EDE6F0801C46BC56B09
:1076E400010E0001DD5D016E000EDE59026E0250D6
:1076F4000801C55D02E10150C45D10E2FC0EC42521
:10770400E16E090EC521E26E6F0087FFE1FF6F0095
:107714008BFFE2FFE66AC44BC52BE2D7C46BC56B93
:10772400000EC55D02E17F0EC45D10E2670EC42544
:10773400E16E090EC521E26E6F0087FFE1FF6F0065
:107744008BFFE2FFE66AC44BC52BEAD7C46BC56B5B
:10775400000EC55D02E17F0EC45D10E2C60EC425B5
:10776400E16E080EC521E26E6F0087FFE1FF6F0036
:107774008BFFE2FFE66AC44BC52BEAD7C60EC26F85
:10778400080EC36F240E0A01A46F000EA56FEF0E3E
:10779400A66FC10EA76F000EA86FEBEC0DF08A0E5A
:1077A4003D01F56F000EF66FF28F5AEC33F03C0E8C
:1077B4000A01856F430E866F000E876F000E886F77
:1077C400000E896F010E8A6FC10E8B6F0A0E8C6FCB
:1077D400FF0E8D6FFF0E8E6F000E8F6F000E906F79
:1077E400C40E916F000E926F000E936F000E946F93
:1077F400A1EC21F0090E0B6E1E0E0C6EE40E0D6E44
:107804000D2EFED70C2EFCD70B2EFAD70000870EB8
:10781400A46FBA0EA56F000EA66F6EEC0EF00801F1
:10782400C46BC56B000EC55D02E10C0EC45D32E293
:10783400030E006E000E016EC4C804F0C5C805F046
:10784400CCEC0FF0B60E0024E96E000E0120EA6EB7
:107854006F00A7FFE9FF6F00ABFFEAFF6F00B8FFFF
:10786400A4FA6F00B8FFA5FA6F00B8FFA6FA6EEC91
:107874000EF0090E0B6E1E0E0C6EE40E0D6E0D2E28
:10788400FED70C2EFCD70B2EFAD700000801C44BF0
:10789400C52BC8D784EC08F00801C46BC56B000E77
:1078A400C55D02E1060EC45D10E22F0EC425E16E33
:1078B400000EC521E26E6F0087FFE1FF6F008BFFB2
:1078C400E2FFE66AC44BC52BEAD703EC10F04AEC9E
:1078D4001CF02EEC2DF001EC2AF007011C6B84EC5B
:1078E40008F0466A660E0A01A46FB50EA56F000E75
:1078F400A66F6EEC0EF0470E0A01A46FBC0EA56FC6
:10790400000EA66F6EEC0EF0000ECBBE010E0A0147
:10791400C16F300EC12780EC00F0E60E0A01A46F9F
:10792400BD0EA56F000EA66F6EEC0EF0000ECBBC64
:10793400010E0A01C16F300EC12780EC00F084EC07
:1079440008F0CBBE03D0CBBC01D006D0CBAE03D065
:10795400CBAC01D001D015D0FC0E0A01A46FA90E46
:10796400A56F000EA66F6EEC0EF0020E0801BB6F41
:10797400C90E0A01A46FB10EA56F000EA66F6EECBE
:107984000EF0CBAE18D0CBBC16D0C29EBA9E080166
:10799400BB6B020E0A01A46FBD0EA56F000EA66F8D
:1079A4006EEC0EF0CF0E0A01A46FAD0EA56F000EA3
:1079B400A66F6EEC0EF0CBBE24D0CBAC22D0C28E20
:1079C400010E0801BB6F190E0A01A46FA40EA56F66
:1079D400000EA66F6EEC0EF0CAAE0AD0BB0E0A0102
:1079E400A46FAC0EA56F000EA66F6EEC0EF009D05E
:1079F400E30E0A01A46FAC0EA56F000EA66F6EEC29
:107A04000EF01E0E0A01A46FBA0EA56F000EA66F2B
:107A14006EEC0EF0240E0A01A46FBC0EA56F000ECE
:107A2400A66F6EEC0EF0DB0E0A01A46FBA0EA56F02
:107A3400000EA66F6EEC0EF01DC7A4FA1EC7A5FAC1
:107A4400670E0A01A66F090EA76FD8EC07F0670E40
:107A5400A46F090EA56F21EC0EF02F0EA46FC10EBA
:107A6400A56F000EA66F6EEC0EF01FC7A4FA20C718
:107A7400A5FA670E0A01A66F090EA76FD8EC07F0E6
:107A8400670EA46F090EA56F21EC0EF084EC08F0CC
:107A9400B10E0A01A46FBA0EA56F000EA66F6EECAC
:107AA4000EF0E8C1A4FAE9C1A5FA670E0A01A66FAF
:107AB400090EA76FD8EC07F0670EA46F090EA56F27
:107AC40021EC0EF0280EA46FC10EA56F000EA66F58
:107AD4006EEC0EF083C8A4FA84C8A5FA670E0A01F6
:107AE400A66F090EA76FD8EC07F0670EA46F090EF6
:107AF400A56F21EC0EF084EC08F0040E0A01A46FCB
:107B0400BB0EA56F000EA66F6EEC0EF080C8A4FA33
:107B140081C8A5FA670E0A01A66F090EA76FD8ECF3
:107B240007F0670EA46F090EA56F21EC0EF0210E6D
:107B3400A46FC10EA56F000EA66F6EEC0EF07EC88A
:107B4400A4FA7FC8A5FA670E0A01A66F090EA76FEB
:107B5400D8EC07F0670EA46F090EA56F21EC0EF0A8
:107B640084EC08F084EC08F0290E0B6E960E0C6E73
:107B74007F0E0D6E0D2EFED70C2EFCD70B2EFAD7D2
:107B8400FC0E0A01A46FB50EA56F000EA66F6EEC75
:107B94000EF0000ECCB2010E0A01C16F300EC127E7
:107BA40080EC00F084EC08F0D76AD66A080ED56E33
:107BB4003901A18B3D01F399F38FF2893901838750
:107BC4003D01F49DADEC0DF05B9187818191D280F4
:107BD4009191D28EBC84C60E0801C26F080EC36F89
:107BE40084EC08F00001856B480E0A01A46FA60E10
:107BF400A56F000EA66F6EEC0EF0AFEC2DF0000139
:107C04008A6B8B6B84EC08F03E01C18FC197C195E0
:107C1400C183C181C38A3A01508B3E01F96BFA6B6F
:107C2400FB6BF86BF885F8993F0EFF6F030EFD6F41
:107C34000D0EF16FF88F0000F88100000000F8A12C
:107C440001D0FDD76F00C0FBE7F9000E0901E86F12
:107C5400E7C919F70701186B3E01EF51070118270F
:107C6400000E1923900E0A01A46FBB0EA56F000E1F
:107C7400A66F6EEC0EF06F00FCFB85FA670E0A012E
:107C8400866F090E876F5FEC21F0670EA46F090EF3
:107C9400A56F21EC0EF084EC08F03B0E0A01A46FF2
:107CA400A90EA56F000EA66F6EEC0EF00001B46B6A
:107CB400466AA80E0A01A46FBF0EA56F000EA66F38
:107CC4006EEC0EF0C60E0A01A46FBA0EA56F000E7C
:107CD400A66F6EEC0EF0300E46240A01C16F80ECE4
:107CE40000F084EC08F04650010A0BE107011C6B1C
:107CF400100E0A01A46F000EA56F300EA66F9FEC44
:107D04000FF00A01856B51EC1CF0330E0A01A46FCD
:107D1400BA0EA56F000EA66F6EEC0EF07DEC2DF082
:107D2400850E0A01A46FAF0EA56F000EA66F6EEC50
:107D34000EF09DEC2DF00001DB6BDC6B0801BF6BDA
:107D4400010E0001856F4B6A516A0701C26B000185
:107D5400B56BDA6B08017C6B040E7A6F586A4C0EB3
:107D64000A01A46F000EA56FDB0EA66FC10EA76FEC
:107D7400000EA86FEBEC0DF04C6ABC9ABC880001B5
:107D8400866B0801BD6BBE6B476A0001876B496A4D
:107D940084EC08F04A6A0A01956B966BE4EC16F0E1
:107DA40000C0B4F0050E0B6E0F0E0C6EF10E0D6ECE
:107DB4000D2EFED70C2EFCD70B2EFAD7430E0A013C
:107DC400A46FBE0EA56F000EA66F6EEC0EF00A0E29
:107DD400046EB4C000F066EC0FF0300E00240A010B
:107DE400C16F80EC00F00A0E046EB4C000F066ECC3
:107DF4000FF008C000F0300E00240A01C16F80ECBF
:107E040000F084EC08F0000E0A01A46F000EA56FC8
:107E1400160EA66F890EA76F24EC08F00001B4516A
:107E2400630A25E184EC08F0010E4A6E06EC11F0B9
:107E3400DD0EA46FB70EA56F000EA66F6EEC0EF0EC
:107E4400D2AE03D00801C08102D00801C091D29EF5
:107E54006BEC36F007011C51020802E2030E1C6FA2
:107E640074EC39F00801C0A101D0D28E37D0240EB1
:107E74000A01A46F000EA56FF40EA66FC10EA76FC2
:107E8400000EA86FEBEC0DF003EC10F0F8EC0FF023
:107E94002EEC2DF001EC2AF04AEC1CF007011C6BCF
:107EA40084EC08F03D0E0A01A46FA50EA56F000E28
:107EB400A66F6EEC0EF00A01956B010E966FCAEC7C
:107EC40017F0000E0A01A46F000EA56F160EA66F20
:107ED400890EA76F24EC08F0B3EC2FF0000E0A0112
:107EE400A46F000EA56F160EA66F890EA76F24EC63
:107EF40008F00001DB6BDC6B466A486AE0EF4CF08B
:107F0400586A0701C26B630EC26F070E0A01A46FA1
:107F1400A60EA56F000EA66F6EEC0EF0CD0E0A0134
:107F2400A46FBE0EA56F000EA66F6EEC0EF0300EA1
:107F340007011C250A01C16F80EC00F084EC08F0F5
:107F4400010E516E000E0A01A46F000EA56F160EED
:107F5400A66F890EA76F24EC08F0C1EC2AF04650F6
:107F6400010A0AE1810E0A01A46FAD0EA56F000E8D
:107F7400A66F6EEC0EF09DD60801BF512A0A04E1EB
:107F8400630E0701C26F05D0070186C047F0010EDA
:107F9400C26F2DEF4DF0770E0A01A46FBE0EA56FD0
:107FA400000EA66F6EEC0EF0B10E0A01A46FBF0EA8
:107FB400A56F000EA66F6EEC0EF04C0E0A01BB6F9F
:107FC400000EBC6F960EBD6F000EBE6F040EBF6F29
:107FD40013EC04F0000E011802E1000E00183AE15F
:107FE4002C0E0A01A46FAA0EA56F000EA66F6EECEC
:107FF4000EF000018551010A09E1E20E0A01A46FA5
:10800400BF0EA56F000EA66F6EEC0EF0BC8ABC9876
:10801400BC96520E0B6E2B0E0C6E000E0D6E0D2EBA
:10802400FED70C2EFCD70B2EFAD700000001855189
:10803400010A09E11A0E0A01A46FC10EA56F000E10
:10804400A66F6EEC0EF0BC9ABC98BC96020E0701AB
:10805400C26F7DD0010E0801C46F000EC56F4C0EB7
:108064000A01BB6F000EBC6F050E006E000E016EA0
:10807400C4C804F0C5C805F0CCEC0FF0960E00247B
:10808400BD6F000E0120BE6F040EBF6F13EC04F031
:10809400000E011802E1000E00183BE1EF0E0A0188
:1080A400A46FB20EA56F000EA66F6EEC0EF0000169
:1080B4008551010A09E1050E0A01A46FC10EA56FDD
:1080C400000EA66F6EEC0EF0BC86BC9ABC98520EE5
:1080D4000B6E2B0E0C6E000E0D6E0D2EFED70C2E9D
:1080E400FCD70B2EFAD7000000018551010A09E1E3
:1080F4000C0E0A01A46FC10EA56F000EA66F6EECE4
:108104000EF0BC9ABC98C4C8DAF0070E0701C26F1F
:1081140009D00801C44BC52B000EC55D02E1060E53
:10812400C45D9DE30801000E006EC551005C02E1D0
:10813400C45105080CE21C0E0A01A46FB40EA56F0D
:10814400000EA66F6EEC0EF0630E0701C26F2DEFEA
:108154004DF0A80E0A01A46FAD0EA56F000EA66F18
:108164006EEC0EF0630E0701C26F1C6B476A496A1E
:10817400BC90D6EC1EF0300EBF5DD8A0D9D2BF5152
:108184003908D8A0D5D2BC8ABC98BC9600018551C8
:10819400010A09E1DA0E0A01A46FBF0EA56F000EF1
:1081A400A66F6EEC0EF0520E0B6E2B0E0C6E000EC4
:1081B4000D6E0D2EFED70C2EFCD70B2EFAD7000019
:1081C40000018551010A09E1130E0A01A46FC10ED1
:1081D400A56F000EA66F6EEC0EF0BC9ABC98300E24
:1081E4000801BF5D0001DA6F620E0A01A46FBD0EC3
:1081F400A56F000EA66F6EEC0EF0BFC8C1FA80EC3E
:1082040000F084EC08F06BD2010E516E030E0701EE
:10821400C26F8ED2240E0A01A46FB20EA56F000E97
:10822400A66F6EEC0EF0D20E0A01A46FAE0EA56F0F
:10823400000EA66F6EEC0EF0630E0701C26FD6EC53
:108244001EF0BF512A0A2DE1BC88BC9A000E0A0117
:10825400956F000E966F160E976F890E986FE80E45
:10826400996F030E9A6FDDEC19F0BC98BC8A520E1C
:108274000B6E2B0E0C6E000E0D6E0D2EFED70C2EFB
:10828400FCD70B2EFAD70000BC9A600E0A01A46F2B
:10829400C10EA56F000EA66F6EEC0EF0050E070161
:1082A400C26F46D2B80E0A01A46FAA0EA56F000EC3
:1082B400A66F6EEC0EF0D6EC1EF0BF512A0A2DE12B
:1082C40000018551010A09E1BA0E0A01A46FBF0E2B
:1082D400A56F000EA66F6EEC0EF0BC8ABC98BC961F
:1082E400520E0B6E2B0E0C6E000E0D6E0D2EFED765
:1082F4000C2EFCD70B2EFAD7000000018551010A81
:1083040009E1360E0A01A46FC10EA56F000EA66F17
:108314006EEC0EF0BC9ABC9804D0630E0701C26FD9
:1083240007D2D20E0A01A46FA80EA56F000EA66F85
:108334006EEC0EF0D6EC1EF000018551010A09E145
:10834400C20E0A01A46FBF0EA56F000EA66F6EECDD
:108354000EF0BC8ABC98BC96520E0B6E2B0E0C6EA3
:10836400000E0D6E0D2EFED70C2EFCD70B2EFAD759
:10837400000000018551010A09E1440E0A01A46FBD
:10838400C10EA56F000EA66F6EEC0EF0BC9ABC98E1
:10839400BFC8BCF81A0E0A01A46FAF0EA56F000E79
:1083A400A66F6EEC0EF0D6EC1EF0BF512A0A2FE138
:1083B40000018551010A09E12A0E0A01A46FC00EC9
:1083C400A56F000EA66F6EEC0EF0BC8ABC98BC962E
:1083D400520E0B6E2B0E0C6E000E0D6E0D2EFED774
:1083E4000C2EFCD70B2EFAD7000000018551010A90
:1083F40009E1B80E0A01A46FC00EA56F000EA66FA6
:108404006EEC0EF0BC9ABC980701C26B04D0070155
:10841400630EC26F8DD117D0226A0001856B1ED006
:108424000001010E226E010E856F18D00001010EAD
:10843400856F020E226E12D00801BC6B226A630E95
:108444000701C26F0BD00801BC51300AE5E0BC51F2
:10845400310AE6E0BC51320AE9E0EED7910E0A0196
:10846400A46FBE0EA56F000EA66F6EEC0EF0BCC816
:10847400C1FA80EC00F084EC08F0C00E0A01A46F8D
:10848400000EA56F300E2224A66F9FEC0FF0030E92
:108494000B6E080E0C6E770E0D6E0D2EFED70C2E85
:1084A400FCD70B2EFAD700018551010A09E1220EEF
:1084B4000A01A46FC00EA56F000EA66F6EEC0EF03D
:1084C400BC8ABC98BC96000E0A01956F000E966F8C
:1084D400160E976F880E986FE80E996F030E9A6FB9
:1084E400DDEC19F000018551010A09E1BF0E0A0112
:1084F400A46FC00EA56F000EA66F6EEC0EF0BC9AB2
:10850400BC9816D1AA0E0A01A46FB10EA56F000E75
:10851400A66F6EEC0EF01A0E0A01A46FAE0EA56FD4
:10852400000EA66F6EEC0EF0630E0701C26FD6EC60
:108534001EF0BF512A0A2DE1BC88BC9A000E0A0124
:10854400956F000E966F160E976F890E986FE80E52
:10855400996F030E9A6FDDEC19F0BC98BC8A520E29
:108564000B6E2B0E0C6E000E0D6E0D2EFED70C2E08
:10857400FCD70B2EFAD70000BC9A9C0E0A01A46FFC
:10858400C00EA56F000EA66F6EEC0EF00A0E07016A
:10859400C26FCED03E0E0A01A46FAB0EA56F000EC3
:1085A400A66F6EEC0EF0630E0701C26F890E0A010E
:1085B400A46FAE0EA56F000EA66F6EEC0EF0D6EC97
:1085C4001EF0BF512A0A3BE1BC88BC8A520E0B6ED6
:1085D4002B0E0C6E000E0D6E0D2EFED70C2EFCD73E
:1085E4000B2EFAD70000BC98BC8A000E0A01956FC6
:1085F400000E966F160E976F880E986FE80E996F9F
:10860400030E9A6FDDEC19F0520E0B6E2B0E0C6EEE
:10861400000E0D6E0D2EFED70C2EFCD70B2EFAD7A6
:108624000000AA0E0A01A46FC00EA56F000EA66F6B
:108634006EEC0EF0BC9A080E0701C26F03D007015E
:10864400630EC26F75D0E90E0A01A46FB40EA56F54
:10865400000EA66F6EEC0EF0630E0701C26F3F0EA4
:108664000A01A46FAE0EA56F000EA66F6EEC0EF09D
:10867400D6EC1EF0BF512A0A2DE1BC88BC9A000E2C
:108684000A01956F000E966F160E976F890E986FFC
:10869400E80E996F030E9A6FDDEC19F0BC98BC8A52
:1086A400520E0B6E2B0E0C6E000E0D6E0D2EFED7A1
:1086B4000C2EFCD70B2EFAD70000BC9AE90E0A0147
:1086C400A46FC00EA56F000EA66F6EEC0EF0160E12
:1086D4000701C26F2DD00701630EC26F29D00001BC
:1086E400DA51000AD8B490D5DA51010AD8B492D537
:1086F400DA51020AD8B48ED5DA51030AD8B48AD52D
:10870400DA51040AD8B486D5DA51050AD8B482D528
:10871400DA51060AD8B4C6D5DA51070AD8B4F2D663
:10872400DA51080AD8B436D7DA51090A8CE0D3D71B
:108734002DEF4DF05D0E0A01A46FBE0EA56F000E65
:10874400A66F6EEC0EF0F00E0A01A46FC00EA56FBA
:10875400000EA66F6EEC0EF0300E0001DA250A0151
:10876400C16F80EC00F084EC08F00001DA51050AD6
:108774001FE10801BB51000A1BE0B20E0A01A46FFD
:10878400B00EA56F000EA66F6EEC0EF0520E0B6EBF
:108794002B0E0C6E000E0D6E0D2EFED70C2EFCD77C
:1087A4000B2EFAD70000630E0701C26F2DEF4DF0B8
:1087B4008BD00701630EC26F6A0E0A01A46FAB0E61
:1087C400A56F000EA66F6EEC0EF0D6EC1EF0BF5136
:1087D4002A0A2EE1BC88BC9A000E0A01956F000E8D
:1087E400966F160E976F890E986FE80E996F030EA9
:1087F4009A6FDDEC19F0BC98BC8A520E0B6E2B0EEE
:108804000C6E000E0D6E0D2EFED70C2EFCD70B2E0B
:10881400FAD70000BC9AE20E0A01A46FC00EA56F3D
:10882400000EA66F6EEC0EF0040E0701C26F03D0AB
:108834000701630EC26F5DD0640E0A01A46FAE0E11
:10884400A56F000EA66F6EEC0EF0630E0701C26FEB
:10885400D6EC1EF0BF512A0A2FE1BC88BC9A000E48
:108864000A01956F000E966F160E976F890E986F1A
:10887400E80E996F030E9A6FDDEC19F0BC88BC8A80
:10888400520E0B6E2B0E0C6E000E0D6E0D2EFED7BF
:108894000C2EFCD70B2EFAD70000BC98BC9AD40E31
:1088A4000A01A46FC00EA56F000EA66F6EEC0EF049
:1088B400050E0701C26F03D00701630EC26F19D002
:1088C4000701630EC26F15D00001DA51000AD8B453
:1088D40070D7DA51010AB0E0DA51020AADE0DA5198
:1088E400030AAAE0DA51040AA7E0DA51050AA4E06F
:1088F400E7D72DEF4DF0360E0A01A46FBE0EA56F1B
:10890400000EA66F6EEC0EF0630E0701C26F500EE0
:108914000A01A46FB40EA56F000EA66F6EEC0EF0E4
:10892400010E516EC1EC2AF0290E0B6E960E0C6EE0
:108934007F0E0D6E0D2EFED70C2EFCD70B2EFAD704
:10894400BC98BC9A8D0E0A01A46FBF0EA56F000ED1
:10895400A66F6EEC0EF04C0E0A01A46F000EA56F0C
:1089640021EC0EF084EC08F00A01856B51EC1CF04C
:10897400F60E0A01A46FAE0EA56F000EA66F6EEC84
:108984000EF00901586B596B0801C46BC56B0A01E1
:108994007E6B0DEC2AF000C0BCF80801BC51000845
:1089A4001EE22E0E0A01A46FB10EA56F000EA66F73
:1089B4006EEC0EF0BCC885FA670E0A01866F090ECC
:1089C400876F5FEC21F0670EA46F090EA56F21EC91
:1089D4000EF084EC08F0630E0701C26F8CD00B0E0E
:1089E4000A01A46FB30EA56F000EA66F6EEC0EF015
:1089F400D6EC1EF0BF512A0AD8A47DD0BC8ABC880C
:108A0400520E0B6E2B0E0C6E000E0D6E0D2EFED73D
:108A14000C2EFCD70B2EFAD70000BC8ABC98000E93
:108A24000A01956F000E966F160E976F880E986F59
:108A3400F40E996F010E9A6FDDEC19F0BC9AEC0EEE
:108A44000A01A46FAB0EA56F000EA66F6EEC0EF0BC
:108A540007011C6B200E0901E76F000EE86F080187
:108A6400C46BC56B000EC55D02E1040EC45D26E255
:108A74004C0EC425E96E000EC521EA6E6F00A7FFF7
:108A8400E9FF6F00ABFFEAFF6F00B8FFC1F8960E75
:108A9400C425E16E000EC521E26E6F0087FFE1FF81
:108AA4006F008BFFE2FF620007F3E6FFC1C8C1FA63
:108AB40080EC00F00801C44BC52BD4D700019A6B9D
:108AC400CEEC11F00A01856B51EC1CF00001866BB1
:108AD4000801B76BB86B0001876B496A080E0A017D
:108AE400A46FBA0EA56F000EA66F6EEC0EF0BC84D8
:108AF4000701C26B00D02DEF4DF0BC88C10E0A01F6
:108B0400A46FAB0EA56F000EA66F6EEC0EF0300EC8
:108B14000001DA250A01C16F80EC00F084EC08F052
:108B24002B0E0A01A46FA80EA56F000EA66F6EECA3
:108B34000EF0D6EC1EF000C0BCF8300EBC5D016E29
:108B440001C0B5F00150000A08E00001B551010A66
:108B540004E0B551090A01E0E1D0BC8ABC98520E88
:108B64000B6E2B0E0C6E000E0D6E0D2EFED70C2E02
:108B7400FCD70B2EFAD70000BC9A290E0B6E960E6A
:108B84000C6E7F0E0D6E0D2EFED70C2EFCD70B2E09
:108B9400FAD7960E0A01A46FAB0EA56F000EA66F4E
:108BA4006EEC0EF00001866BD6EC1EF000C0BCF833
:108BB400BC512A0AD8A4AED0E30E0A01A46FB50EA4
:108BC400A56F000EA66F6EEC0EF0300E0001DA25D4
:108BD4000A01C16F80EC00F0200E0A01C16F80EC25
:108BE40000F00001B551000A1CE1500E0A01A46F07
:108BF400BE0EA56F000EA66F6EEC0EF0290EE16E90
:108C0400000EE26E0001DA51E126D8B0E22A6F00CC
:108C140087FFE1FF6F008BFFE2FFE66A060E0701A4
:108C2400C26F0001B551010A21E1F10E0A01A46FDE
:108C3400BC0EA56F000EA66F6EEC0EF0DAC07EFAC5
:108C4400C0EC33F0290EE16E000EE26E0001DA5141
:108C5400E126D8B0E22A6F0087FFE1FF6F008BFFA7
:108C6400E2FF010EE66E060E0701C26F0001B55168
:108C7400090A21E1580E0A01A46FBC0EA56F000E6B
:108C8400A66F6EEC0EF0DAC07EFAC0EC33F0290E5B
:108C9400E16E000EE26E0001DA51E126D8B0E22A5C
:108CA4006F0087FFE1FF6F008BFFE2FF090EE66EA6
:108CB400330E0701C26F84EC08F0BC8ABC98BC96E2
:108CC40000018551010A09E11A0E0A01A46FC00EC0
:108CD400A56F000EA66F6EEC0EF0520E0B6E2B0EEF
:108CE4000C6E000E0D6E0D2EFED70C2EFCD70B2E27
:108CF400FAD7000000018551010A09E1910E0A0129
:108D0400A46FC10EA56F000EA66F6EEC0EF0BC9A98
:108D1400BC9803D0630E0701C26F03D00701630E32
:108D2400C26F2DEF4DF0230E0A01A46FBD0EA56F87
:108D3400000EA66F6EEC0EF0520EE16E000EE26EA7
:108D44000001DA51E126D8B0E22A6F0087FFE1FF83
:108D54006F008BFFE2FFE66A290EE16E000EE26E01
:108D6400DA51E126D8B0E22A6F0087FFE1FF6F00F5
:108D74008BFFE2FF090EE66E0801C46BC56B000EA3
:108D8400C55D02E1040EC45D1FE2050E006E000E17
:108D9400016EDAC004F0000E056ECCEC0FF0960EF6
:108DA4000026000E0122C4510024E16EC5510120A9
:108DB400E26E6F0087FFE1FF6F008BFFE2FF2E0E74
:108DC400E66EC44BC52BDBD72F0EE16E000EE26EB0
:108DD4000001DA51E126D8B0E22A6F0087FFE1FFF3
:108DE4006F008BFFE2FFE66ADAC07EFAC0EC33F074
:108DF40007011C6BBC84CEEC11F00A01856B51ECAD
:108E04001CF00701C26B2DEF4DF00F0E0A01A46F89
:108E1400BE0EA56F000EA66F6EEC0EF0CB0E0A010F
:108E2400A46FAF0EA56F000EA66F6EEC0EF0010ED0
:108E3400516EC1EC2AF00801BF512A0A04E1630E05
:108E44000701C26F2DD11C0E0A01A46FBF0EA56FBE
:108E5400000EA66F6EEC0EF04C0E0A01A46F000E0D
:108E6400A56F21EC0EF084EC08F0DAC07EFA0DEC6C
:108E74002AF000C0BCF8BC8ABC98BC96000185519D
:108E8400010A09E1020E0A01A46FC00EA56F000ECB
:108E9400A66F6EEC0EF0520E0B6E2B0E0C6E000EC7
:108EA4000D6E0D2EFED70C2EFCD70B2EFAD700001C
:108EB40000018551010A09E18A0E0A01A46FC10E5D
:108EC400A56F000EA66F6EEC0EF0BC9ABC9808015C
:108ED400BC51000AD8A4E1D00F0E0A01A46FB10E50
:108EE400A56F000EA66F6EEC0EF0D6EC1EF0BF510F
:108EF4002A0AD8A4CED0C46BC56B000EC55D02E1AE
:108F0400040EC45D34E24C0EC425E96E000EC52186
:108F1400EA6E6F00A7FFE9FF6F00ABFFEAFF6F0087
:108F2400B8FFC1F8050E006E000E016EDAC004F041
:108F3400000E056ECCEC0FF0960E0026000E0122FA
:108F4400C4510024E16EC5510120E26E6F0087FF19
:108F5400E1FF6F008BFFE2FF620007F3E6FFC1C889
:108F6400C1FA80EC00F00801C44BC52BC6D7050E2E
:108F7400006E000E016EDAC004F0000E056ECCEC3B
:108F84000FF0960E0026000E0122040E0024E16E5E
:108F9400000E0120E26E6F0087FFE1FF6F008BFF80
:108FA400E2FFE66ABC86BC9ABC9800018551010ABE
:108FB40009E16E0E0A01A46FC10EA56F000EA66F23
:108FC4006EEC0EF0520E0B6E2B0E0C6E000E0D6E30
:108FD4000D2EFED70C2EFCD70B2EFAD70000000165
:108FE4008551010A09E1750E0A01A46FC10EA56F2E
:108FF400000EA66F6EEC0EF0BC9ABC98BC8ABC98AE
:10900400BC9600018551010A09E1C40E0A01A46F4E
:10901400730EA56F000EA66F6EEC0EF0000E0A0123
:10902400956F000E966F160E976F880E986FF40E5C
:10903400996F010E9A6FDDEC19F0BC9ABC9800018F
:109044008551010A09E1980E0A01A46FC10EA56FAA
:10905400000EA66F6EEC0EF0520EE16E000EE26E84
:109064000001DA51E126D8B0E22A6F0087FFE1FF60
:109074006F008BFFE2FF010EE66E07011C6BBC84E0
:10908400CEEC11F00A01856B51EC1CF00701C26BA8
:1090940003D00701630EC26F03D00701630EC26FD2
:1090A4002DEF4DF01C6B476A496ABC90620E0A01B1
:1090B400A46FAF0EA56F000EA66F6EEC0EF0300E0F
:1090C4000001DA250A01C16F80EC00F02AEC34F0CB
:1090D400BC8A000E0A01956F000E966F160E976FEC
:1090E400880E986FF40E996F010E9A6FDDEC19F0EB
:1090F400BC9A0701C26B2DEF4DF05A0E0A01A46F02
:10910400AD0EA56F000EA66F6EEC0EF007011C6B82
:10911400100E0A01A46F000EA56F300EA66F9FEC0F
:109124000FF0030E0B6E080E0C6E770E0D6E0D2EE7
:10913400FED70C2EFCD70B2EFAD7010E466E070174
:10914400C26B2DEF4DF06A0E0A01A46FAC0EA56F31
:10915400000EA66F6EEC0EF0630E0701C26F4D0E8B
:109164000A01A46FB50EA56F000EA66F6EEC0EF08B
:109174000801C46BC56B000EC55D02E1040EC45D3D
:109184001BE2B00E0901E76F000EE86FB00E080194
:10919400C4250A01956F000E0801C5210A01966FC6
:1091A400E4EC16F000C0BCF8BCC8C1FA80EC00F0D6
:1091B4000801C44BC52BDFD71B0E0A01A46FB50EE3
:1091C400A56F000EA66F6EEC0EF00801C46BC56BA4
:1091D400000EC55D02E1040EC45D42E2000E0A0108
:1091E4007D1902E1000E7C193BE1ADEC0DF0480E57
:1091F4000A01A46FC20EA56F000EA66F6EEC0EF0EE
:10920400520E0B6E2B0E0C6E000E0D6E0D2EFED735
:109214000C2EFCD70B2EFAD700000A017C6B7D6B59
:10922400670EA46F090EA56F4B0EA66FC20EA76F33
:10923400000EA86FEBEC0DF00A01066BFC0EA46F98
:10924400090EA56F670EA66F090EA76F28EC0EF026
:1092540000C07CFA01C07DFA0801C44BC52BB8D705
:10926400FC0E0A01A46F090EA56F21EC0EF084EC2C
:1092740008F0000E006E0A017D51005C02E17C5191
:10928400000810E2BC88BC8A030E956F010E966F2D
:10929400CAEC17F0BC98BC9A84EC08F00B0E0701DA
:1092A400C26F03D00701630EC26FBC98BC9AD3D3BC
:1092B400880E0A01A46FA60EA56F000EA66F6EECB1
:1092C4000EF0630E0701C26F41EC1AF0BF512A0A77
:1092D40004E1630E0701C26FBAD0BC88BC8A000ED9
:1092E4000A01956F000E966F160E976F880E986F91
:1092F400E80E996F030E9A6FDDEC19F0BC9ABC98D6
:10930400290E0B6E960E0C6E7F0E0D6E0D2EFED773
:109314000C2EFCD70B2EFAD7340E0A01A46FB50E0F
:10932400A56F000EA66F6EEC0EF0D6EC1EF0BF51CA
:109334002A0AD8A48CD0BC88BC8A000E0A01956F76
:10934400000E966F160E976F890E986FE80E996F40
:10935400030E9A6FDDEC19F0BC9ABC98ADEC0DF0DD
:10936400670E0A01A46F090EA56F320EA66FBF0E19
:10937400A76F000EA86FEBEC0DF06D0E0A01956F50
:10938400090E966F4C0E976F000E986F040E996F2E
:10939400000E9A6F19EC10F0670EA46F090EA56FFA
:1093A40021EC0EF07A0E0B6EC10E0C6E810E0D6E5A
:1093B4000D2EFED70C2EFCD70B2EFAD70000000082
:1093C400056B670EA46F090EA56F7B0EA66FBF0E0B
:1093D400A76F000EA86FEBEC0DF0FC0E0A01A46F52
:1093E400090EA56F670EA66F090EA76F28EC0EF085
:1093F40000C07CFA01C07DFAFC0E0A01A46F090EBC
:10940400A56F21EC0EF084EC08F0000E006E0A014A
:109414007D51005C02E17C5100080DE20C0E070155
:10942400C26F050E0A01956F010E966FCAEC17F014
:1094340084EC08F00CD0E10E0A01A46FB80EA56FFD
:10944400000EA66F6EEC0EF0630E0701C26F03D31D
:10945400070E0A01A46FA90EA56F000EA66F6EEC8D
:109464000EF0B00E0901E76F000EE86F0801C46B3F
:10947400C56B000EC55D02E1040EC45D48E2240E16
:10948400C425E16E000EC521E26E4C0EC425E96EC2
:10949400000EC521EA6E6F00A7FFE9FF6F00ABFF66
:1094A400EAFF6F0087FFE1FF6F008BFFE2FF6F00B1
:1094B400BBFFE6FFC4510901E7250A01A46F0801B7
:1094C400C5510901E8210A01A56F4C0E0801C42504
:1094D400E96E000EC521EA6E6F00A7FFE9FF6F0079
:1094E400ABFFEAFF6F00B8FFA6FA9FEC0FF0030E84
:1094F4000B6E080E0C6E770E0D6E0D2EFED70C2E15
:10950400FCD70B2EFAD70801C44BC52BB2D7C451D4
:109514000901E7250A01A46F0801C5510901E821E1
:109524000A01A56FA66B9FEC0FF0240E0A01A46F2D
:10953400000EA56F21EC0EF084EC08F0BC8A520EEC
:109544000B6E2B0E0C6E000E0D6E0D2EFED70C2E18
:10955400FCD70B2EFAD70000BC9ABC9ABC98070122
:10956400C26B79D20D0E0A01A46FB80EA56F000E5E
:10957400A66F6EEC0EF00001B46B0A01A46BA56B30
:10958400A66B9FEC0FF0030E0B6E080E0C6E770E9D
:109594000D6E0D2EFED70C2EFCD70B2EFAD707011D
:1095A4001C6B0A0E0A01A46F000EA56F300EA66F85
:1095B4009FEC0FF0030E0B6E080E0C6E770E0D6E03
:1095C4000D2EFED70C2EFCD70B2EFAD74A6ABC8878
:1095D400BC9A2EEC2DF04AEC1CF003EC10F0F8ECE5
:1095E4000FF0226ACEEC11F0BC8ABC9806EC11F0A4
:1095F400BC9A290E0B6E960E0C6E7F0E0D6E0D2E00
:10960400FED70C2EFCD70B2EFAD7FF0024D20A016A
:10961400F20EA46FA70EA56F000EA66F6EEC0EF0EF
:10962400BC8A000E0A01956F000E966F160E976F96
:10963400880E986FF40E996F010E9A6FDDEC19F095
:10964400BC9A290E0B6E960E0C6E7F0E0D6E0D2EAF
:10965400FED70C2EFCD70B2EFAD7BC8A000E0A01BB
:10966400956F000E966F160E976F880E986FF40E16
:10967400996F010E9A6FDDEC19F0BC9A290E0B6EEE
:10968400960E0C6E7F0E0D6E0D2EFED70C2EFCD793
:109694000B2EFAD7BC8A000E0A01956F000E966F46
:1096A400160E976F880E986FF40E996F010E9A6FCD
:1096B400DDEC19F0BC9A290E0B6E960E0C6E7F0E23
:1096C4000D6E0D2EFED70C2EFCD70B2EFAD70701EC
:1096D400C26BC1D1990E0A01A46FB90EA56F000E19
:1096E400A66F6EEC0EF0010E0101656F010E496E5E
:1096F400010E0001876FBC98BC9A08017C6BBF6B9C
:109704000001B56BDA6B4B6A0701C26B236A4C0E1E
:109714000A01A46F000EA56FE00EA66FC10EA76F1D
:10972400000EA86FEBEC0DF04C6A030E07011C5DF4
:10973400D8A01C2BD90E0A01A46FBE0EA56F000E73
:10974400A66F6EEC0EF0300E07011C250A01C16FE6
:1097540080EC00F0100E0A01A46F000EA56F300E0D
:1097640007011C250A01A66F9FEC0FF0030E0B6E78
:10977400080E0C6E770E0D6E0D2EFED70C2EFCD738
:109784000B2EFAD79E0E0A01A46FBD0EA56F000E14
:10979400A66F6EEC0EF0030E07011C5D73E2000170
:1097A400DA51000A0AE1B60E0A01A46FBB0EA56FD6
:1097B400000EA66F6EEC0EF021D00001DA51000805
:1097C40014E2060EDA5D11E2000E0A01A46FBC0E6B
:1097D400A56F000EA66F6EEC0EF0300E0001DA25B8
:1097E4000A01C16F80EC00F009D0DC0E0A01A46FFD
:1097F400BB0EA56F000EA66F6EEC0EF084EC08F0A5
:10980400840E0A01A46FBF0EA56F000EA66F6EEC46
:109814000EF0330E0A01A46FBD0EA56F000EA66FE5
:109824006EEC0EF00001876B866BBC848B0E0A0114
:10983400A46FB10EA56F000EA66F6EEC0EF0000EB5
:109844000A01A46F000EA56F160EA66F880EA76FEF
:1098540024EC08F0060E0001DB6F000EDC6F010E35
:10986400876F010E496EF40E0B6E820E0C6E050EA0
:109874000D6E0D2EFED70C2EFCD70B2EFAD7876B50
:10988400496A7CD0000E0A01A46F000EA56F160E63
:10989400A66F890EA76F24EC08F05F0E0A01A46F6F
:1098A400B30EA56F000EA66F6EEC0EF0F00E08015D
:1098B400B76F000EB86F090E2A6E090E2B6E090ED3
:1098C4002C6E090E2D6E090E2E6E536A546A556A5B
:1098D400566A576A9B0E0A01A46F000EA56F300EDC
:1098E400A66FC20EA76F000EA86FEBEC0DF0A00ED2
:1098F4000A01A46F000EA56F2B0EA66FC20EA76FF0
:10990400000EA86FEBEC0DF0A50E0A01A46F000E7B
:10991400A56F260EA66FC20EA76F000EA86FEBEC04
:109924000DF0AA0E0A01A46F000EA56F3F0EA66FDC
:10993400C20EA76F000EA86FEBEC0DF0AF0E0A017C
:10994400A46F000EA56F3A0EA66FC20EA76F000E8D
:10995400A86FEBEC0DF0BC94F00E0A01A46FB00EEE
:10996400A56F000EA66F6EEC0EF0010E0001866F5F
:10997400010E476E010E876F010E496E0701C26B1F
:109984006AD084EC08F02F0E0A01A46FB00EA56F04
:10999400000EA66F6EEC0EF0C2C785FA670E0A01C0
:1099A400866F090E876F5FEC21F0670EA46F090EB6
:1099B400A56F21EC0EF00701C26B4DD00701C25117
:1099C400000AD8B482EF3FF0C251010AD8B4CDEFF7
:1099D4003FF0C251020AD8B4ABEF40F0C251030ABF
:1099E400D8B49CEF43F0C251040AD8B47DEF44F0DC
:1099F400C251050AD8B47FEF45F0C251330AD8B436
:109A040095EF46F0C251060AD8B407EF47F0C251A9
:109A1400070AD8B454EF48F0C251080AD8B47FEF0B
:109A240048F0C2510A0AD8B4A5EF48F0C2510B0A53
:109A3400D8B43ED4C2510C0AD8B40AD5C251160ABD
:109A4400D8B490D5C251620AD8B4E1D5C251630AE0
:0C9A5400D8B440D696D780EF3FF0FFD783
:109A600000C019F001C018F0390194A12ED0A4A1B2
:109A70002CD0800E0801BA19006E800E005C02E145
:109A8000010EB95D06E2B290390194910901FB83A0
:109A90000BD0010E0801B95D006E000EBA59016EBF
:109AA00000C0B9F801C0BAF8010E00018825006EA7
:109AB000000E8921016E00C088F001C089F0CF0E30
:109AC000B16E2C0EB06E3901A49119C000F018C00F
:049AD00001F0110090
:10C2600010EE22F0940E006E090E016ED40EF66EE2
:0EC270009A0EF76E000EF86EA1EC39F0120077
:1073540020536F75726365203A20436C61766965CA
:10736400725F4449474954333030305F31384632D4
:10737400374B34325F5F323032322D303332302E7D
:10738400630D0A20416E6E657865733A206D656CF5
:107394006F646965735F636C61766965725F656E5E
:1073A4005F52616D5F323032322D303331395F7468
:1073B4006F5F696E636C7564652E7478740D0A0072
:0873C400524F5547450D0A0028
:019AD4000091
:019AD5000090
:059AD6003132333400C1
:069ADB0000090909090958
:069AE1000000000000007F
:049AE700456E640064
:079AEB00436F6E666967001E
:069AF20056616C6964007E
:019AF800006D
:019AF900006C
:019AFA00006B
:019AFB00006A
:019AFC000069
:019AFD000068
:059AFE003030303000A3
:019B03000061
:069B04000000000000005B
:019B0A00005A
:109B0B000B0201000B0201000B0201004B020100D2
:109B1B00930202004B0202000B02010093020100B0
:0C9B2B004B0201004B0201000B02040081
:019B3700002D
:019B3800002C
:019B3900002B
:029B3A00000029
:029B3C00000027
:0A9B3E003030303000393939390079
:109B48002E2E2E2E002E2E2E2E002E2E2E2E002EB7
:0E9B58002E2E2E002E2E2E2E002E2E2E2E0005
:019B660000FE
:019B670000FD
:109B6800C5A500F0BA009BA800B1A40068A30054E2
:109B78007300C7A6007FB50033AD007AB30067A4B1
:049B88000082A500B2
:019B8C0000D8
:029B8D000000D6
:029B8F007F0055
:0F9B9100ADC10048BF0071BF0048BA005DBA0007
:109BA0003132333435363738393031323334353673
:109BB0000031323334353637383930313233343599
:109BC0003600313233343536373839303132333488
:109BD0003536003132333435363738393031323377
:109BE0003435360031323334353637383930313266
:109BF0003334353600313233343536373839303155
:109C00003233343536003132333435363738393043
:079C10003132333435360018
:019C1700004C
:099C180052656C6169732332008E
:099C210052656C61697323310086
:099C2A0052656C6169732334007A
:099C330052656C61697323330072
:0D9C3C0054657374735F536575696C730034
:029C49003B00DE
:079C4B00436F6461676500CF
:029C52003B00D5
:109C5400C507850821078E04E40359029E064F05B3
:049C64001D05EB01EE
:0A9C6800427566666572310D0A0050
:0B9C7200526573746F72655F4F4E0007
:099C7D0052656C61697323370024
:089C86004D5361626F743D0053
:089C8E005265732E4D43550091
:049C960000000000CA
:029C9A00DC05E7
:019C9C0000C7
:109C9D0047696D6D6547696DFF0133B1009601CD63
:109CAD005F009602676300960000000096026763EE
:109CBD00009601CD5F00960133B1012C000000022A
:109CCD0058000000012C00000000960133B10096F1
:109CDD0001CD5F00960000000096026763009601BB
:109CED00CD5F00960133B1009601599C0096016E2F
:0E9CFD00140096019ADF009601CD5F012CFF46
:109D0B00416C667265644869FF00891C007800002D
:109D1B00000078005B85007800000000F000B70AB7
:109D2B0000F000CD6F003C000000003C00B70A00C3
:109D3B0078000000003C00ACCE0078000000003C36
:109D4B000099D80078000000003C00ACCE007800F1
:109D5B00000000F000B70A0078000000003C00CDC6
:109D6B006F0078000000010E00891C0078000000D5
:109D7B000078005B85007800000000F000B70A0057
:109D8B00F000CD6F003C000000003C00B70A0078EB
:109D9B00000000003C00ACCE0078000000003C004E
:109DAB0099D80078000000003C00ACCE0078000091
:109DBB000000F000B70A0078000000003C00CD6FF7
:109DCB000078000000010E00891C007800000000E4
:109DDB0078005B85007800000000F000D98E0078D9
:109DEB00000000003C01123900F000000000780078
:109DFB00F4460078000000003C00D98E007800008B
:109E0B000000F00112390078000000003C0145D041
:109E1B0000F00000000078012269007800000000CB
:109E2B003C011239007800000000F00145D00078A9
:109E3B00000000003C019ADF00F0000000007801F8
:109E4B006E140078000000003C01599C0078000063
:109E5B0000003C0122690078000000003C0112392F
:109E6B000078000000003C00F44600780000000081
:109E7B003C00D98E0078000000003C00CD6F0078CC
:0B9E8B00000000003C005B8500F0FFC1
:109E96004C617572656C416EFF01B31D00F00244A2
:109EA600D3010E02DC28007F0244D3010E01B31D4C
:109EB600007F0244D3010E02DC28007F0244D30156
:109EC6000E01B31D007F0244D301E0028BA0007F88
:109ED60002DC2800F0028BA000F00244D300F0025E
:109EE6002472010E0244D3007F028BA0010E01B33F
:109EF6001D007F0244D301E002DC28007F0244D328
:109F0600010E01B31D007F0244D301E002DC2800EC
:109F1600F00244D301E001B31D007F0244D300F0F8
:109F2600028BA000F002DC28007F028BA0010E024B
:0A9F3600DC28007F0244D3010EFF77
:109F400050696E6B50616E74686572FF00A2E80024
:109F5000BC00ACCE00BC00000002EE00C1D100BCD1
:109F600000CD6F00BC00000002EE00A2E800BC00C3
:109F7000ACCE00BC000000005E00C1D100BC00CD32
:109F80006F00BC000000005E01123900BC0102EA53
:109F900000BC000000005E00A2E800BC00ACCE00E7
:109FA000BC000000005E0102EA00BC00F44602EEC4
:109FB00000000002EE00E6AF005E00CD6F005E0024
:0F9FC000ACCE005E0099D8005E00ACCE02EEFF82
:109FCF00416374696F6E5F52656C616973FF013332
:109FDF00B1009601CD5F0096026763009600000006
:109FEF000096026763009601CD5F00960133B101C1
:029FFF002CFF35
:10A00100536F6D657468696EFF00D98E012C010272
:10A01100EA012C0102EA012C0102EA012C0102EA07
:10A02100012C012269012C012269012C0122690103
:10A031002C012269012C0145D0012C0145D0012CB4
:10A041000145D0012C0145D0012C01599C012C0165
:10A05100599C012C0145D0012C0102EA012C01225D
:10A0610069012C012269012C01599C012C0145D067
:10A07100096000000004B000E6AF012C0102EA0112
:10A081002C0102EA012C0102EA012C0102EA012C55
:10A09100012269012C012269012C012269012C0193
:10A0A1002269012C0145D0012C0145D0012C01452B
:10A0B100D0012C0145D0012C01599C012C01599C46
:10A0C100012C0145D0012C0102EA012C0122690178
:10A0D1002C012269012C0145D0012C012269096062
:10A0E10000000004B00102EA012C01599C012C017D
:10A0F100599C012C01599C012C01599C012C018373
:10A10100A3012C0183A3012C0183A3012C0183A3AF
:10A11100012C01B31D012C01B31D012C01B31D0143
:10A121002C01B31D012C0205D4012C01CD5F012CA2
:10A1310001B31D012C01CD5F012C01B31D0258019A
:0FA1410083A3012C0183A3096000000004B0FF79
:10A150006178656C66FF00C1D1017700E6AF00D37E
:10A1600000C1D100BC00C1D1005E00F44600BC00BB
:10A17000C1D100BC00ACCE00BC00C1D1017701123E
:10A180003900D300C1D100BC00C1D1005E0133B1A0
:10A1900000BC01226900BC00E6AF00BC00C1D100D8
:10A1A000BC01226900BC0183A300BC00C1D1005ED8
:10A1B00000ACCE00BC00ACCE005E00913400BC0010
:0AA1C000D98E00BC00C1D101D4FF0C
:02A1CA00000093
:01A1CC000092
:01A1CD00038E
:01A1CE000090
:02A1CF002C0161
:02A1D100140573
:10A1D300536D6F6B65206F6E2074686520776174B3
:10A1E300657200FF00891C021800A2E8021800B77C
:10A1F3000A029E00891C021800A2E8021800C1D1BD
:10A20300010C00B70A0218000000021800891C02A2
:10A213001800A2E8021800B70A029E00A2E802187A
:10A2230000891C0218000000042F000000010C002C
:10A23300891C021800A2E8021800B70A029E0089CE
:10A243001C021800A2E8021800C1D1010C00B70AD1
:10A253000218000000021800891C021800A2E8027C
:10A263001800B70A029E00A2E8021800891C02180F
:01A27300FFEB
:01A2740000E9
:02A27500E40102
:10A277004D697373696F6E2020FF0133B1004F0181
:10A2870045D0004F0133B1004F0145D0004F013396
:10A29700B1004F0145D0004F0133B1004F0145D008
:10A2A700004F0133B1004F0133B1004F0145D000DA
:10A2B7004F01599C004F016E14004F0183A3004FBB
:10A2C700019ADF004F019ADF009E000000013C0168
:10A2D7009ADF009E000000013C01E88D009E00000F
:10A2E70000009E022472009E000000009E019ADF7B
:10A2F700009E000000013C019ADF009E0000000163
:10A307003C016E14009E000000009E0183A3009E86
:10A31700000000009E019ADF009E000000013CFF44
:05A3270053746F70008B
:01A32C000030
:01A32D00002F
:01A32E00002E
:01A32F00002D
:02A33000D80E45
:02A33200F00A2F
:01A334000028
:02A33500C40959
:10A33700426F6C65726F00FF01123902EE0112392C
:10A3470001770102EA00BC01123900BC0133B100F8
:10A35700BC01123900BC0102EA00BC00E6AF00BC38
:01A36700FFF6
:10A3680020456570726F6D3A2020456E20466C61FD
:10A378007368204020333130203030303020E020E6
:10A388003331302030334646462E200D0A20436CA8
:10A3980061766965725F31384632374B34325F44D3
:10A3A800494749545F56342D56365F323032322D84
:0CA3B800303331372E696865780D0A00DB
:10A3C4002043616C63756C20646972656374204614
:10A3D400303D20282028666C6F61742920496E6303
:10A3E40072656D656E74202A204E434F315F436C55
:10A3F4006F636B5B4E434F315F436C6F636B5F43C3
:10A40400686F69785D20292F323039373135322E23
:05A41400303B0D0A00C1
:10A419000D0A2050696E2052413720656E20656E05
:10A42900747265652C6C27696E666F206469737434
:10A43900616E7465204232207365726120726574A1
:10A4490072616E736D6973652076696120426C75FE
:0EA4590065546F6F746820484330350D0A005B
:10A467002052656C61697320312C322C332C342CCB
:10A477003520656E206D6F64653D303D546F6767AD
:10A487006C652020313D4D6F6E6F737461626C6532
:10A4970073207375722031207365632C6F752039B3
:0AA4A7003D426C6F7175E90D0A006B
:10A4B10020436F6E66696720626974203A205031CB
:10A4C100384632374B34325F466F73635F496E747F
:10A4D10065726E655F36344D687A5F776974685F5F
:10A4E1004956545F323032322D303231302E63666C
:07A4F100677363680D0A00A8
:10A4F800204E434F31206F70657261746573206917
:10A508006E204669786564204475747920437963C0
:10A518006C65206D6F646520353025202C206469BA
:10A5280076696465206279203220202850464D3DA6
:05A5380030290D0A00AE
:10A53D00200D0A205661726961626C657320657425
:10A54D00205461626C657320656E2052414D2072FE
:10A55D00E9696E697469616C6973E96573202C2012
:10A56D0065742045656570726F6D203D2076696458
:05A57D00E9730D0A0066
:10A5820020436F6E666967204170706C6963617405
:10A59200696F6E20426C7565456C656374726F6E8F
:10A5A200696373203A0D0A20204469676974333065
:10A5B20030305F323032325F303378782E6B776CE6
:03A5C2000D0A007F
:10A5C500204469726563746F7279203A433A5C5F1F
:10A5D5004D696B726F435C5F4D657350726F6A6551
:10A5E50074735F4D696B726F435C434C41564945CB
:10A5F500525F31384632374B34325F323032320DAA
:02A605000A0049
:10A607000D0A20457461706520300D0A2053616979
:10A6170073696520636F6465202050726F67722EBF
:10A62700206F7520636F6465206364652052656CD5
:10A6370061697320283420646967697473290D0A76
:01A647000012
:10A6480020496E69742047656E657261746575721C
:10A65800206465204672657175656E6365204E439A
:10A668004F202C736F7274696520524330203D3E31
:10A678002042757A7A6572207069657A6F0D0A00D2
:10A688000D0A204574617065203131200D0A205370
:10A69800616973697220636F64652050494E202890
:10A6A8003420746F7563686573206E756D2920702A
:0FA6B8007569732056616C69646572200D0A0024
:10A6C70020436C6176696572204D6563616E6971BF
:10A6D7007565204D61747269636520347833207421
:10A6E7006F7563686573206574204C6564205247F5
:0FA6F7004220547269636F6C6F7265200D0A0008
:10A70600203165726520496E697420636172206626
:10A716006C616720616472657373652030783030D0
:10A72600303020454570726F6D20646966666572CB
:0DA73600656E74206465203939200D0A001D
:10A743000D0A20436F6461676573204E4F4E20727C
:10A75300657374697475E973202C207361756620C1
:10A76300636F64652050726F6772202C206361727F
:0CA77300204D5361626F746167653D000A
:10A77F000D0A20546F75636865204E4F4E206E751D
:10A78F006D6572697175652064616E73206C6120EF
:10A79F0073616973696520436F64616765203D3E2E
:0AA7AF0020616C61726D650D0A00F7
:10A7B9000D0A205265737469747565204574617456
:10A7C900206465732052656C61697320312C322CC9
:10A7D900332C34202B20524137203C2D2D20403062
:09A7E9007830304130203D2000A1
:10A7F2002045746170652039383A0D0A20416C6138
:10A80200726D652C2063617220524137206E6F6E2B
:10A8120020636F6E6669677572E920656E20536FFB
:09A822007274696520210D0A0021
:10A82B002043686F697820636F6465203A2030207D
:10A83B003D3E4F4E2F4F4646206F752031203D3EFB
:10A84B004D6F6E6F737461626C6520393D3E206293
:08A85B006C6F7175E90D0A0034
:10A863002052657374697475652064617461732023
:10A87300656570726F6D2020436F64652050726F41
:10A8830067722E206574203520436F6465732052F0
:08A89300656C6169730D0A0098
:10A89B002050726F6A6574203A436C6176696572F9
:10A8AB005F31384632374B34325F44494749545F46
:10A8BB00333030305F323032322D303378782E6D8A
:07A8CB00637070690D0A00C3
:10A8D2002063686F6978206D6F6465204254203070
:10A8E2003D696E746572646974202C312D3E504945
:10A8F200432D3E42542C2032205049433C2D3E20D1
:05A9020042540D0A00A3
:10A907000D0A204574617065203132200D0A204EF2
:10A91700657720636F64652050494E2076616C69C6
:10A9270064E920657420736175766567617264E90F
:04A93700203A2000A2
:10A93B002052415A20466C616720656570726F6DBD
:10A94B00203D3E20546F757465203165726520493A
:10A95B006E6974206E6563657361697265200D0A9B
:01A96B0000EB
:10A96C000D0A205374657020333A20536169736962
:10A97C0072204E6F757665617520636F646520502B
:10A98C00726F6772616D6D6174696F6E2E0D0A0066
:10A99C000D0A2045746174206465732072656C61C6
:10A9AC00697320782C312C322C332C342C65742088
:10A9BC00524137202040307830304130203A20004E
:10A9CC000D0A20526573746974756520436F6E6649
:10A9DC006967732064657320352052656C616973F7
:10A9EC00203C2D2D2040307830303830203D200058
:10A9FC002020506173206427657874656E73696FCD
:10AA0C006E20456E747265652F536F727469652084
:10AA1C0061766563205241375F417578200D0A00DD
:10AA2C002041636365732070726F6772616D6D6135
:10AA3C0074696F6E2076696120636F646520507253
:0FAA4C006F67722020656E2052414D200D0A0069
:10AA5B0020496E69742064652062617365204E43E2
:10AA6B004F2028766F69722070616765203435340A
:0FAA7B002064617461736865657429200D0A0099
:10AA8A000D0A205265737469747565204574617482
:10AA9A00206D6F646966203620636F646573203C9D
:0EAAAA002D2D2040307830303930203D2000F6
:10AAB8002043686F6978204D6F6465204254202CCC
:10AAC800417474656E746520546F756368652056AB
:0DAAD800616C69646174696F6E200D0A0085
:10AAE5000D0A204D656D6F20536F72746965205294
:10AAF500656C616973203620636F646573203C2D36
:0DAB05002D2040307830304130203A2000C3
:10AB120020496E6372656D656E743D323531362043
:10AB220020202D3E28666C6F61742920496E637265
:0CAB3200656D656E742029203D3E2000FA
:10AB3E0020706F75722052455354415552415449FD
:10AB4E004F4E207669612073657175656E63652061
:0CAB5E00636C617669657220200D0A00AE
:10AB6A0020417474656E74652076616C69646174E1
:10AB7A00696F6E20494420746F756368652070613F
:0CAB8A0072207665727465202A0D0A00A6
:10AB96000D0A20417474656E74652076616C696473
:10ABA6006174696F6E2070617220746F7563686579
:0BABB60020566572746520200D0A0017
:10ABC1000D0A20457461706520350D0A20536169B5
:10ABD10073696520436F6E66696720706F757220B7
:0BABE1006C652052656C6169732000F8
:10ABEC005361757665676172646520636F64652077
:10ABFC0050726F677220656E2052414D2065742033
:0AAC0C00454550524F4D200D0A003F
:10AC16000D0A20537465702035203A2053617576ED
:10AC260065676172646520636F6465732020656E75
:0AAC360020656570726F6D0D0A0055
:10AC40000D0A205265737469747565204D6F6465D3
:10AC500020426C7565546F6F7468203C2D2D204028
:0AAC6000307830304330203D2000F2
:10AC6A000D0A2045746170653D31300D0A204D6F23
:10AC7A0064696620436F64652050494E20426C75B2
:09AC8A0065546F6F74680D0A0037
:10AC930020416E6E756C6174696F6E2073616973A8
:10ACA300696520766961202876696120746F756310
:08ACB30068652023200D0A0052
:10ACBB002A5541757820496E3D312A3B2A42523044
:10ACCB004732353542302A3B2A57202A3B2A4E52EF
:08ACDB0030473042302A3B00F3
:10ACE3002A5541757820496E3D302A3B2A4252321B
:10ACF3003535473042302A3B2A57202A3B2A4E52C9
:08AD030030473042302A3B00CA
:10AD0B0020416E6E756C6174696F6E20736169732F
:10AD1B00696520766961202876696120746F756397
:08AD2B0068652023200D0A00D9
:10AD3300204E434F206F75747075742073757220A5
:10AD4300524330202D3E2042757A7A657220506935
:07AD5300657A7A6F0D0A001A
:10AD5A000D0A204574617065202038200D0A2052A2
:10AD6A006573746175726174696F6E2076696120AA
:07AD7A0049443D380D0A00B9
:10AD81000D0A20526573746175726174696F6E206A
:10AD910076696120425020524331206F75204279FB
:07ADA100204169720D0A0058
:10ADA8002045746170652032200D0A205361697353
:10ADB8006972206C6520636F6465204944203020E7
:07ADC800E02020390D0A0014
:10ADCF002A5752373D4F46462A3B2A4E5232353587
:10ADDF00473042302A3B2A55202A3B2A42523047DD
:06ADEF003042302A3B0057
:10ADF5000D0A2045746174206D6F646966203620E4
:10AE0500636F646573203C2D2D20403078303039D8
:05AE150030203A20008E
:10AE1A0020417474656E746520746F75636865206B
:10AE2A0076616C69646174696F6E207665727465A7
:05AE3A00202A0D0A00B2
:10AE3F0020417474656E746520746F756368652046
:10AE4F0076616C69646174696F6E20766572746582
:05AE5F00202A0D0A008D
:10AE640020417474656E746520746F756368652021
:10AE740076616C69646174696F6E2076657274655D
:05AE8400202A0D0A0068
:10AE890020417474656E746520746F7563686520FC
:10AE990076616C69646174696F6E20766572746538
:05AEA900202A0D0A0043
:10AEAE00204D6F646520636F6E6669672072656CF6
:10AEBE00616973203C2D2D204030783030383020A1
:04AECE003A20200006
:10AED20020417474656E746520746F7563686520B3
:10AEE20076616C69646174696F6E207665727465EF
:04AEF200200D0A0025
:10AEF60020436F6D706172652061766563205241F3
:10AF06004D2C20524F4D2C20657420454570726F94
:04AF16006D0D0A00B3
:10AF1A0020417474656E746520546F75636865208A
:10AF2A0056657274652056616C69646174696F6EE6
:04AF3A00200D0A00DC
:10AF3E000D0A20526573746974756520436F6465DC
:10AF4E002050494E203C2D2D20403078303042305C
:04AF5E00203D200072
:10AF62000D0A204574617065202037200D0A2041AA
:10AF72006374696F6E207375722072656C61697398
:03AF820020230089
:10AF850020496E69742054696D6572345F666F720D
:10AF95005F416C61726D652020302C3573656320CF
:03AFA5000D0A0092
:10AFA800200D0A205374657020323A20546F75635F
:10AFB80068652056657274652065786967E965205B
:03AFC8000D0A006F
:10AFCB0020436F646520706F7572204E6F757665C8
:10AFDB00617520636F64652052454C414953200DC8
:02AFEB000A005A
:10AFED000D0A20436F6E66696720436465205265C4
:10AFFD006C616973204030783030383020203A2031
:01B00D000042
:10B00E000D0A2045746174204D6F64696620646575
:10B01E0020436F64652040307830303930203A203C
:01B02E000021
:10B02F0020424144204574617065202120414E4FDC
:10B03F004D414C49452021202045746170653D20CC
:01B04F000000
:10B050000D0A204572726F722073757220636F64DF
:10B06000652050726F6720656E2052414D203A2056
:01B0700000DF
:10B071000D0A204D6F646520426C7565546F6F74C5
:10B0810068203C2D2D2040307830304330203A204C
:01B0910000BE
:10B0920020436F64652050726F677220657420636D
:10B0A2006F64657320352072656C6169730D0A00E7
:10B0B20020524137206E6F6E20636F6E666967752E
:0FB0C20072E920656E20534F525449450D0A0024
:10B0D1000D0A205374657020343A20546F756368EB
:0FB0E100652056657274652065786967E96500BA
:10B0F000205265706F727420416C61726D652044DE
:0FB10000697374616E7465203D4F55490D0A00E7
:10B10F000D0A2056616C696465722076696120545E
:0FB11F006F75636865205665727465200D0A00B0
:10B12E00204572726F72203A204475706C696361AB
:0FB13E00746120746F7576E9206378203D2000DE
:10B14D00200D0A205374657020313A20436F6465D9
:0FB15D0020494420302065786967E9200D0A00F9
:10B16C0020506F6C6172697479203D3020284E6FCD
:0FB17C007420696E76657274656429200D0A006F
:10B18B00205265706F727420416C61726D65204442
:0FB19B00697374616E7465203D4E4F4E0D0A004E
:10B1AA0020706F7572204E6F757665617520636FBA
:0FB1BA0064652050494E2048433036200D0A006E
:10B1C9002A57202A3B2A4E5230473042302A3B2AFE
:0FB1D90055202A3B2A425230473042302A3B0051
:10B1E8000D0A204E4F4E204D6F64696669E9202E86
:0EB1F8003D3E20696E6163746966200D0A0099
:10B206000D0A204175746F7269736174696F6E20DF
:0EB2160042542040307830304330203A20003F
:10B2240020706F7572204E6F757665617520636F3F
:0EB234006465202052656C616973200D0A006C
:10B2420020417474656E74652031202066726170CD
:0EB25200706520636C6176696572200D0A00DC
:10B2600020417474656E746520342066726170705C
:0DB27000657320636C61766965720D0A00DC
:10B27D002052656C656374757265206461746173C9
:0DB28D0020656570726F6D203A200D0A007B
:10B29A0020417474656E7465203420667261707022
:0DB2AA00657320636C61766965720D0A00A2
:10B2B700203D3E2052415A20436F646167652062FA
:0CB2C700792054696D654F75740D0A0004
:10B2D30020436F6D706172652C2061766563202059
:0CB2E300636F6465205573696E65200080
:10B2EF0020202E2E636F64652052656C6169732078
:0CB2FF004F4B20656E2052414D0D0A009F
:10B30B000D0A20417474656E746520546F75636803
:0CB31B0065205665727465202A0D0A003A
:10B327000D0A20436F64652050494E20484330364C
:0CB337002040307830304230203A2000B6
:10B34300203D3E2052415A20436F6461676520626D
:0CB35300792054696D654F75740D0A0077
:10B35F00416C61726D6520426C6F7175616E7465C1
:0BB36F0020313230207365630D0A00AE
:10B37A0020557361676520496E74657272757074C1
:0BB38A0020566563746F72730D0A009B
:10B395002E31342E372E2E2E2A2E32352E382E2EA5
:0BB3A5002E302E33362E392E2E2E2394
:10B3B0000D0A204572726F72207375722056616C8F
:0BB3C00069646174696F6E200D0A0063
:10B3CB000D0A205072656D6965726520496E69744E
:0BB3DB002E20537465703D300D0A00F9
:10B3E6000D0A20436F64652050696E203C2D2D2088
:0BB3F60040307830304230203A200018
:10B401002020646F75626C6F6E20636F64652055D8
:0BB4110073696E652030303030200081
:10B41C00202E49442072656C616973206E6F6E201A
:0AB42C0074726F7576E90D0A2000B6
:10B436000D0A205374657020393A205265636F6D8A
:0AB446006D656E636572200D0A004B
:10B4500020706F7572204E6F757665617520636F11
:0AB4600064652070726F670D0A002A
:10B46A002A4F4F7576657274202A3B2A525232351A
:0AB47A00354732353542302A3B00D9
:10B484002A4F4F7576657274202A3B2A5252323500
:0AB49400354732353542302A3B00BF
:10B49E00204364652065787465726E65206465204E
:09B4AE0072656C616973203D00B8
:10B4B7002046696E206465203165726520696E6972
:09B4C70074202E2E4F4B0D0A00DB
:10B4D0002056616C69646174696F6E204944203D37
:09B4E000203020204F4B0D0A0022
:10B4E9002053657175656E63652052455345542037
:09B4F9005573696E65200D0A000F
:10B50200204D5361626F74616765203C2D2D2020B0
:09B512004030783130203D20006A
:10B51B000D0A20436F6E6E656374696F6E207375D1
:09B52B007220484330360D0A007D
:10B534000D0A20546F756368652056657274652022
:09B5440065786967E9650D0A00EC
:10B54D0020457820636F64652050696E20656E20FC
:09B55D00456570726F6D203D0020
:10B566002A562056657273696F6E20323032322D3C
:09B57600303332302A3B0D0A008B
:10B57F002031384632374B34322055415254312026
:09B58F003131353230300D0A0073
:10B5980020526573756C7461742046726571204F12
:09B5A80075747075743D202000DB
:10B5B1002A5541757820496E3D302A3B2A42523244
:09B5C1003535473042302A3B00C9
:10B5CA002A5541757820496E3D312A3B2A4252302C
:09B5DA004732353542302A3B00AE
:10B5E3000D0A4F4B2C204E657720436F6E666967BB
:09B5F3002052656C6169732000AF
:10B5FC000D0A2045746174204250205265737461A9
:09B60C0075726174696F6E3D00F6
:10B615002A4A52333D4C6F636B2A3B2A45523047C9
:08B625003042302A3B0D0A00FF
:10B62D00204D6F6465205465737420536575696C86
:08B63D0073204144430D0A0093
:10B645002A4B52343D4C6F636B2A3B2A4652304796
:08B655003042302A3B0D0A00CF
:10B65D002A4F416374697665202A3B2A525232354E
:08B66D0035473042302A3B0052
:10B675002A4852313D4F4E2A3B2A435230473042E9
:08B685003235352A3B0D0A00A5
:10B68D002A4A52333D4F4E2A3B2A455230473042CB
:08B69D003235352A3B0D0A008D
:10B6A5002A4952323D4C6F636B2A3B2A445230473C
:08B6B5003042302A3B0D0A006F
:10B6BD002A4952323D4F4E2A3B2A4452304730429E
:08B6CD003235352A3B0D0A005D
:10B6D5002A4852313D4C6F636B2A3B2A435230470F
:08B6E5003042302A3B0D0A003F
:10B6ED0020466C616720456570726F6D2040307823
:08B6FD0030303030203D200008
:10B705002A482052313D4F4E202A3B2A435230478A
:08B7150032353542302A3B00B9
:10B71D002A4B2052343D4F46462A3B2A465232355B
:08B72D0035473042302A3B0091
:10B735002A492052323D4F46462A3B2A4452323549
:08B7450035473042302A3B0079
:10B74D002A492052323D4F4E202A3B2A445230473F
:08B75D0032353542302A3B0071
:10B765002A4B2052343D4F4E202A3B2A4652304721
:08B7750032353542302A3B0059
:10B77D002A4A2052333D4F4E202A3B2A455230470C
:08B78D0032353542302A3B0041
:10B795002A4A2052333D4F46462A3B2A45523235E6
:08B7A50035473042302A3B0019
:10B7AD002A4F416374697665202A3B2A52523235FD
:08B7BD0035473042302A3B0001
:10B7C5002A572052373D4F46462A3B2A4E5232359C
:08B7D50035473042302A3B00E9
:10B7DD0020526573746974756520506172616D6571
:08B7ED0074726167650D0A002A
:10B7F5002A4B52343D4C6F636B2A3B2A46523047E5
:08B805003042302A3B0D0A001D
:10B80D00202052455345542076696120636F64654D
:08B81D002049443D390D0A00E9
:10B825002A4B52343D4F4E2A3B2A4652304730422E
:08B835003235352A3B0D0A00F3
:10B83D002A5752373D4C6F636B2A3B2A4E52304785
:08B84D003042302A3B0D0A00D5
:10B855002A5752373D4F4E2A3B2A4E5230473042E7
:08B865003235352A3B0D0A00C3
:10B86D002A482052313D4F46462A3B2A4352323513
:08B87D0035473042302A3B0040
:10B885002A4F4665726D65202A3B2A52523047324F
:07B89500353542302A3B006B
:10B89C002A572052373D4C6F636B2A3B2A4E52304D
:07B8AC00473042302A3B0047
:10B8B3002A572052373D4F4E2A3B2A4E52304732A9
:07B8C300353542302A3B003D
:10B8CA000D0A204572726F722073757220636F645D
:07B8DA00652049440D0A003E
:10B8E1000D0A2042616420636F6E662050494E202C
:07B8F100636F64650D0A009E
:10B8F8002A4B2052343D4C6F636B2A3B2A46523008
:07B90800473042302A3B00EA
:10B90F002A482052313D4C6F636B2A3B2A435230F9
:07B91F00473042302A3B00D3
:10B926002A4F4665726D65202A3B2A5252304732AD
:07B93600353542302A3B00C9
:10B93D002A4A2052333D4C6F636B2A3B2A455230C5
:07B94D00473042302A3B00A5
:10B954002A492052323D4C6F636B2A3B2A445230B1
:07B96400473042302A3B008E
:10B96B002053746172742054696D656F7574203344
:07B97B00207365630D0A0053
:10B9820020417520636C616972206465206C6120BE
:07B992006C756E650D0A00E3
:10B999000D0A204574617065203939202020416CD9
:07B9A90061726D650D0A00DB
:10B9B000204F4E2070656E64616E74203153656354
:06B9C000202E2E2E2000B7
:10B9C600204D5361626F7461676520403078303076
:06B9D6003130203D20008D
:10B9DC000D0A20436F6465206163746966202E2E06
:06B9EC00204F4B0D0A0084
:10B9F200204D5361626F746167652040203078305A
:06BA0200303130203D0050
:10BA0800205265706F727420416C61726D653D20C3
:06BA18004E4F4E0D0A0026
:10BA1E002A4F202E2E2E2E2E2A3B2A5252304730BF
:05BA2E0042302A3B003C
:10BA330020496E69742054696D657231203130304C
:05BA43006D530D0A0027
:10BA480020204D46494E544F53432028353030204E
:05BA58006B487A290093
:10BA5D00204D46494E544F53432F34202833312027
:05BA6D006B487A29007E
:10BA72002050422064652056616C69646174696F6C
:05BA82006E200D0A001A
:10BA87000D0A2050726573656E746174696F6E205C
:05BA97003A200D0A0039
:10BA9C00202E2E20657869737420656E20456570A4
:05BAAC00726F6D200027
:10BAB10020536575696C73204F757672616E7420C1
:05BAC1004261733D002D
:10BAC600204574617420526573746175726174697E
:05BAD6006F6E203D0031
:10BADB0020536575696C73204973737565732020EA
:05BAEB004261733D0003
:10BAF000204D696B726F432070726F20372E363085
:04BB0000200D0A000A
:10BB040020536575696C7320416C61726D652042C8
:04BB140061733D001C
:10BB18000D0A2052656C61697320524137204F46E7
:04BB2800460D0A00BC
:10BB2C002A4F2E2E2E2E202A3B2A5252304730429C
:04BB3C00302A3B0070
:10BB40002A4F2E2E2E2E202A3B2A52523047304288
:04BB5000302A3B005C
:10BB5400205265616420666C616720403078303023
:04BB6400203D200060
:10BB6800002474980024749800007A8D002474913D
:04BB78000030728D9A
:10BB7C002E4964783D2A5436353533352A3B2A47CD
:04BB8C00302A3B0020
:10BB9000204144434C434B2072656769737472655E
:03BBA000203D0045
:10BBA30020202E2E20657869737420656E20524103
:03BBB3004D200022
:10BBB6002049442050726F6772616D6D6174696FC0
:03BBC6006E2000EE
:10BBC900202D3E2052617A207361626F746167652E
:03BBD9000D0A0052
:10BBDC00204D61757661697320636F6465204944FB
:02BBEC00200037
:10BBEE00204E434F31434C4B2063686F6978203DA4
:02BBFE00200025
:10BC000020494420706F75722052656C6169732001
:02BC100023000F
:10BC12002056616C69646174696F6E204F4B200D10
:02BC22000A0016
:10BC240020536575696C7320414443205242350D9D
:02BC34000A0004
:10BC36002A4820202A3B2A435230473042302A3BAA
:01BC460000FD
:10BC47000D0A20457461742050696E205242373DB9
:01BC570000EC
:10BC5800206D6F646520426C6F7175E9204F464610
:01BC680000DB
:10BC690020416C61726D652073696D706C650D0A98
:01BC790000CA
:10BC7A000D0A2053617576652043646573200D0AA9
:01BC8A0000B9
:10BC8B00526573746F7265206279204169720D0A77
:01BC9B0000A8
:10BC9C002A4B20202A3B2A465230473042302A3B3E
:01BCAC000097
:10BCAD002A4A20202A3B2A455230473042302A3B2F
:01BCBD000086
:10BCBE0020466C6167204020307830303030203D97
:01BCCE000075
:10BCCF002A5720202A3B2A4E5230473042302A3BF7
:01BCDF000064
:10BCE0002A4920202A3B2A445230473042302A3BFE
:01BCF0000053
:10BCF100206D6F6465204D6F6E6F737461626C654A
:01BD01000041
:10BD02002052413720656E20736F727469650D0A87
:01BD12000030
:10BD1300303132333435363738394142434445467E
:10BD23000D0A20457461706520203531200D0A000D
:10BD33006E6F6E20626C6F7175616E74650D0A00B3
:10BD4300204D656C6F6469652073697A65203D00D9
:0FBD53002E4964783D2A5436353533352A3B0066
:0FBD6200204E756D65726F20204944203D2000F2
:0FBD71000D0A20636F64652050726F67722E0099
:0FBD8000202E2E2E2054696D654F75740D0A000C
:0FBD8F00202E457863657074696F6E203A20002E
:0FBD9E002020436465456E436F757273203A0031
:0FBDAD002E4370743D2A5436353533352A3B000A
:0EBDBC0020436F6E64616D6EE921200D0A0058
:0EBDCA0020636F64652072656C6169732000F0
:0EBDD80020496E6372656D656E74203D20001B
:0EBDE6002065742050696E205242363D2000C8
:0EBDF400204E657720436F64616765203D0037
:0DBE02002056616C69646174696F6E2000E8
:0DBE0F000D0A20457461706520360D0A0093
:0DBE1C0020646966666572656E740D0A002B
:0DBE2900200D0A2E2E20424144210D0A005A
:0DBE36000D0A20457461706520340D0A006E
:0DBE4300466C61675F456570726F6D3D0074
:0DBE5000206D6F6465204F6E2F4F666600F9
:0DBE5D000D0A20457461706520330D0A0048
:0DBE6A0020487A202C4475726565203D004B
:0DBE77000D0A20457461706520310D0A0030
:0DBE840020467261707065204EB0202000D5
:0CBE9100204D6F6465204254203D2000CD
:0CBE9D005265736574204D43550D0A007A
:0CBEA900200D0A2E2E204F4B210D0A0008
:0CBEB50020467261707065204EB02000C5
:0CBEC1002070756973204F46460D0A0082
:0CBECD00204D5361626F746167653D0099
:0CBED900204D5361626F746167653D008D
:0BBEE500204672617070652023200071
:0BBEF000204D656C6F64696520230025
:0BBEFB000D0A436F75636F750D0A00A0
:0BBF06000D0A436F75636F750D0A0094
:0BBF11000D0A2052656C61697320006E
:0BBF1C000D0A20436F646167653D0063
:0BBF27002020436F64616765203D002F
:0BBF320041542B50494E2E2E2E2E00A5
:0BBF3D002020436F64616765203D0019
:0BBF4800204846494E544F5343200050
:0ABF53002A5A36353533362A3B00F2
:0ABF5D00204465666175740D0A004A
:0ABF670020546F75636865203D00EB
:0ABF7100204C46494E544F53430044
:09BF7B004F4B73657450494E00F0
:09BF840020416C61726D65200022
:09BF8D0020436F646167653D000B
:09BF9600206964656D200D0A00AC
:09BF9F002052656C6169732000F9
:09BFA8002044454255540D0A00E5
:09BFB1002076657269662020000B
:08BFBA00524F5547450D0A00E6
:08BFC200524F5547450D0A00DE
:08BFCA00524F5547450D0A00D6
:08BFD200524F5547450D0A00CE
:08BFDA00524F5547450D0A00C6
:08BFE200524F5547450D0A00BE
:08BFEA00524F5547450D0A00B6
:08BFF200524F5547450D0A00AE
:08BFFA00524F5547450D0A00A6
:08C00200524F5547450D0A009D
:08C00A00524F5547450D0A0095
:08C01200010204081020408027
:08C01A00524F5547450D0A0085
:08C022004A41554E450D0A008C
:08C02A00524F5547450D0A0075
:08C03200524F5547450D0A006D
:07C03A002043646520230090
:07C041004E4F49520D0A00A9
:07C048004E4F49520D0A00A2
:07C04F00564552540D0A0092
:07C0560020736F69742000E4
:07C05D00564552540D0A0084
:07C06400424C45550D0A0096
:07C06B004E4F49520D0A007F
:07C072004E4F49520D0A0078
:07C079004E4F49520D0A0071
:07C08000204364652023004A
:07C087004E4F49520D0A0063
:07C08E004E4F49520D0A005C
:07C09500204F46460D0A0092
:07C09C002E2E4F4B0D0A0090
:07C0A300202D3E204C3D0062
:07C0AA002E2E4F4B0D0A0082
:07C0B10020546573743D008B
:07C0B8004E4F49520D0A0032
:07C0BF004E4F49520D0A002B
:07C0C60020546573743D0076
:07C0CD00424C45550D0A002D
:07C0D4002E2E4F4B0D0A0058
:07C0DB00564552540D0A0006
:07C0E2002E2E4F4B0D0A004A
:07C0E9002E2E4F4B0D0A0043
:07C0F00020564D656D3D0077
:07C0F7004E4F49520D0A00F3
:07C0FE0020546573743D003E
:07C10500424C45550D0A00F4
:07C10C004E4F49520D0A00DD
:07C113004E4F49520D0A00D6
:07C11A004E4F49520D0A00CF
:07C1210020486175743D0028
:07C1280020486175743D0021
:07C12F0020486175743D001A
:07C136004E4F49520D0A00B3
:07C13D0020546573743D00FE
:07C144004E4F49520D0A00A5
:07C14B0020546573743D00F0
:07C1520020546573743D00E9
:07C1590020546573743D00E2
:07C160002E2E4F4B0D0A00CB
:07C167002043646520230062
:07C16E00424C45550D0A008B
:07C175004E4F49520D0A0074
:07C17C004E4F49520D0A006D
:07C18300204F46460D0A00A3
:07C18A004E4F49520D0A005F
:07C191004E4F49520D0A0058
:07C198004E4F49520D0A0051
:07C19F00424C45550D0A005A
:07C1A6004E4F49520D0A0043
:06C1AD0020464F53430041
:06C1B3004144433D200061
:06C1B900204F4E0D0A00AC
:06C1BF00204F4B0D0A00A9
:06C1C500204F4B0D0A00A3
:06C1CB0020487A0D0A0075
:05C1D1003030303000A9
:05C1D6002E2E2E2E00AC
:05C1DB002E2E2E2E00A7
:05C1E0002020202000DA
:05C1E5002E2E2E2E009D
:05C1EA002E2E2E2E0098
:05C1EF00313233340081
:05C1F40031323334007C
:05C1F9002E2E2E2E0089
:05C1FE002E2E2E2E0084
:05C203002E2E2E2E007E
:05C208002E2E2E2E0079
:05C20D002E2E2E2E0074
:05C212002E2E2E2E006F
:05C217002E2E2E2E006A
:05C21C002E2E2E2E0065
:05C221002E2E2E2E0060
:05C226002E2E2E2E005B
:05C22B002E2E2E2E0056
:05C230002E2E2E2E0051
:05C235002E2E2E2E004C
:05C23A002E2E2E2E0047
:05C23F002E2E2E2E0042
:04C244002020200096
:03C248004154005E
:03C24B004F4B0056
:03C24E000D0A00D6
:03C251002040008A
:03C254002A3B0082
:03C257002A5A0060
:03C25A0020400081
:03C25D002040007E
:020000040030CA
:0A00000004092DA70B3F9F0F01001C
:0200000400F00A
:020000040031C9
:100000000000FFFFFF00466C616700FFFFFFFFFF7E
:100010003000000000005361626F74616765730017
:10002000303030300000436F64652050726F6700DD
:100030002E2E2E2E000052656C6169732023310034
:100040002E2E2E2E000052656C6169732023320023
:100050002E2E2E2E000052656C6169732023330012
:100060002E2E2E2E000052656C6169732023340001
:100070002E2E2E2E000052656C61697320233700EE
:1000800030393939393900436F6E6669672052005B
:100090003030303030300056616C696420524C0092
:1000A000303030303030004574617420524C0000E4
:1000B000313233340000436F64652050494E0000F4
:1000C0003000000000004D6F6465204254000000C5
:1000D0004449474954343030305F323032320D0AAF
:1000E0000000FFFFFFFFFFFFFFFFFFFFFFFFFFFF1E
:1000F00000FFFFFFFFFFFFFFFFFFFFFFFFFFFFFF0F
:1001000000FFFFFFFFFFFFFFFFFF00FFFFFFFFFFFD
:1001100000FFFFFFFFFFFFFFFFFFFFFFFFFFFFFFEE
:1001200000FFFFFFFFFFFFFFFFFFFFFFFFFFFFFFDE
:1001300000FFFFFFFFFFFFFFFFFFFFFFFFFFFFFFCE
:10014000000000000000000000FFFFFFFFFFFFFFB6
:1001500000FFFFFFFFFFFFFFFFFFFFFFFFFFFFFFAE
:1001600000FFFFFFFFFFFFFFFFFFFFFFFFFFFFFF9E
:1001700000FFFFFFFFFFFFFFFFFFFFFFFFFFFFFF8E
:1001800000FFFFFFFFFFFFFFFFFFFFFFFFFFFFFF7E
:1001900000FFFFFFFFFFFFFFFFFFFFFFFFFFFFFF6E
:1001A00000FFFFFFFFFFFFFFFFFFFFFFFFFFFFFF5E
:1001B00000FFFFFFFFFFFFFFFFFFFFFFFFFFFFFF4E
:1001C00000FFFFFFFFFFFFFFFFFFFFFFFFFFFFFF3E
:1001D00000FFFFFFFFFFFFFFFFFFFFFFFFFFFFFF2E
:1001E000FFFFFFFFFFFFFFFFFFFFFFFFFFFFFFFF1F
:1001F000FFFFFFFFFFFFFFFFFFFFFFFFFFFFFFFF0F
:10020000FFFFFFFFFFFFFFFFFFFFFFFFFFFFFFFFFE
:10021000FFFFFFFFFFFFFFFFFFFFFFFFFFFFFFFFEE
:10022000FFFFFFFFFFFFFFFFFFFFFFFFFFFFFFFFDE
:10023000FFFFFFFFFFFFFFFFFFFFFFFFFFFFFFFFCE
:10024000FFFFFFFFFFFFFFFFFFFFFFFFFFFFFFFFBE
:10025000FFFFFFFFFFFFFFFFFFFFFFFFFFFFFFFFAE
:10026000FFFFFFFFFFFFFFFFFFFFFFFFFFFFFFFF9E
:10027000FFFFFFFFFFFFFFFFFFFFFFFFFFFFFFFF8E
:10028000FFFFFFFFFFFFFFFFFFFFFFFFFFFFFFFF7E
:10029000FFFFFFFFFFFFFFFFFFFFFFFFFFFFFFFF6E
:1002A000FFFFFFFFFFFFFFFFFFFFFFFFFFFFFFFF5E
:1002B000FFFFFFFFFFFFFFFFFFFFFFFFFFFFFFFF4E
:1002C000FFFFFFFFFFFFFFFFFFFFFFFFFFFFFFFF3E
:1002D000FFFFFFFFFFFFFFFFFFFFFFFFFFFFFFFF2E
:1002E000FFFFFFFFFFFFFFFFFFFFFFFFFFFFFFFF1E
:1002F000FFFFFFFFFFFFFFFFFFFFFFFFFFFFFFFF0E
:1003000000FFFFFFFFFFFFFFFFFFFFFFFFFFFFFFFC
:10031000FFFFFFFFFFFFFFFFFFFFFFFFFFFFFFFFED
:10032000FFFFFFFFFFFFFFFFFFFFFFFFFFFFFFFFDD
:10033000FFFFFFFFFFFFFFFFFFFFFFFFFFFFFFFFCD
:10034000FFFFFFFFFFFFFFFFFFFFFFFFFFFFFFFFBD
:10035000FFFFFFFFFFFFFFFFFFFFFFFFFFFFFFFFAD
:10036000FFFFFFFFFFFFFFFFFFFFFFFFFFFFFFFF9D
:10037000FFFFFFFFFFFFFFFFFFFFFFFFFFFFFFFF8D
:10038000FFFFFFFFFFFFFFFFFFFFFFFFFFFFFFFF7D
:10039000FFFFFFFFFFFFFFFFFFFFFFFFFFFFFFFF6D
:1003A000FFFFFFFFFFFFFFFFFFFFFFFFFFFFFFFF5D
:1003B000FFFFFFFFFFFFFFFFFFFFFFFFFFFFFFFF4D
:1003C000FFFFFFFFFFFFFFFFFFFFFFFFFFFFFFFF3D
:1003D000FFFFFFFFFFFFFFFFFFFFFFFFFFFFFFFF2D
:1003E00056657231372D30332D323032320D0A00DE
:1003F0007061756C666A756A6F40667265652E001D
:00000001FF
